:20000000004B002085510100FDC90110FDC90110FDC90110FDC90110FDC90110FDC9011094
:1C002000FDC90110FDC90110FDC90110FDC90110FDC90110FDC901103BCA0110A4
:20003C00BD0400214D040021810400218504002121050021A10500215106002179060021DA
:20005C00F8B51047F8B50E4600210125AD0430470A48037800F00FF89B070BD0124C2078D9
:20007C00FF2807D0FF2121700E490F24240220436031C882F8BDF8B5014800476B02002147
:20009C00E54C0000094801E00848000C064C05492278FF2A01D1CA7A22706031C8827046E9
:2000BC00801C004700620840C8060021070F0808F0B4084710B501480047000089090000A8
:2000DC0070B503461546012906D0002906D0114A2846FFF7B5FF70BD0F4800E00F480524E5
:2000FC00834203D84008641E002CF9DCE340012040031818820B012907D006490023803111
:20011C002846FFF79FFFE0B270BD0249044B6C31F6E70000835C0000A0BC862300830D2357
:20013C0098060021F8B51A4E0546716B1948CC09E401002D11D01849097802290FD0007B18
:20015C00044372B60120154F4002B847114820380088C109C90704D016E0C07AF0E7407BE5
:20017C00EEE70F497463CC61400AC0070CD001208003316B002D01D0014300E081430846D1
:20019C0031630749403948630020B84762B6F8BD80020021880000219B0200217B3F00008B
:2001BC004040044010B5224A0021516121498968C90009D42149204BCA0598424B6B01D84D
:2001DC00134300E093434B631D49FFF771FF10BD38B51A4D287F002827D11A480088C009E2
:2001FC00C00722D1124C606900281ED1684600F04FF868460078012817D168464078102831
:20021C0013D208206061686A4009400120600E4A0021D1620D4A0221116001210843206094
:20023C00032108436862206038BD0948804738BD00400440180000210000930880020021EC
:20025C00CF680000680000210011044080E200E0C33B00000749002800D00420064A72B649
:20027C000978C90701D0105800E0802062B640B2704700006B0200215860044010B5034CF9
:20029C00FFF718FF20680028FAD110BD0011044003B40148019001BDA56F00000000000035
:2002BC00010003000A001F005900EB003902EA04F9099712EB1FA132784A0A66FA828C9E28
:2002DC0063B617C964D6EDDEC1E3E0E5FF000000A36100007F1407134D00F1242E1F133FEA
:2002FC00B00A3F0007FF0000304000400140034007400F404F40CF40CF41CF43CF47CF4F25
:20031C00CF3FCF2FCF1FCF0F000000000F00080000003F00000040003F00000004006800A8
:20033C000E00DC00060043001A00050000000000020000003F00000000000400C00000004A
:20035C000400C0000000070050C00091007070C00091007082312100319110B1007001812B
:20037C0001B100A18231329110B101911110418141224F40F106007051C0019130181039D5
:20039C00833108D01831416F3100319110B1831414165B680070251050C00091F4C3C0C007
:2003BC002014036F3110410422C082312100319110B163393110410482C0823121003191C2
:2003DC0010B163393110A2C082312100319110B1501015310514059200703F6452C03110EE
:2003FC0031066131C102426412C13110213971065131E102426400708A65996588C0208278
:20041C0050398039001E9F4041C001301814181A89C0308260398039001EA94041C001306B
:20043C001914191A3C64369110B1349110B154B0007154A064B0F0800022AF404012B09002
:20045C0032B053825339533985643F6411C122C1426470C1C26811C1C2C0426470C1C76815
:20047C0050C00091277298921516141642105310F0C12182313131398139313151B070B293
:20049C0072652772999270B262107310F0C331822131213981391B107265E2C08231608289
:2004BC0080318039020061B00071329110B151A061B0277230C2F36800008012B09032B012
:2004DC00007050C000912772999262107310F0C3318221312139813951B070B27E652772CB
:2004FC00989270B242105310F0C1218231313139813931311A107E6551A061B02772B0C08B
:20051C0018693F6401C122C1426401C1C2C04264151A3C64359110B153828564C012B09040
:20053C0032B000703F6472C281C0426422C111C1426402C011C1426462C031C3426462C319
:20055C0011C1426402C311C14264538253398564E2C347641122404142C281C8426452C275
:20057C0011C1426472C2E1CE426402C281C8426402C201C84264B0C0546900703F6442C234
:20059C0001C8426452C211C0426472C2E1C0426402C001C1426462C001C3426422C101C16F
:2005BC00426462C301C1426402C301C1426453828564007061B000711214231C7A4D33911F
:2005DC0010B10070329110B17269007061B000711318321C8649329110B10070339110B1BC
:2005FC007E690070C2C047641510C2C01216476441311514C0C0803105145410A078040478
:20061C000070E6C0863101CC161467106182F0C3010417140070067305720B720E7250B060
:20063C000071818060B050A092804122C3458080F1C11004301601110114016CD661D761A0
:20065C00D861D961DA61DB61DC61DE61E061E261E461366339639180F2C0210421318280DE
:20067C00422A1214321601112114016CEE610B62F4613963EE610B62F4613963E661E661E8
:20069C00E661E661E661E6619464E661F964E6612A65E6615665E6614667E6611012B09011
:2006BC000E720673057210123090A761F0CF3C67D4C103C0C0C354644078509150781092CC
:2006DC00607820927078309280784092907860923078909110824039F006011010311014C6
:2006FC0000924267E661BCA0E2A054A0F08050221546408000222B470D6240A02D828D313D
:20071C008D391082F1C0100409101A824A391A041082803910040E10AB10BC10C2106364AD
:20073C002972E0CF3C6713B003B0C86653B050B054B064B013B0A5661082E0223846AE66FD
:20075C000071418001222B47F08010224B46F022184764B03122384263B0CE661082E02256
:20077C0038467066386264B06F818F318F3DD0DFFF923C670071418001222B4764B0F080B1
:20079C005022654263B01182C1226046CE6605671182D12252467066526261817281813126
:2007BC00813D8231823DC0EFF19202933C670B62B081C091D381978290A2D3187F4EF30B3F
:2007DC001316E31CA44AC391E3813B149062BA1C8B46231E8B4AE31C8B4E90B207228B4221
:2007FC0090A21B1A9662E31CA44AC391E3813B18AB1CA04E9B1CA24ABC1CA442B21010821C
:20081C00D0229D42F0801022A4466364A566A462AB1094629B10946200703082F1C010044E
:20083C0063B00071A86ABC10E0B00070B281C291D281018212185181121841828131813D85
:20085C00121CBF4AE2B032B0B0DFF2923C67F1C72114C34E12C86291729131B0E1B000706B
:20087C0008C006C000C86091709100700182B081C091D0811018518110180614E1804282ED
:20089C008231823D201CE44AE2B02122E84632B00510A0DFF5923C672122E842E2A032B0EC
:2008BC0031824139F0C00104011EF642181610C01030081C04476010103C0610F1C7611437
:2008DC00FA4E16C8669171818131813D161C014B769131B006C008C0007061818131813DC7
:2008FC00408280390118F11C174B0114B080C0221747BCB033B090EFF1920F933C6700704E
:20091C0003A063B064B0EFB056650071408000222B4764B02A65EFA00071408000222B47DB
:20093C0064B003B03862018262818231823D80EFF19202933C6703A05665E661A2806364AA
:20095C00E66150B00071E661E092D08200223D47C0B20070A080F022594330B002C162312C
:20097C0001C0A080001E5243F0225343A0F56031603953632010101A136F236E11161216EE
:20099C00546B007025CA000015C900000DAD00000000000000000000B9B300008F85010004
:2009BC003D22010029800100297901000D790100952901000000000000000000A111010075
:2009DC0091420100A555010045DF0000A3810100E7410100E16D010055D300006F8501004E
:2009FC0055860100CD200100096E0100C7850100D3850100CD85010005000000958601007F
:200A1C0000000000611D01000F3F000E3FBE0D0F6A0ACB3D06C422240A000005240A0000FD
:020A3C00050AA9
:200A400000FD00000F1125550100140A7F0000A0090000EC0030793300B000312C1C0020A7
:200A600000319D3D01B008800104AF12023FCB1894EF9C0600C8CD00070000BB320FC8E0E3
:200A800038C40D00F2818F00001405C9E001F800F295952B01F32201F102CBEFF002E4159A
:200AA00001FEE4AF0D2D7D0100013901B7008D86E7350208E7CFF6030A6824B5211940B09D
:200AC0000300FA9803FFE5FF0538000040130020FAFFE183015019AD0000805F020304404F
:200AE0001F01B30801B4658201BC0303702B870810FFE05D84FFE14E9055FFE20701FAFFCD
:200B000021030F0080002307BF98E008003FA7FFE193AF03008005FFE004047880F70188CA
:200B20006A03F5F4011058FF0000FC0400C42264FEFFEF42B5220100C38301CB00B50030B0
:200B4000813476FFEF3C21E05857B011523EDF067017FFE1FF000330FFEF0F023102670325
:200B6000070F0FFFE304D3FEFFEFD4012C0200208BF9013300DF0030FFEF06EDF71D7F4409
:200B8000FFE9FB07187670403700A384FF06002040007F6440FF4000030507B12305FF33EE
:200BA000058305480A0306FFB87A02009F840200FF44C7030401026384FF10004302B004F2
:200BC0005D40FF0140800200180200FFDF7D838803008460FFF13588601A418C60FF238257
:200BE000A388020002007FF80C430900006300303621CF02C8A0624732A12BFF34676981A9
:200C0000FE28EF106DBF1C894088F188D149B2C53D0D6EF04000011B0CB000B0DF02002A91
:200C200000028B30180CDD0EFFE026000288F0440D5D0E71301200024AD0E001701F02006C
:200C40000C00038A708B718B51DF0C9E0100054F00256B9E3BFF3414180020003178B90487
:200C600074FFE591F123527307C2014EF17C13BF07FFED0F2005800400301DFE5DBF2E0813
:200C800080800031047F268569BDC55852000069818756008F381B00200175027D02F5307B
:200CA000FE001C60005000A000403F018002F004E02AF0FFEF0EFB40118EFD01008C190061
:200CC0000920003101BF02A801B0003128EF22552953782E6E333CFF0F08B08F1430632FB6
:200CE0001DAF701A0020003178003480AA0034880034900034980034A0060034290EA0C77F
:200D000072F10C4D02F1FFE1A9D005F00031D80034E00034E86A0034F00034F800349C0112
:200D20000033E4A731A6E93B7170FFEF12DD76015D008441FF0014FFE2CC801036A84148EC
:200D40001C84B3B80600F3FFEF0C91F0003446F031C1C034EF1005600097F180010032C461
:200D60002AF00031CCAA0034D40034DC0034E40034EC2A0034F40034FC0034040AB00031BD
:200D8000A50C003414003479327FFFE748011623BF004275FFF0007D000000441C002038FA
:200DA0000030593C007000F1004B00700500927F2001010000E0290174000044FFF000F376
:200DC0000100000700B9D01A0020EC01A80252401C0133340100052000313C0034FFF000E5
:200DE0009D0000016CDC02007200C094EF1900200300C48169011F00AF7F0100FFF000FD31
:200E0000000004F0180020A01AC700200101000031002A1B0001200031FFF0007B010000D0
:200E20000F00701A0020016100FFF00051300100A78301007D840100003D000000F01800B4
:200E400020FFF00000000000020000007F120000000F08000000FFF00001000000FFF000FA
:200E600001000004FFF00001000004FFF0000000400A000008020020960D0000440100200E
:200E8000BE0D000000010020DF0D0000A4010020FE0D0000780100201B0E0000C8010020FF
:200EA000380E0000E4010020480E0000481C0020500E000000020020580E0000EC0100201A
:100EC0005F0E0000F0010020660E0000F801002017
:201000003C000000000000000000000034100000000000000000000001000000000000004F
:1C10200000000000000000000000000001000000000000000800000000000000AB
:20103C003400000000000000000000006810000000000000000000000100000000000000E7
:14105C00010000000000000000000000080000000000000077
:2010700030000000000000000000000098100000040000000000000001000000FFFFFFFF87
:10109000FF00000001000000080000000000000048
:2010A0002C0000000000000000000000C4100000040000000000000001000000FFFFFFFF2F
:0C10C000FFFFFFFF080000000000000020
:2010CC0038140000E410000095A1011091A70110A1C2011009B2011041B8011000000000EA
:0810EC00000000002D000000CF
:2010F400280000000000000000000000141100000000000000000000FFFFFFFF0000000093
:081114000800000000000000CB
:20111C00341400003011000065C2011069C101101BC2011091BA011000000000000000006D
:04113C002F00000080
:20114000341400005411000071C20110A5B6011099BF011045B601100000000000000000BD
:04116000300000005B
:201164002400000000000000000000008011000000000000000000000000000008000000AE
:041184000000000067
:20118800240000000000000000000000A41100000000000000000000000000000800000066
:0411A8000000000043
:2011AC00240000000000000000000000C8110000000000000100000000000000080000001D
:0411CC00000000001F
:2011D00000000000C41B00200400000000000000000000002000000070100000300000002C
:2011F0001C110000CC1B00200400000000000000000000000C000000301300001800000040
:2012100040110000D41B0020040000000000000000000000240000004813000018000000C3
:2012300000000000DC1B002004000000000000000000000010000000A01000002C00000097
:20125000CC100000E41B0020040000000000000000000000200000006411000024000000C6
:20127000FFFFFFFFEC1B002004000000000000000000000028000000881100002400000052
:20129000FFFFFFFFF41B0020040000000000000000000000580000003C1000003400000037
:2012B000FFFFFFFFFC1B00200400000000000000000000001000000060130000180000004C
:2012D000FFFFFFFF041C00200400000000000000000000001C000000AC11000024000000C1
:2012F000FFFFFFFF0C1C002004000000000000000000000038000000F41000002800000032
:20131000FFFFFFFF141C002004000000000000000000000054000000001000003C000000CD
:1813300018000000000000000000000040130000080000000000000032
:1813480018000000000000000000000058130000080000000000000002
:18136000180000000000000000000000701300000800000000000000D2
:0813780002000000F0A40100D6
:041384000100000064
:0413880000000E0053
:04138C0000000F004E
:041390003200000027
:041394000100000054
:04139800381B0020DE
:04139C00000200004B
:0413A000FD850100C6
:0413A400FDC901106E
:0413A8000000000041
:0413AC00000000003D
:0413B0000800000031
:0413B4000000220013
:0413B8007819002080
:0413BC00010000002C
:0413C000501B00209E
:0413C400080000001D
:0413C8000000000021
:0413CC00000000001D
:0413D0000000000019
:0413D400080000000D
:0413D8000000000011
:0413DC00000000000D
:0413E0000100000008
:0413E400A01A00202B
:0413E80006000000FB
:0413EC0001000000FC
:0413F00014180020AD
:0413F40000000000F5
:0413F80000000000F1
:0413FC0000020000EB
:0414000000000000E8
:021406002900BB
:021408000100E1
:02140A002500BB
:02140C002F00AF
:02140E003000AC
:021410002D00AD
:021412000100D7
:0114140001D6
:08141800030000009CA4010088
:081420000000000000000000C4
:0414280000000100BF
:04142C0000000300B9
:0414300083C4011060
:041434003C14000064
:041438003C14000060
:04143C0000000000AC
:041440008000000028
:041444008000000024
:0414480000000000A0
:04144C00501B002011
:04145000FD81010019
:041454002000000074
:0414580034A40100B7
:04145C0060A3010088
:0414600009C30110AB
:04146400C32B010095
:04146800332C010020
:04146C0095C801100E
:0414700097C8011008
:041474000000000074
:0414780033A4010098
:04147C0064A2010065
:041480007CA2010049
:041484004CA2010075
:0214880008005A
:02148A00090057
:02148C0001005D
:02148E0000005C
:01149000015A
:041494000000000054
:041498000000000050
:04149C00000000004C
:0414A0000000000048
:0414A4009986010024
:0414A80009610100D5
:0414AC00B173010017
:0414B000F1640100E2
:0414B400EF650100DF
:0414B800B169010015
:0414BC00B128010052
:0414C000D1830100D3
:0414C400693D01007D
:0414C8000DC801103A
:0414CC001DC8011026
:0414D0000800000010
:0414D40024000000F0
:0414D80018000000F8
:0414DC0028000000E4
:0414E00020000000E8
:0414E4003C000000C8
:0414E8000C000000F4
:0414EC0034000000C8
:2014F000CA482DE9F04F0C4601210170DFF82493DFF82483DFF824A3DFF824B3C4494FF0EC
:20151000000C2027ADF14C0D65461F4081F800C0C7490E9391F838600D9205EA020008BF05
:2015300000287AD10D984FF0E047194662460F4002EA000008BF002843D10E9E0D9B4FF441
:201550008601B9F8B200DFF80CC3CDF8289012EA060701EA030108BF002919D1BC4912EA9B
:20157000060701EA030108BF00296FD0374643460D9E1C8103F130015881002F81E8C0008C
:2015900004BF311CB1F1806F60D102285ED111E0374643460D9E1C8103F130015881002FA4
:2015B00081E8C00004BF311CB1F5803F4ED1B0F5505F4BD1186A674643693868214698472D
:2015D00042E04646C449B6F9087091F90000BC42A0F10100087017D1728906F1300003C8B2
:2015F000002904BFB0F5803FB2F5505F08D0002904BFB0F1806F022A02D012F051F803E0B5
:2016100013F058FA16F002FC524692F90000401E10706FF00101318114E043466FF0010070
:2016300003F1080108806EB1B4480078832802D08120594608704646316919B160468847E8
:201650002146E8E7CDF82890B9F8B2000D9A0E9E02212F461140374008BF002900F07C83D2
:20167000A84A43F201418142119200F04F83C91C814200F04B8398490A4691F9001047460B
:20169000491E1170B7F908108C4205D043F60401814240F04A8346E3654890F838C007F19B
:2016B000300090E800034FF482062F4617EA090706EA080008BF002810D15748303003C88C
:2016D0004FF400322F4602400F4008BF002A02D111F0E6FF29E313F0EDF926E30020BCF10A
:2016F000010F4FF081045D460F9003D0287808B116F0AEFD2C70824C002067786081119EEE
:20171000E770054635702069DFF8FC91017A457A05F0070201EB022135F07F05A1F10401FE
:201730001FFA81F840F0D982B8F5006F80F2D5820A30414610F0C2F9E16904F114000522A1
:20175000083116F09FFBA8F1030305201FFA83F8E27DA57D6081217E354B0C96C2F301105F
:20177000109093F83800617105EB022518B91099022900F0B2821099022900F3AE8260B13C
:2017900015F0070F00F0A9825C480078862804D105F00700022840F0A082281300F0020AB5
:2017B000BAF1020F58DAA37805F00700022841D14E46D6F804B0002B3CD1E16909A801226C
:2017D0000D3116F05FFB06206081D84780460B96C24F4A48B6683A680078862822D122B977
:2017F00016F036FD48463A6886689DF9240016F043FF9DF924705077002090774046D77794
:20181000B04705F0100011F02DF90DE09E1B0020941B0020D8120020181700209A1B0020D2
:20183000C22E00204046B04716F080F959E2C04620150020314800780026862808BF012643
:20185000CDF82C905EB1002013F0A6F9E77805E000000C8CEC190020CDF82C90A37887B151
:201870007BB9012F00F03682022F03D115F0070F40F03082032F04D105F00700032840F0EC
:201890002982280908D315F4405F00F02382C2480778002F00F01E82BAF1020F02DAA80AB2
:2018B00080F01882BE480078C0F3810B8611BBF1010F00F00F82012E00F00C821099B74828
:2018D00002290BD010F80B10805D4018C7B20EB3E8091FD3BF1E0EE09B1B002000EB0B01E5
:2018F0008019097900794018C7B2E8090ED25BEA06030FD0BF1CFFB20CE0C046C62E0020E3
:201910000C2E0020C42E0020C01500205BEA060308BF0227C5F30029A7EB09008045C0F225
:20193000D981A8EB07002909484480B2208124BF25210F910F994018743080B216F080FBF2
:2019500094F80280E060002800F0C4810021742210F032FC0020B8F1000F207103D10C9905
:2019700005F0200008700C9803784FF00008002B53D0B9F1000F50D1D548008805F007019A
:2019900003291ED18108424609D3544991F82E30A3B90B681BB15B7E33F07F030ED16AB990
:2019B0008008C24607D3D6498B68887813B1984794F8048010B9BAF1000F02D004202071DE
:2019D0008046D14890F8383013B11098022824DACC490220002301F10A0AB8F1000F8AF8FA
:2019F00000006279CB72AAF1020007D000F1020A9AF8001041F010018AF8001002710A9AC1
:201A10000521A2F87810C2F8840015F04BFC5046032110F053F894F80480E16801F1740020
:201A30004860886523890B812089A1F85C0028090ED3C9F1030082B2A1F85C20886DD54900
:201A500016F020FAE1688A6DB1F85C00801888655348D04B0078C0F3011218788D81B9F150
:201A7000000F00F0780040EA020048EA00050D744FF0FF038B730CBF6079002081F83060EF
:201A900081F83AB081F849006089002FA0EB090085B2658100F01381E0693A46E780291853
:201AB0000831684616F0EEF93D48EE19B5B26581E16800780A7C6E46C0F38103C0F3011A69
:201AD000C0F38108002B02F0400949D0C0F301100023022804D1D0090ED201E0700D00201E
:201AF0009DF801209DF8000000EB0220A1F844000DF10206A1F84200AE4AB1F84400B2F831
:201B10005220824203D04FF6FF72824222D1B8F1030F12D072783078A64B00EB022082B2DE
:201B30004A86B3F85010B61C0120914211D04FF6FF71914218BF00200BE0E0683146323088
:201B500016F078FDE0689B493230473115F0FCFF08360346002B00F0B5802046E168C07D31
:201B7000831125D0BAF1020F03D0087CC00903D309E059EA080206D172783078B61C00EBBE
:201B90000220A1F84200032B0CD07078327802EB00220A850CE0C0466C0F0020A8A4010024
:201BB000232E0020E0683146283016F043FDE16888890009C0F08380886D3A46694616F007
:201BD00061F9E068816D79188165E669B0F85C1001227F18A919A0F85C7008310DF125004F
:201BF00016F050F96F1CBDB26581E1689DF82500896D0870E2689DF825609DF82530906DEA
:201C1000401C9065B2F85C00401CA2F85C0006F0070082F82400C3F3C10182F825102089A0
:201C300092F824708046002F4CD0604F7F183E78361D8642E68045DCE0692918324608318C
:201C500005A816F01FF93A789DF817C0111D481980B29DF81450608105EB0C60E3689DF8B4
:201C7000165000EB05409DF81550042900EB052098610BDDE06806A9521E1C3016F002F9F2
:201C90003878E3686844C07D83F82600986D05A9324616F0F7F8E068816D71188165B0F842
:201CB0005C10A8EB06077118A0F85C10791E89B22181B0F85C2001818918A0F85C1000F0CC
:201CD00043FC0EE016F0EAFB11F0EAFC09E0C046BC16002016F018FA03E016F015FACDF83F
:201CF0002C90DDF82C80D8F804008047E1690A68002313710968E161D8F80810884714E03B
:201D1000A01B0020101A00202015002040462A4F80784146401C887097F900003946401EFA
:201D3000087011F0BDFC15F081FC26480A99214F00226FF0010690F83800A1F8B2203E81EC
:201D500010B11198007808B916F060F81B481B4990F90000401E0870174890F9000010B99B
:201D7000134800210170154890F90000A0B10D9A0E9F02214FF0E0401140384008BF0029A0
:201D90000ED00E4890F90000002809DC16F060FA06E0C046222E00200020014605F09CF9BC
:201DB0000749002013B00870BDE8F08F78A40100921B0020181700209B1B00209A1B002060
:201DD0009E1B0020201500202DE9F04FCF4CDFF840A3DFF844936088ADF16C0D4108C0F0F5
:201DF0008E800CA808A911F0C3F801287BD14D4624352868D8B10769CFB1062002268DF867
:201E100008000022ADF80A600FADADF80C2002AB009593E803000C23B84740B9BDF83C0014
:201E3000E085109F27631198606316F0CDF89DF82D00012806D0022084F82800BDF822104F
:201E500021840BE0032009AF84F828003A6804F120010A6078684860BDF82210BDF82000FD
:201E700009AA11F065FE011C02D0A4A016F0C4FB022014F04FFB5546BDF830009DF82C7022
:201E900028870DA985F83A7005F1480016F058FBBDF8320005F13E0609A9A5F846003046E3
:201EB00016F04EFBBDF82200298FA887502015F08DFEB5F84610532015F088FE4A20314623
:201ED00016F0B6F995F83A10E12015F08BFEA98F4B2015F07BFE102105F1080015F062FD23
:201EF0000120207005E0012014F014FB002016F029F9A01C012115F047FD204640888008E3
:201F1000C0F00782206B14F073FC00274421384610F0DEFB00B10127381C2ED07D4D04207E
:201F30000222294616F030FA061C22D029460A881006000C40EA2220C0F380360880C00B6F
:201F500017D38D1C01200222891C16F01DFA061C0FD0A91C0320022216F016FA06462978C7
:201F7000AF78EB78687840EA0120A08143EA0720E08116F069FA304600E0002004F10C05E1
:201F9000D44EB5F9028000B32888801014F098F8CF4F394610F0CFF831460BF057F914F02E
:201FB00085FA28801FFA88F0801014F089F8394610F0C1F831460BF049F914F077FA00B231
:201FD00001216880C0A016F017FB0020452110F07FFB28B3012017A9022216F0D5F9051C9A
:201FF0001AD0BDF85C000025C013C003B0F5004F08BF0125B0F5004F0ED1002017A9022263
:2020100016F0C2F9051C07D0BDF85C00BDF85C10000240EA2120A08016F016FA284600E0D4
:202030000020271D3D8820B9CAA0012116F0E4FA1CE0C5F30B0014F040FD8346884628134C
:2020500014F03BFD05F046FEC4A20CCA0BF07EF80B460246414658460BF078F810F072FDB6
:2020700031460BF0F3F814F021FA3880D84F387878B10020432110F02BFB50B100208DF8CC
:20209000660001210DF1660013F002FF387016F0DBF9DA48006843F69821B1FBF0F016F0B0
:2020B000B5FB3B78181C1BD00020432110F010FBF8B113F08FFA387016F0C6F97988BA881A
:2020D0003B7804F110050806000C40EA212011062880090C41EA222841EA2221618204E030
:2020F00004F11005B4F8128028880121012B397014D0B9A0012116F07FFA3CE04175746855
:20211000204572726F723A20307800C0B81300207C140020982E0020D411002000B214F087
:20213000CCFCAEA797E80C000BF010F8ADA20CCA0BF00CF8ADA20CCA06F0F4FE10F002FDB4
:2021500031460BF083F814F0B1F980B22880404614F0B3FC97E80C000AF0F8FFA5A20CCA28
:202170000AF0F4FF10F0EEFC31460BF06FF814F09DF980B268800020772110F0A9FA002868
:2021900000F0B680F7200DF15E01062216F0FCF8074616F059F95FB19DF85E0001278028FB
:2021B00006D19DF85F0018B99DF8600000B90027002F00F09B80DD489DF861209DF8621022
:2021D0009DF86360038841EA02210A0142EA2612B0F90A50B0F90260C3EB2211D210A2EBF1
:2021F000430206FB02F3B0F9042049430E1302FB06F1891301EBE32101EB81028032491020
:202210004FEA222EA1F57A418A105243531303FB05F6B0F908504FF4004C4D436D1005EBB9
:20223000E6050CEBA546C5887543EE13B0F90A506B43B0F908504D436D1005EBE30563467B
:2022500003EBA543C5885D43ED1345D0B0F90E305943D312B0F910205A4302EB41029DF8F3
:202270005E30B0F90C10090401EBA2010A139DF85F1041EA03219DF86030090141EA231161
:20229000AB4B40F6354C0CFB11310CFB1211CA0F19BFB1FBF5F149004900B1FBF6F1B0F9FD
:2022B0001460B0F91630B0F91200CA088D085243520B5A4306FB05F35B1303EB2233C01878
:2022D00001EB201109E0C04654454D5000C046C00000003D0000003FE169642004F118028D
:2022F0009EFBF0F31360B1FBF0F05060012F03D08CA0012116F080F98E4801687D2707FBEE
:2023100001F04009606103F00FFE8E48022115F03BFB55462889410805D305F108000121F1
:2023300015F032FB2889810805D305F10800022115F02AFB288901096AD395F8540005F12F
:20235000080600285CD0401E44D0401E0AD0401E3BD058E04C47485400C046C07B14AE4747
:20237000E17A843F95F85010472015F03BFC95F85110542015F036FCA98F4B2015F026FC3C
:20239000298F502015F022FC0A27802395F83A008DF8597016AA8DF85A3067498DF858009D
:2023B00001278DF85B7018201CF012FFB4F85A00B4F85810884226D195F85200012822D16A
:2023D0003046202115F0EEFA1DE0032019E0C046902E0020022014E048554D00000000004C
:2023F0000000F03E0000000000A064400000000000004440000000000000594010A5010088
:20241000012010F055FF3046082115F0BDFA2889410911D395F8520005F10806032818BF18
:20243000042802D1A86D14F0CBF913F031FC3046102115F0A9FA2889810907D30FF0E6FF38
:2024500005F10800202115F09FFA2889C10907D30FF0FAFB05F10800402115F095FA2889A2
:20247000400A0DD395F8550015F06CFE41F2883014F0D6F905F108004FF4807115F084FA5E
:202490004D46E88840080DD368780026000904D3A878012801D113F093FA6E70A81D0121AB
:2024B00015F072FA6088002839D10A200825234CADF812004FF0FF37ADF81050616A059723
:2024D00004A8884700282AD10720ADF84850616AADF84A0012A88847149E1596F8B9184938
:2024F0009DF84E20087890420ED19DF84C004A78824206D089684B6C33B100213246984757
:2025100002E0304601F004FE159840B1ADF818500320ADF81A00616A079606A888471BB023
:20253000BDE8F08F5052455300C046C04C2E0020000050C32850094087850100C0150020F7
:20255000681B0020BA1300202DE9F04FB94C0C3CE0686189E2692589806DADF13C0D0E46E6
:20257000891808312A4615F08DFCA81986B2E068816D6D188565E0690122311808310EA831
:2025900015F080FCE069761CB5B2042265812918083104A815F076FC9DF813109DF8100062
:2025B00000EB0160E3689DF812102D1D00EB01409DF81110658100EB0120049015F05EFDAB
:2025D000D863049815F034FAA3F84000EA2015F0D6FA0221B648E2680170117C20790843DA
:2025F00010749DF9380016F047F882F846009DF93800118982F84800002082F8470002F176
:2026100074009065B2F85C00401A5168091851609089830A18D2030957D310F0070F07D0A3
:2026300000F00700032812BF081C5068401C48E05068C17801F00703491001F0380101EBDC
:2026500043014018001D3CE0171C02D115F000FEE268B889800A2ED379684878C6112AD103
:202670003E89796600204D780B7805F07F056D0005EBE3157E2D0DD07F2D09D003F07F03EC
:202690001818801C5B1880B2991C8642EBDC08E0002100E00121801C87F8601080B28642E5
:2026B00001DA002005E07968411879603989091A3981A7F86800506E10B1B2F86800B0B17F
:2026D000506850619089000916D292F86000002800F0FC80104611F0F9FEE268D06C0028FD
:2026F00000F0F480B2F85000002840F0EF8015F0C3FE0020E06024E24FF0000B154610467E
:2027100005A9CDF814B007ABCDF818B095F82470CDF81CB006AA04F0D8FB002840F0CB8067
:20273000059A6E6968682B89311A581A1FFA80F80AB915F08DFDB5F85C0000900196CDF8FA
:2027500008800698001D03900598A969AB6D3A4615300AF0E3FF002840F0AD80AD4895F824
:2027700060302E89C15D701A288113B1284611F0ADFEAE8906F00706032E02D1686800784D
:20279000E87395F80F90732009A914F085FB83200DF13A0108F00AFCDFF8D082DA4651461F
:2027B0000AE0C278012A03D1002F08BFDC2027D0001D491C0990C9B29DF83A00884279DD78
:2027D00009988278032E07D00378B3420DD098F800300BB1022E08D0032EE9D10378032BE1
:2027F000E6D103465B784B45E2D1BB10B3EBA20F05DA02F0030207F003039A42D1DD5046A6
:202810008146059895F80FC090F814E0514601E0491CC9B28E4549DD07694B00032E03EB41
:20283000070209D1FB5C032BF2D152786245EFD10BE0C046182E00201278B24205D098F8F2
:202850000020002AE4D0022EE2D10698077D002F08BFB9F1DC0F2DD0A869B0F1FF3F23D0FA
:20287000712008A914F018FB5346089AA9690598824206D106989A4600EB8A00C068884285
:2028900010D85B1C2C32022BF1DB0698491CB1F1FF3F00EB8A00C16002D107980121817074
:2028B000584608E0DB2007E0DB2004E0DC2002E0C22E0020DD206870E2685070906957782C
:2028D00050651FB1F22015F05AF9E2689F4DDFF8849295F83810002900F0AD8090899C4EB8
:2028F000DFF874B200F00700022858D1A078002855D15078002852D1E1684FF000080CA8C4
:202910008DF83980283115F095FE06F11C01E7680888EB6D401C0880786E0DF13902042105
:20293000984704F10C0A30B94846006818B19DF8391080F8681015F015FA90B1E76897F8F4
:20295000300002280ED1DAF80000594602222031283014F0EFFC28B90BF116010CA815F054
:2029700069FEE7680DF12E0000906D6E786E0CA942460BABA84779480078862808D1F08BF7
:20299000E768401CF083B88900F0100010F06AF815F072FD4046E06015F0C8F8D3E0704BF9
:2029B0001A78002702B101277248026827B16F7817B115F0D7F928B91878002831D015F054
:2029D000D1F970BB53782779002B40F0BA809DF83800318C02F12803002F207002F11C027A
:2029F00001F10100308414BF082600265D490020086015F0C3F901460096584601922630A6
:202A100006881A460D20334605F068F820B914F049FC03E07CA4010015F026F81348E268CF
:202A3000017841B1D5F880702FB13946104688470E48E26801780A9251B1907BFF287AD0A7
:202A50001046C17B042976DC40680078072872D0938913F0070040D0401E56D0801E6AD131
:202A7000C3F30130022808D102E0C046581500205068007807282ED0FFE7108900285AD0B9
:202A9000104641684A1C42600F788446C7739CF824607EB9002F4ED00A2F4CDA0189324E8F
:202AB000F01910F8010C884209D0082F43D1082905D040E0C07B00283DD00A283BDA604677
:202AD0000189491E0181C17B0B3101700A99C87B401CC8731BE0322018E0244E96F8A10027
:202AF0000F280CD015F0E8FA48B9181300F00200022804DA0A984D462D1D2968884796F839
:202B1000D7000A9A1074152000E0162010700A994D4605F1280013F0AFFC154E70688047D7
:202B300095F83010491C85F83010B1688847202015F0D6FB02E00AA812F02CFE4FF0000891
:202B500028E710F0ADFD0FB0BDE8F08F20150020401A0020700D0020340F0020C62E0020E6
:202B7000C42E0020141A00205CA00100A00E0020C0150020182E00202DE9FE4FE549804668
:202B90000122A1F130000260DF480768002FFCD0DE4ADF4EC027E048E04B17603268920813
:202BB00008D2324652F8042C03F14104120C42F0F00222704FF0000A8346C1F800A0DFF8EA
:202BD00064C3DBF80810D64D0191880E43D2480E41D3802018744FF6D802A3F8512018702A
:202BF0002868C0F30464162CA8BF203C1F460F3F387800F01F001628A8BF2038844223D0ED
:202C1000624602F1980EDA4ACEF800A0261A022E05DC16F1020FB8BF6FF0010600E002268B
:202C30003018166800F01F06844246F4F856A7F866604FF001061660E8D110683746176015
:202C50001068CEF80060106828460068C0F30420162808DB06E0A5F1D0000068C0F30460B5
:202C7000162800DB203800EB2170401C162805DA10F10A0FB8BF6FF0090000E01520DE4FA3
:202C900000F01F0040F4F850A3F85900386880083ABFEA48C0F800A041F04061019E6246E1
:202CB000A5F13804C80E8F0E80F0010000F00100106087F0010000F0010090602068C0F359
:202CD0008367C0F38F21B00C23D2304640F3072000280BD542425046490805D17F0806BF81
:202CF0000127391C4FF6FF71521EF5D1002810DD4FF6FF72490041F001018A4207D27F00F1
:202D100047F001070F2F92BF01210F27111C401EF0D141EA0741182013F090FA2068D24E51
:202D30002768C94CA6F10409C0F3870107F0030041EA0021D9F8040040F2FF3253468FB2A8
:202D50002C21466800972746A7F14000B0470C3D2868C0F30D011C2013F070FAB84955F804
:202D7000080C014000F07C400143142013F066FA55F80C1C01F47C000904090C01431020EB
:202D900013F05CFA624955F8042C0968C2F30350C2F30345490813D2DBF800100B0510EB08
:202DB000237003D41028A8BF0F2000E05046090415EB217503D4102DA8BF0F2500E0554688
:202DD00045EA001502F47F4002F0FF01B8F1220F40EA054041EA000124BF02F08042114398
:202DF0000C2013F02BFA974DB8F1220F32BF01202868C0F30070B8F1220F4FEA400040F069
:202E1000200084F8090126BF2868C0F3407001208E4EB8F1200F40F0100084F8090138BF92
:202E3000514606D33168C80C00F44070C1F384510143282013F002FAB8F1200F26BF306898
:202E5000C0F301505046B8F1220F4FEA400040F0600084F80C0126BF2868C0F3C06050467E
:202E7000B8F1220F4FEAC00040F0800084F8010126BF2868C0F345505046B8F1200F4FEADD
:202E9000800040F47C40A4F89C0138BF70490AD3306801038A15920501F47C1100F00F0099
:202EB000114341EA0031082013F0C8F94FF48000A5F1D0012060674A886D40F21E236FF341
:202ED0001F40834216D90868030E13F00F0F03F00F01C0F3034018BF491E072805D00628C4
:202EF0000EBF0720801C00F00F0041EA0011A2F108000170DDF804C0CCF381477F1E13D04B
:202F10007F1E3BD036E0C0469402224300600C40B03F005040100940AC3F00501562084064
:202F3000881300500000204328460068810C21D24FF480412160D2F80210430AC0F3033742
:202F500003F0800321F08F010B4347EA0301C2F80210D2F80130060A66F30303C2F80130A6
:202F7000116800F0E70721F0E70147EA010004E02C2009404FF00040224610603B48006804
:202F9000C0F3C0070FB94020A0624FF40070206428684027C0F3C14040F0300084F8C800F7
:202FB000CCF3815050B3401E03D0401E1FD002211EE0012013F0C4FD06460420314610F003
:202FD00037FC042013F0BCFD8642FAD12248066826F07F4013F0C4FBD9F814000368072154
:202FF0004FF06022300E98474FF4806020600321042010F01DFC08E0000009400420012168
:2030100010F016FC154813F0ABFB203D2868144947F6180600F03F0084F8CB0F144B0E8071
:20303000D9F800201868D1680220884711480D4D076001212960BDE8FE8FC04694042A43E3
:20305000FCFCFC008C13005040A00C409813005000803F400A600840A83F0050BD378600F4
:2030700070B00C4094046042A4010010B03F00502C20094000600C402DE9F04F0320ADF14F
:20309000540D13F085FBCF4C0025022004F11C0141F80C5F401E8D60FAD104F14000A946EA
:2030B000062701467F1E21F80C9BFBD14FF0080BC549A0F800B0C54A8160C549121D22F07C
:2030D0000303CF1A2762A361E361A66904F11C08944618460A46B14200F2F881B910E8273A
:2030F00000EB810121F8049C4FF6FC761F8006EA0C033746D21A00F1E80607EA0201266182
:20311000EC39A0F8E81028461CF0ACF86061B149D8F80000DFF8C4A220610A680AF10C0703
:203130003A6049687960AC4938465A4614F002F9B84628B9CA4801683A46116040685060A6
:20315000C848C94FC0F8B070C0F8B850C0F8C850C64EC0F8CC50C64BC0F8B460C54AC0F843
:20317000BC30C54FD0F8B010C0F8C020C0F8C47009B1284688471CF0F1F8C04ECDF83890AC
:2031900029460C2206F12C000FF016F8CE4F0222ADF820B041F270733763F08DADF8222088
:2031B000616A73631027099740F0BF00F08508A8884700280CBF0A9F2F1C0120ADF82CB01B
:2031D000616AADF82E000BA888479DF83000544620700D99616077B1D021397087F8019097
:2031F000B87087F8039087F804903946BD600220FD6012F0A9FBBA49182001221BF0E8FF61
:20321000E220414615F014F818201CF0CDFA60706068B046C8F808000CF03AF8BC4F08F171
:203230007C00A060D8F80850AE4C49466762F520A56014F0D7FCAC4D05F1180005F10C018D
:203250000DF06EFCA8600F2014F0DCFE00B1CB46042014F0D7FE08B94BF0100BA349A86810
:2032700015F0DAF8A249C82205F1240011F0DEFDA048BBF1100F686011D1606A78B1C26822
:203290006AB1FF204FF6FC778DF81000F81CADF8120004AEADF8140096E803009047964F24
:2032B00007F1180007F10C010DF03AFC3860484615F0D6F84E46BD1C824605F8029F0220C8
:2032D000687015F0D3F9014638685246C9B212F0A7FD761C042EF0DB884907F124004FF4D6
:2032F000FA7211F0A3FD484613F0D0FB012013F0CDFB484677210FF0EBF978B180498820C6
:20331000182215F041F838B1B6208DF8440011A90122E02013F024FE15F096F833208DF830
:203330004500772148460FF0D3F938B1F4200DF14501012213F014FE15F086F84846432159
:203350000FF0C6F960B11020ADF842000DF142010220024613F004FE6A49087015F074F82B
:20337000484612F057F9012012F054F9664903200860606A002855D00769DFF890A16FB104
:203390000094514612A80A688988026012AE818096E8030001234A46B847606A002841D05B
:2033B000C26852B1514612A80B688988036012AF818097E803009047606A002832D0076919
:2033D00087B30DE0C01500204DF90100C72E0020004B0020C8FF0100C8A40100681B002022
:2033F00006208DF80800ADF80A0010AEADF80C9002AD009695E803004A460223ADF84020DD
:20341000B847666ABDF840007769A08057B1BDF8400002AE401CADF8400096E80300022245
:2034300010ABB8472BA014F0A1FE606A0626002836D00769002F33D08DF818600425ADF8C3
:203450001A500EA8ADF81C9006AB009093E803004A462B46B84798B90E98193081461FE026
:20347000F01200500802002065550100855A01008D6D0100F95D01005DF30000B813002098
:203490008DF818604846676AADF81A5006AE0F907C69ADF81C9096E803002A460FABA04796
:2034B000CDF8389048460EF0D3FCE0200E2114F099FB14F04DFA08F10200012114F072FA75
:2034D000FEF782FCFCE7C04620BF020026F8029B01E6C04654492053656E736F7200C046BA
:2034F00055940000D41100206018002051630100157D0100AD7E0100A8180020491A01007E
:203510004C2E0020902E002000500940FEA40100B80200202DE9F04FADF18C0D1C911E9323
:20353000CC491D920A6806460DF156000260496841603046694612F017FE00281F9004BF1B
:203550000020229000F0F78102200027B61CDFF84CB32090D34D2297304602A911F033F85A
:203570005FEA000900F0E48122990EA816220EF023FE9DF809707F1E00F082807F1E40F062
:20359000CF81B9F10A0F40F3D681B61C316804A80160361D318805AF42F20B0039800DF150
:2035B000160111F015FABDF81600BDF81410884200F3C181B61C16F8010B16F8017B16F8AD
:2035D000014B8DF8380016F8011B8DF839700EAA8DF83A40304605F081FDBF490978002829
:2035F000064400F0A8811F9C012904F1020400F091814FF400500DF14E0111F0E9F90DF1B5
:203610004E000DF15601082213F094FE40B11C990DF14E00082213F08DFE002840F07A813B
:2036300042F2010004A906F089F942F20B0005A906F084F942F205000EA906F07FF90DF164
:20365000390142F2060006F079F90DF13A0142F2070006F073F90DF13B0142F2090006F03B
:203670006DF99DF83B0028B1022840F0538142F2030001E042F20D000FA906F05FF949E174
:20369000B9F1040F40F35781B61C16F8010B16F8017B16F8014B8DF8380016F8011B8DF816
:2036B00039700EAA8DF83A40304605F017FD0028064400F040811C9806A905F09BFF9DF871
:2036D0003600002840F00A819DF83B0000287AD195F83170002F00F0FD8095F8330087422B
:2036F00007D095F88C000A2801D10AF06DFDA86B1EE0AF6B4FF400500DF15E0111F068F9E5
:2037100013F004FF4FF0FF08229C2190A24695F83100A04240DCA86BB8F1FF0F08D008EBA5
:2037300088040019007912F08BFFA86B071923D195F831300746002B08BF229C19D0584636
:20375000229C40681946D8467F1F7F1DFA782AB1491E04F10104F8D17F1D0AE0804795F8EB
:203770003310491C85F83310D8F80810884795F83130A34200F094801C980CF037FB3871B8
:203790000120F870FC788DF8364038798DF83700229B8DF82330A1E0387911F063FC014646
:2037B00008220DF15E0013F0C5FD40B138880104219814F04BFF82453CBF8246A046641C01
:2037D0007F1DA4B2A3E795F83070002F00F0828095F83200874207D095F88C000A2801D193
:2037F0000AF0F2FC686B1EE06F6B4FF400500DF1660111F0EDF813F089FE4FF0FF08229CBA
:203810002190A24695F83000A0424DDC686BB8F1FF0F08D04FEA48140019C07F12F010FFD7
:20383000686B071925D195F830300746002B08BF229C1CD0DBF80400229C1946D846203F48
:203850002037BA7F42B1491E04F10104F8D120370DE0C046B8A40100804795F83210491C09
:2038700085F83210D8F80810884795F83030A34216D02299384620220EF09EFC1C980CF047
:20389000B5FAF8770123FF2039462022BB770446787206A8FC720DF00FF81FE0C01500207C
:2038B000612055E0CC100020F87F11F0DBFB014608220DF1660013F03DFD38B17968219863
:2038D00014F0C4FE82453CBF8246A046641C2037A4B297E764203BE0211500209DF8360037
:2038F0000EA9162240F004008DF8360008A80CF0E3FF1F9C9DF83B00A41C40B19DF84D70BE
:203910000FA8394610F084FA3F1A8DF8357006A80FF036FD20984844801C80B2209003E0DB
:203930001F9C4E44B61CA41C209884423FF714AE2098022803DC229A6720114604E01F9A2A
:20395000911C121A2298921C1D9B19801E990A8023B0BDE8F08F70472DE9F843C74C0F461D
:203970000646F80B80F0DD81E07AB90F80F06B81B80880F05881F80A80F03181207A10B114
:20399000380980F02981206C002840F093803809C0F09380002501262570B948A67114F0C4
:2039B0001DFD284613F0F2FDB64904F170002A4614F043FE04F1580090E8000314F018FB85
:2039D0002379B0EB08004FEA103071EB09010905012B40EA0100606606D194F86810B0EB18
:2039F000C12F01D8E07860B340F60900A08294F82100267100F0F00040F0010084F8210030
:203A100094F82000E57000F0F00084F82000A56114F0F8FED14A131D196821F002011960C0
:203A30006FF00203136004F1140642F8106C11688908FCD31360516841F00201516014F0EC
:203A5000DDFE2E4604F1580080E86000666611F0F3FF6078012803D0E068403014F0CAFEDB
:203A7000C6480660022012F037FC11200BF0CCFCE068007C10B90E200BF0C6FCA07A18B11C
:203A9000A572052012F028FCBD49A5710878E57128B10D7004F1EC00042114F047FAB4F974
:203AB0005000B4F95210884214BF022007200CF0F1F98EE0380980F08C80B80B77D2780B11
:203AD00029D2380CC0F0518104F13C0014F0C8FDF0B1C16849680978022919D190F827005B
:203AF000400915D2206C90F82700400910D3206C806840880028FAD0206C8068408801288C
:203B1000F5D0206C0026A0641920266414F0F8FB27F4004729E111F065F938B1B569304618
:203B30006FF4807100224FF00073A847954904F17000002214F081FDB16800254FF00108F1
:203B500040F602026572088884F8008082420AD0B0F5C15F07D00A8B4FF61F60104040F4A1
:203B70003470088306E00A8A4FF61F60104040F434700882757414F03BFAD4F85421E36868
:203B900004F5AA719A4208BFA846266E46B1864226BF301A401E801B01EB8801000B88608D
:203BB0002566192014F0ACFB27F48057DDE004F1400014F055FD061C08D0706830B17568BC
:203BD000F068B6F9241000222023A84727F40057CBE027F00807C8E000202072F9E714F0C5
:203BF00011FE054604F13C0014F03AFD061C15D0E06810B1783013F079FDF068E0602846B8
:203C100014F0FCFD14F0F4F920665F4814F0E6FB4FF4006104F1EC0014F088F9002027F44F
:203C300080672072A1E004F14C05284614F018FD07F010FB284614F013FD27F0020708B150
:203C500047F0020791E020B1042012F045FB0020E07214F0D7FDB1688046088840F6020279
:203C7000824211D0B0F5C15F0ED00A8B4FF61F60104040F4347008830DE0C046A00A002023
:203C900049C10000610C01000A8A4FF61F60104040F43470088204F1580090E80C00002B96
:203CB00008BF002A18D0042012F04AFFA0B1A56D14F09EF9854226BF401B401E401B000BE3
:203CD000F060F168708A401840F6C411F06081422CBFB0F5FA7FF160404614F08FFD11F04A
:203CF00081F898B1B56930466FF4807100224FF00073A84704F13C0014F0B2FC002808BF75
:203D100047F0020702D0192014F0FAFA75692DB1002130464FF080630A46A84727F000572E
:203D300023E014F06FFD014604F1440014F098FC0646B569A80813D296B125EA0500B0617D
:203D5000084614F05BFD706868B165B12A46F068B6F9241075680023A84704E010100440C0
:203D7000084614F04BFD27F4804727B104F1EC00394614F0DBF8BDE8F883C046000004601E
:203D9000BD2E002031CB000009B500002DE9F04FDFF8E0C292F808B009AF88460646ADF1CE
:203DB000240D049338F07F05039206BF604600884FF6FF700590F08A800934BF0020082070
:203DD0003076F08AC00834BF102080207076F08A400903D260460E30007800E00020B07628
:203DF000F08A41082CBF20240024000928BF44F010047568002108F07F08307D06916D1E19
:203E100002280EDB0C2808DC0C2803D1022044F40854069044F0030404E00D280CBF0220D2
:203E30000120044396F8880008B144F00804210900D328B1DFF8C89299F8CC3013B908B1E2
:203E5000DF2051E121096DD396F88950DFF8B4A206F1240133891AF8052007910AEB000186
:203E7000097908908918491DC9B2C918B1F5006F80F23C8100284CD0049A039906F180007C
:203E90000AF08EFE0799002808603FD0806AB0F1FF3F39D070680023401E8DB196F88A10BC
:203EB000524600F80119515D491EC9B241B1721892F87F20491EC9B2002900F80129F6D11F
:203ED000079970660968896AB162090E00F8011996F82A1000F8011996F82910089A00F881
:203EF000011996F8281005F0030500F8011902F0070141EAC501017071683289091AC9B235
:203F100070608918318105E0DB2700E0F3277770EDE00023F08A7370C00828BF44F0100462
:203F300075686D1E336DA3B9B36D93B999F8E510012903D13089B0F5EE7F06DA200904D273
:203F500002290AD144F4005401E044F48054012002E044F4085402200690DFF8ACA19AF8CD
:203F7000010001280FD013F0FDFE60B19AF8380048B196F86B00042805D1022024F480544D
:203F9000069044F4005444EA8834B8F1020FA4B20AD0B8F1030F10D1ED1F09F1D801284632
:203FB00014F048FB6D1E08E0B9F8BE00001205F8010999F8BE0005F80109069802280CD0B5
:203FD000B8F1000F15D0BBF1000F0CD004990598814208D144F040040BE0BBF1000F08D1D0
:203FF000B8F1000F05D00599081205F8010905F8011944EA8B24BBF1020FA4B209D0BBF1D9
:20401000030F0ED10399ED1F284614F013FB6D1E07E003990888001205F80109087805F843
:204030000109BBF1000F05D00498011205F8011905F801093878F8B934480178307D0D28D1
:2040500014D068B9306D28B999F8A800411C89F8A8100AE099F8CD00411C89F8CD1004E017
:2040700099F8B600411C89F8B610014605F8011904E0C0465A0F002044F48074201205F819
:2040900001092C7070683189401B7560C0B240183081200927D3B06D00B130629AF83800E0
:2040B00010B1307D0D281ED1726A12F1150002D114F0CEF8726A916A481C9062306A32894B
:2040D000B162471B0092D21B019090B20290706A96F888202B46153008F000FB00281CBFBB
:2040F0007070071C07D10020707005E0E5277770F32013F044FDF8B209B0BDE8F08FC04619
:20411000A00E002078A4010020150020112E0020B0B50446BC480768ADF1480D002F00F0BC
:20413000AC812078401E112800F2A781DFE810F06E0156013C0127011F010801F100E3000A
:20415000C300B2008D005D0053004200A5012A001C001200F86B002800F08F8168462146BD
:204170000DF006FAF96B86E1386C002800F085816846002101220EF01FF860788DF8000041
:20419000396C78E1F86A002800F07781684600210E220EF011F8A11C684613F0CBFDA57B43
:2041B000A1890022ADF80A1005B101228DF80C20F96A61E1B86B002800F05F8168460021CB
:2041D00002220DF0F9FFA5788DF8015060788DF80000B96B4FE1786B002800F04E8168469A
:2041F00021460DF0C5F9796B45E1386B08B36846002114220DF0E0FFA5788DF80150A36846
:204210000193A289ADF80820A17B8DF80A1060788DF80000E57B8DF80B50237C8DF80C304A
:2042300094F911208DF80D2061690491396B684688476068002800F020810146F22008702C
:204250000020487011F080FB17E1B86A002800F014816846002124220DF0AEFF6078A11CDF
:204270008DF800000DF1020013F064FD04F10C0103A813F05FFD257EE08A04F119018DF898
:2042900018500B22ADF816000DF119000CF014FBB96AF0E0786A002800F0EF806846002171
:2042B00002220DF089FFA5788DF8015060788DF80000796ADFE0386A002800F0DE8068468D
:2042D000002112220DF078FF658862796078ADF8025023798DF80520E11D8DF80000A57987
:2042F0008DF804300B220DF107008DF806500CF0E3FA396ABFE0F869002800F0BE80684668
:20431000002101220DF058FF60788DF80000F969B1E0B86910B1204610F002F9A07D00281D
:2043300000F0AB80A07820B9A069002800F0A58003E0A069002800F0A08013F097F89CE0E9
:204350007869002800F099806846002113220DF033FF6D46A01C0168406829600B2268600A
:2043700004F10A0102A80CF0A7FA796983E03869002800F0828020460BF08CFC7DE0F86840
:2043900000287AD0684600210E220DF015FF6078A11C8DF800000DF1020013F0CBFCA0897E
:2043B000ADF80C00F96866E0B868002865D06846002114220DF000FFA01C01686D462960B6
:2043D00040686860A07A0B2204F10B018DF808000DF109000CF070FAB9684CE078680028C6
:2043F0004BD06846002110220DF0E6FE60786588211D8DF800000B22ADF8025001A80CF05F
:204410005BFA796837E0C046701B00203868A0B36846002119220DF0CFFEA01C01686D46EF
:20443000296040686860A07A410824BF01218DF80810810824BF01218DF80910C10824BF96
:2044500001218DF80A10010924BF01218DF80B10C10924BF01218DF80C1030F07F001CBFF2
:2044700001208DF80D000B220DF10E0004F10B010CF022FA39686846884712B0B0BD704723
:204490002DE9F04FC34E37688246ADF12C0D17B913F0DEFE3768DFF80C8308F10300DFF8E1
:2044B0000C930578002D3FD0002538897968BA4B0795C400097818781034890906D340F672
:2044D000485191FBF0F1091901F5AF743B7D60438400352B0CBF2F1C4FF4FA570DF126017D
:2044F000E82010F037FC9DF82600032808BF44F620673068007D3C19352807D112F0E4FD81
:20451000014630686C300FF083FC444302204F468DF8200007F10C000068069406A909F001
:2045300047FBAC480C3805709C4901209C4F08703978012902D0002102F0CEFD3068048963
:20455000456814F071F8DFF860822888000932D398F83870316877B34A6A4F6E906A4646C8
:20457000B0F1FF3F22D00FB3431C93628862030E07F8013991F82A0007F8010991F82900A2
:2045900007F8010991F828003870086A00940190401B201A80B2029091F88820486A8B6AE1
:2045B000153019462B4608F099F800E0DB20F16F002840F0E380214628460DF07FFA642088
:2045D00009A910F0C7FB494698F83870087837B9774800780BF058FA012805D0CAE00BF0F9
:2045F00053FA012840F0C680DFF8C8C1A01C241D6D1EA1B2ACF87800C1F3022040F008005A
:2046100005F80109002629700227CCF884509DF82450ACF86A60002D0CBF6748674864468C
:20463000C4F8C000664DC4F8800068688047AB460A90BAF1010F54D0BAF1040F51D0BAF174
:20465000000F4ED094F84000BAF1050F04F13005C0F3C0002CD0E8200DF1250110F07AFB58
:2046700098F8380000B39DF8250003281CD1687B2B7C00F0F00005F1110140F0030068735D
:2046900043F018002874F42010F064FBD8F89C00804704968DF814706686A064B0468DE87F
:2046B0008001D9F80C004EE0464B04F168050EE028B9687B00F0F00040F0010004E0687BE1
:2046D00000F0F00040F003006873404B6686049638468DF8147031468DE80300D9F80C0078
:2046F00032E094F83D0000F0F00040F0030084F83D0094F8400004F130010D46113140F04C
:20471000180084F84000F42010F024FB98F83800002808BF4FF4FA5002D0D8F89C00804739
:20473000A06404961F498DF81470D9F80C008B78002B06BFA4F84E6004F14C056686324696
:2047500039468DE806001F4B294604AA01F02EFD1D490880DBF80810002809D41C4A92F9DD
:2047700000001C4F6834401C10700A983C600DE00A9888471A200DF095F808E0002908BF0E
:20479000E420F8D0144A00201070E42088470BB0BDE8F08F700D0020201B0020931B0020C7
:2047B0009E1B0020401A002020150020E0190020770F0020D81200204E9055550E7A5555BE
:2047D000C0150020ADAB0000101A00201DD800009A1B002024170020C62E00202DE9F04FA4
:2047F000C24D4FF0000AADF1140DDFF81C83E868CDF808A000288DF80CA040D1CC4CBC49D8
:20481000843C2068814210D0BA4981420DD0BA4981420AD0B949814207D0B949814204D025
:20483000B849814201D013F013FD13F021F821684FF0FF32012805D1C1F30330083806D0AF
:20485000C01F01D0012A02D10120E87001E085F803A012F00FFA4446206A00F1200118B91E
:2048700013F0F6FC216A2031096805F1140088474FF4FA70E884A54FAF620626EE624446E9
:20489000E26992F82670E7B9A14892F8257001788F4216D05046342404FB002C9CF8267082
:2048B00037B99CF82530401C9942C0B2F4D103E09CF82500884204D1604611F0A9FDD8F849
:2048D0001C20DFF850B2D8F824001BC88BE81B00E878012814BF50460520DFF83C928F4CB7
:2048F0008BF8000099F8157127B990690068C4F8A40005E0D0690068C4F8A40013F0A6F8E6
:20491000632004A910F026FA99F8E720104611F0CFFFB4F896C007462CF0070C4CF0010CB3
:20493000A4F896C0D4F8980004F18806812A40F00F00C4F8980001DB842A05DB397B052904
:2049500014BF2421292100E0212184F89C10717D812A01F03F01717501DB842A18DBBB7A39
:204970006BB99DF810203F3262F305017175F28A4FF6C07303EA020141F0180113E09DF8D6
:20499000102001F0C00102F03F020A43114603E021F03F0141F002017175F28A4FF6E071EE
:2049B000114041F02001F182FA7A397B491D5143D8F81C200A230CF0010C91FBF3F1C90430
:2049D0004CEA1141F181F97A1923890391FBF3F161F31C203061308B92F824104FF6F773D9
:2049F00061F3020003EA0001308392F8240000F008000843308399F9D6000EF0A9FFA4F862
:204A1000A20079683B68D8F81C203889401E414303EB51004FF47A71B0FBF1F0A4F8A80074
:204A3000106A0078A4F88AA084F8AC00C4F88CA0707B00F0F00040F00100707313F022FD9D
:204A5000A0B9F87A364A99F8E740B1FBF0F01070F87A022CB1FBF0F0C0B2B1FBF0F0687035
:204A700004D1304802214170A8270770EF68D8F820402FB3504610F045FA287999F8E71058
:204A9000884211D1697999F81521E86891420CD10221524653468DE80600314602AA01F0CE
:204AB00085FBC8F80C6017E0E868D8F8201049688847D8F8207001201B493C68087000E092
:204AD00024681A4805F1140359463246A047E860D8F82400C8F8280099F8E70099F815711A
:204AF000287105B06F71BDE8F08FC046E019002000F0022000F0012000F000200080022060
:204B10000080012000800020181700206D720100870F0020782E0020A00E0020D8120020C1
:204B3000201B0020401A00209F1B002018290020181300502DE9F04F09AFADF13C0D08904E
:204B50000A92388809911E46ADF81800101C08BF002000F08481002700F101094FF0FF3A8C
:204B70004FF0010BB8466CE1252940F063811078521C0A922D2818BFADF8068005D15846D0
:204B9000551CADF8060010780A9530281CBF4246434605D10A9908785A465B46491C0A9144
:204BB0002A28CDF80080554616D1306804930A99CDF808A0C01C4B1C20F00300001D30608A
:204BD00050F8044C0A93002C0878009418D5ADF806B06442009413E044460AE0610001EB1A
:204BF000C40140180A99A0F1300408780094491C0A91302801DB3A28F0DBCDF808A00493A7
:204C10002E282BD10A9908782A2801F101010A9111D13068CDF80880C01C20F00300001D5B
:204C3000306050F8045C002D48BF454608782B46491C0A9111E0454643460AE0690001EB38
:204C5000C50140180A99A0F1300508782B46491C0A91302801DB3A28F0DB02930AB12246B3
:204C700004926C2804D04C2818BFADF8048005D10A990878ADF804B0491C0A910BA9CDF8E7
:204C90000C800FAB07916428059300F08B80692800F08880BDF818C0752872D078286ED034
:204CB0006F286AD0702850D063283DD073281ED009980A990128A1F101010A9115D96B49FC
:204CD0000C68B5F1FF3F03D0A84288BF6D1C00D8099D029508A80AA932466B46A047C71977
:204CF0000A99039801F1010974E040462AE030680A99C01C20F00300001D306050F8040C57
:204D1000BCF1000F01F10109014608B955A00146079113F0EFF90390B5F1FF3F5BD0A84278
:204D3000C4BF281C039056E03068C01C20F00300001D306010F8040C5D468DF82C000A9990
:204D50000395584601F1010945E0082035680490E81C20F00300001D306050F8041C08223D
:204D700010230FA80DF026FF401E0790402101700A99079801F1010929E0082302E01023C9
:204D900000E00A230A99306801F10109C01C20F00300001D306050F8041CAA42BCBF2A1C0E
:204DB000049210E00A99306801F10109C01C20F00300001D306050F8041CAA42BCBF2A1C75
:204DD00004926FF009030FA80DF0F4FE0790059D281A0390009C241ABDF8065000945DB97F
:204DF00006E008A8202109AA11F0DDFF009C7F1C641E0094F5D503980546401E039075B920
:204E1000BDF80600E8B10098401E009019D408A8202109AA11F0C7FF00987F1CF4E70798A3
:204E3000411C0791017809AA08A811F0BCFF03987F1CE1E708A809AA11F0B5FF7F1C09F12A
:204E500001094A460A9812F8011C401C00290A907FF48AAE089808B14146017038460FB087
:204E7000BDE8F08F286E756C6C2900C020A501002DE9F04F002898461546ADF12C0D00F0EF
:204E9000158111F47C1F40F00E8111F00F0F00F00D8107460591002006900A904FF0000AF4
:204EB0000990544608944FF0010BCDF810B0044650460790059805990BEA000021EA0B0185
:204ED0004FEA4B0B401E059100F0CD80401E7BD0801E68D0001F40F0E08005B12F66072062
:204EF000152642F2D002022307F8010B01A907F8016BA2F1CF0007F8013B0FF069FD68466C
:204F100003A90BF05BFA9C4801783E46812907DB9848B0F8B600842905DA49F6D05104E00A
:204F30009448B0F8B60042F2D00108180099019A4FF47A6390FBF3F040180090824206D8B6
:204F5000801ABDF80C300090581CADF80C00009B50085146814609041804030C1943000418
:204F7000534610EB090041EB0A0102F0AFFFBF1D0090BDF80C309DF80C009DF8002006F8FC
:204F9000010B181206F8010B9DF8011006F8012B9DF8023006F8011B9DF8032006F8013B1E
:204FB0000934327078E00220152607F8010B042307F8016BB8F1000F07F8013B0CBF099851
:204FD00098F80000241D65E01DB1EF6595F86B0006900520152642F2D002049B07F8010BEB
:204FF0000DF10E01DDF8189007F8016BA2F1CC0007F8013B0FF0ECFC02A810F069FC5E4876
:2050100001783E46812907DB5A48B0F8B600842905DA49F6D05104E05648B0F8B60042F2F7
:20503000D001081802994FF47A6390FBF3F09DF80E209DF80E3040183F1D0290000206F86A
:20505000019B00EB6300B0FBF2F002909DF808009DF8091006F8010B9DF80A3006F8011BF9
:20507000E41D337018E00320152607F8010BB8F1000F07F8016B034607F8013B04BF0A980F
:2050900007F8010B05D098F8000007F8010B98F80100641D07F8010BA4B2059800287FF4DA
:2050B00009AF264661E011F00F0F01D000205DE080468A4602264FF4803908F1020509EA81
:2050D0000A002AEA090A4FEA4909B0F580301AD0B0F5803014D0B0F500300ED0B0F5802094
:2050F00009D0B0F5002004D0B0F580102AD1072404E0062402E0052400E00424002704E0A7
:205110000224012701E001242746A81C214600F073FC47B104F00F04C0F30A0141EAC42167
:2051300041F4004105E004F07F0400F0FF0141EA042105F8011B36180912B61C2970B6B2F8
:2051500045196D1CBAF1000FB9D1022ED8BF00260BDDB01E4FF6FE7708F8010BB819C0F327
:20517000022040F0A00088F8000030460BB0BDE8F08FC046A82A0020870F0020BA482DE992
:20519000F84F0025B94CB749056094F8E200002800F06381012800F02F81B54E02283CD0BD
:2051B000032840F05A8151F8250CD4F8B8100029A0F5C060C4F8D400B8BF49420028B8BF8C
:2051D0004042814226DA4FF08057D7F8A4014568B4F8BC0030214FF47F4208230090304655
:2051F000A847D7F8A4014568B4F8C00004214FF4F802122300903046A847D7F8A401B4F877
:20521000D070456820214FF440620A2330460097A847012584F8D8501AE151F8258C13F080
:20523000E9F82F4600B901273946924F38680028FCD0B146012609F10409D9F82CA03E60D3
:2052500009B113F0DDF8CAF30720C4F8BC0013F0D1F8AA4600B9B2463B68002BFCD0D9F878
:2052700000B0BAF1000F3E6001D013F0C9F8CBF38440C4F8C00013F0BDF8AA4600B9B2462A
:205290003B68002BFCD0D9F81C90BAF1000F3E6001D013F0B5F8C9F38120C4F8D000B8F578
:2052B000C061C4F8B81000F09C8094F8D80068B9C4F8D410D4F8C000C4F8C800D4F8BC7000
:2052D000C4F8C470D4F8D030C4F8CC30D4F8D410D4F8BC30002954BF02206FF0010004F12F
:2052F000C802176801EB41014018411000EB917107EBA1001060D4F8C810C4F8C430002911
:205310001CDD1E293CDDD4F8CC0030B93429B4BF15391E21C4F8C81025E02A29BABFD4F815
:20533000C8000B381E20C4F8C800D4F8C4003F28B4BF401C3F20C4F8C4001FE0D4F8CC0054
:20535000032812D011F10B0FC6BFD4F8C8000B30301CC4F8C800D4F8C4000028C4BF401E57
:20537000051CC4F8C450032508E011F1150FC6BFD4F8C8001530301CC4F8C800C4F8CC50F0
:205390004FF08057D7F8A401B4F8C43030214FF47F424568364800930823A847D7F8A40132
:2053B00004214FF400321123456831480096A847B4F8C860D7F8A40104214FF4F802122385
:2053D00045682B480096A847D7F8A40120214FF440620A23B4F8CC60456825480096A847DA
:2053F00001E084F8D85040F2FF50404502D8801C40452DD208202EE051F8251C1E4F4BF2AE
:20541000F5204843060A3868C0F3814001280AD111F056FD10F0F2FA12F0F8FF3111C01069
:20543000484306EBE03694F8E50030B91348006820F07F408019460801E084F8E55010480D
:20545000310C0660012741600E4D8760287808B90B2000E0052084F8E40004F03DFBBDE8CC
:20547000F88FC0462D400C402C500C40B80F002000A00C4000800C40B43F005010200940B3
:205490003C600C4066A401002DE9F04FAC4C04F128000068ADF1240D0FF0FCFF08B112F0B3
:2054B000CBF9A248DFF89CA2DFF888B20068A24E089011F0F5FD11F0E9FFE569A769B5F534
:2054D0007A7F13D0C01B4FF47A720023A5FB000102F0FCFC80464FF47A72002312F0F6FC1C
:2054F0002A46002302F0F2FCC01901E0A0EB0708A0618D488C49006820F002000860706870
:205510008047DBF80010DBF8043045466918B1F57A7F0DD34FF47A72B1FBF2F2D2184FF453
:205530007A73CBF804201F46B1FBF7F25A43891ACBF80010B168884770688047DAF804100D
:2055500002466818B168CAF8040010468847DAF8000000285FD007464FF000097068804712
:205570004FF000081FFAA5F3079083B95FFA95F36BB93979E8B2884204DD7968284688423B
:2055900009D20AE03879E9B2401A387108E079682846884201D3414601E07968091A7960CD
:2055B000B88878B9FB8853B9FB6843B13B8933B1B87A19460AF060FEF8687860B88808B9BA
:2055D000FB880BB13B896BB9B9F1000F04BF3868CAF8000003D03868C9F800003868B846E4
:2055F000074601E0B9463F68B16807988847B8F1000F0ED0B8F8043043B9B8F806302BB900
:2056100098F80A00B8F808100AF036FE404611F01DFF002FA2D144484349006840F00200F3
:205630000860E06828B3804723E015F8060C2169A5F10C07032819D0E16A9DF81600097828
:20565000884210D115F8080C11F04AF9B979012903D0022908BFA87000E0287000202946EA
:205670000EF036FA05E012F0E7F802E009B12846884708200727ADF81000716AADF8127040
:2056900004A88847069D0028CFD0294800680088C8B1706880472649096800220D880A807B
:2056B000B1688847089A00202946207090470546FF202070706880471D4909680A88154300
:2056D0000D80B168884711F0EBFC0746B7F1FF3F1CD0706807B9194F216AB94238BF0F1C96
:2056F00080471C230546626AADF802300820ADF80000716A019268468847A16A3846491C00
:20571000A16210F03FF9B1682846884708200A27ADF808004FF0FF35ADF80A70716A0395DD
:2057300002A88847C5E6C04610E000E00CA50100B42E0020AC1B0020C01500208EC2F52862
:20575000B0190020882E00202DE9F04FA54C064600200F46ADF13C0DDFF89092ADF80C00E2
:205770002068A44D017D252900F010816C3005A903F040FF002818BFC0B240F0308120461F
:205790000068C18AC9080DD3007D03280AD09DF81F0038B99DF820004C463870B534207006
:2057B00000201CE101A804A90AF008FEA5F12F018B4691F82F30019A3468DBF808104FF482
:2057D0007A7A504641F208155843891A0AFB12000AFB01F1001B091B8D42C8BF002965DC94
:2057F000854205DD002803DD346804F5915434609DF81F00002857D042F204000DF135016B
:205810000FF0E6F811F092FE044606980DA9241A42F206000FF0DCF89DF834109DF81D0096
:20583000FF2904BF0A218DF83410FF2808BF0A209DF834206C499DF81C30D046B4FBF1F13B
:20585000801880B24843991008FB01F1814298BF081C2D1805A811F04AFC9DF81C20346861
:20587000B0FBF2F15143411A8BB251464B4308FB02F1CA1AC91A121B091B8D4201D9002959
:2058900008D56942914216D2002A14D5B5FBF8F109B203E06900B1FBF8F189B232684FF455
:2058B000916303FB012405E0002004E0306841F630342418346005460DF1120102A80AF0D5
:2058D0007DFD0298DBF80810B4FBFAF210180290814203D99BF82F30834204D94B4603F1AC
:2058F0005804267836BB9DF81C0055190004A84298BF2D1A9DF81F00002808BF9DF82000AA
:2059100016D09DF81C00B5FBF0F084B29DF833000FF0A8FB9DF83120014620460FF03AFBE9
:20593000044611F0D1FB024608A920460FF080F94C460DE0814204D8BDF81200401CADF883
:2059500012004C46BDF8120094F85B100CF0E2FF3870244E84F8B5003068007D05287FF4F8
:205970001FAF2348007820B112F0FCF900283FF417AF387803A9ADF80C0042F20C0003F03D
:20599000DDFFBDF80C00A4F8B00009E768460DF10E010AF013FD3068009A2B7841F2081435
:2059B0004FF47A7101FB0202009259438A1A944210DCA1F5FA619142BCBF00F5FA603060F7
:2059D0004C4694F85B10208F0CF0A4FF01460020397002E039784C46652084F8B5100FB026
:2059F000BDE8F08F700D0020A0860100A82A00205D0F0020932B0020F0B504460846ADF178
:205A10006C0D401E6BD0401E0DD0801E00F00381401E00F0E980401E00F0DB80401E00F069
:205A3000A88000203CE142F2010007A90EF0D0FF42F20B0008A90EF0CBFF42F206000DF14F
:205A500065010EF0C5FF42F207000DF166010EF0BFFF42F2050019A90EF0BAFF04A80AF05A
:205A700015FB05460DF1670142F209000EF0B0FF9DF86700002808BF002303D0022011F067
:205A900033F8034607A8006808A920600988271D3C46B81C218005F007079DF865609DF87C
:205AB00064109DF8662000F8011B9DF8674000F8016B03F0030600F8012B620747EA9261E6
:205AD00004AC41EA8611012700F8011B9DF8672000942946019707F0B1FC0A3099E042F2C6
:205AF00006000DF165010EF073FF42F207000DF166010EF06DFF42F2040019A90EF068FF53
:205B100004A80AF0C3FA05460DF1670142F208000EF05EFF9DF86700002808BF002303D0E9
:205B3000012010F0E1FF03469DF864009DF8657004F8010B9DF8666004F8017B9DF86720B1
:205B50009DF86770790704F8016B03F0030705F0070646EA916004AE40EA8710294604F8E3
:205B7000010B002700962046019707F067FC001D4FE042F2150011A90EF02AFF13AD42F28A
:205B9000160029460EF024FF15AE42F2170031460EF01EFF17AF42F2180039460EF018FF09
:205BB00011A801682160406860606A6804F108035A6028681860306803F10801086074685D
:205BD0004C60386801F1080528607A686A60202066E042F214000DF122010EF0F9FEBDF89D
:205BF000221002200A1258E009A8002120220CF0E3FA42F2130009A90EF0EAFE09A812F06E
:205C100079FA024609A920460AF056FE09A812F071FA80B244E042F20E0002A90EF0D8FE1E
:205C30000DF10A0142F20F000EF0D2FE0DF10B0142F20A000EF0CCFE03A942F210000EF03C
:205C5000C7FE0DF10D0142F211000EF0C1FE0DF10E0142F212000EF0BBFEBDF808009DF805
:205C70000B209DF80C709DF80D609DF80E509DF80A1004F8010B02F00102001204F8010B1D
:205C900007F0010042EA400206F0010042EA800205F0070042EA4012042004F8011B2270A1
:205CB0001BB0F0BD2DE9F04F06469E48001D0068ADF1340D80470B900AA9822005F076F956
:205CD0009DF8280018BB00248DF828404FF6FF75ADF804509DF82800ADF80650FF2108225F
:205CF0008DF8000002A812F0CBFC8DF81840D420694602F0D3FA9DF82800401CC0B28DF84D
:205D100028000328E4DB82200AA902F0C7FA0020DFF808A2DFF808828DF8280081469DF84E
:205D300028008DF8019069468DF80000D02005F03DF901274D46E8B99DF80B30012B07D196
:205D50009DF80A0020B90DF1020012F08FF888B9747B002C0CBF052209224F469C4209D16C
:205D70000DF1020006F10E0111F070FC002818BF012507D1002F40F0BF801DB9707F002818
:205D900000F0BA804C469DF828008DF8214008A98DF82000D12005F009F9002832D19DF896
:205DB0002200FF282ED08DF800006946D42005F0FDF8002833D102A8311D082211F046FCE9
:205DD00000B330887788ADF80400ADF8067045B1307B9DF82810B7698DF818000DEB8101E0
:205DF0000F61D420694602F059FA75B1307F9DF82310884209D08DF8230008A9D12002F0BF
:205E10004DFA02E0641C032CBDDB032C74D14F468DF80070D420694605F0C8F828B1DAF801
:205E300008100B988847192074E002AB184612F01DF84C4600B101242046341D30B91846B3
:205E50002146082211F002FC00284AD030887388327BADF804009DF82810ADF80630002D82
:205E70008DF818200DEB810000F110000CBF4946B1690822016002A8214612F003F898F83E
:205E9000380030B1D8F888201AB19DF80010204690474C469DF828008DF8214008A98DF849
:205EB0002000D12005F082F8E82807D09DF82200FF2803D0641C032CECDB10E09DF80000BF
:205ED0008DF82490337F8DF8220069468DF82330D42002F0E3F908A9D12002F0DFF9032C3C
:205EF00002DB7F1C032F93DB032F05D1DAF808100B9888471A200DE09DF82800401CC0B264
:205F100002288DF82800FFF60AAFDAF808100B98884748460DB0BDE8F08FC046C015002026
:205F300020150020C0150020F0B500215022ADF15C0D02A80CF040F9F22016A912F070F9AD
:205F5000974DBDF8580016A9A5F87400F32012F067F9BDF858000DF10901A5F87600E220D1
:205F700012F04EF9E88DADF81200410806D305F10C01096805A80160BDF81200810805D3D0
:205F9000291D098806A80180BDF81200C10807D305F1100109680DF11A000160BDF81200C9
:205FB000810907D305F1180005C808A981E80500BDF81200010A06D305F1140109680AA89A
:205FD0000160BDF81200010907D30BA805F1580124220AF071FCBDF81200400903D3686B3D
:205FF00015902F6B1497012011F008FEBDF8120041082CBF0F240B24810824BFA41CA4B2A0
:20601000C10824BF241DA4B2810924BF0834A4B2010A24BF241DA4B2010924BF2434A4B20E
:20603000400924BF0834A4B2204610F00DFF071C00F0B48005260DF1090100F8016B0A68D0
:20605000026049684160BDF81210083012F002FABDF81210844648080BD3BDF81410604621
:2060700012F0F8F9BDF8161012F0F4F9BDF812108446880807D3BDF81810604612F0EAF9E0
:20609000BDF812108446C8080BD3BDF81A10604612F0E0F9BDF81C1012F0DCF9BDF81210B2
:2060B0008446880909D3089960460FF02CFE09990FF029FEBDF812108446080A06D30A9932
:2060D00060460FF020FE8446BDF81210354A9388080949D3BDF82C10604612F0BBF9BDF883
:2060F0002E1012F0B7F9BDF8301012F0B3F9BDF8321012F0AFF9BDF8341012F0ABF9BDF808
:20611000361012F0A7F9BDF8381012F0A3F9BDF83A1012F09FF9BDF83C1012F09BF9BDF807
:206130003E1012F097F9BDF8401012F093F9BDF8421012F08FF9BDF8441012F08BF9BDF807
:20615000461012F087F9BDF8481012F083F9BDF84A1012F07FF9194612F07CF9117812F0E2
:2061700079F9BDF812108446480906D3149960460FF0C9FD15990FF0C6FD05F120012246CB
:2061900030463B4606F06CF80820ADF80260064D01972968ADF800006846884717B0F0BD5D
:2061B000B8130020D4110020E41500202DE9FE4F9B4692468946054612F024FB02908C4809
:2061D000353801680CAFA94208BF416801A84A4653460090284604F06FF8834C061C13D1C3
:2061F00094F8880140F0040084F888010298C4F87C5112F003FB9DF8040002280CBF6FF031
:2062100002086FF00108ECE005F1780011F06EFAB08CA4F85000B6F92480C6F808909AF8F6
:206230000400C6F804B086F82600A6F824806F48F56097E80C00202106F110071940104063
:2062500087E80300002786F82770F06840680078022809D19AF80500012805D196F82700B9
:2062700040F0100086F82700029812F0C7FA94F88901042807D1D4F88001B4F9841194F897
:20629000862112F07CF912F0BDFA814694F8890130F004033ED104F13C000368D3B9314665
:2062B00010F034F838B3A5F8C08096F8270040F0800086F8270085F8C270E07920B120785F
:2062D00010B101202072E771484612F097FA484800781FE004F13C00314610F017F850B102
:2062F000A5F8C08096F8270040F0800086F8270085F8C27048E0B4F9500000F6FF706FF30C
:206310001F30A4F85000484612F078FA6FF00100BDE8FE8F02280ED196F8270040F0800030
:2063300086F8270085F8C270484612F067FAB6F92400BDE8FE8F012811D104F1C80011F03A
:20635000D5F996F8270040F0800086F8270085F8C270206C0028E7D1484612F04FFA206CD5
:2063700000282AD12078A76400BB6079012838D012F048FA8146A079A0B9B0680DF064F894
:2063900058B9607A012803D1484612F037FA28E0484612F033FA04211FE004F1C80012F09C
:2063B00025FAF1E7134901200870EDE7012011F0C1FA192011F0A4FF13E0206CC068406804
:2063D000007802280DD1F06840680078022808D19AF8050028B94FF4004104F1EC0011F0D4
:2063F000A5FD4046BDE8FE8FA00A0020FDEFFF9F290C0020BD2E00202DE9FE4F0646307D23
:2064100001280AD196F916000DF0A2FA4FF6FF71814208BFE82000F00281F07B814A20B961
:206430001146491C0978022908DB012803D110460078022802DBF120BDE8FE8F346AB6F8A0
:20645000289096F8347096F835B0B58B4FF000085FEA040A17D0744890F83830002B2ED035
:20647000016D00292BD004F0FF0088476E49096D04B20AF47F008847001900B2001D00B2EF
:20649000C43084B200E0C4240DB12D1DADB267480078012809D147B16548C11991F80480DD
:2064B00010F80B002418641DA4B205EB090020184044801C80B210F02BFF071C02D11A20C9
:2064D000BDE8FE8F08EB09002B193881002D07EB030078600EBF0020E019801C002174224E
:2064F000C7F8A00007F10C0012F0CAF84C442D1907F13C00FF211022A7F84C5012F0C0F814
:2065100007F12C000F21102212F0BAF800243C707C707868716A328D0AF0CEF907F18000C2
:2065300006F12C010B220AF0C7F907F18C00314611F018FB7089A7F89600307B87F8980041
:20655000707B06F10E0587F899002A6869460A60AB888B80AA798A719DF8001020460129E2
:2065700008BF01209DF80110012908BF40F004009DF80210012908BF40F008009DF80310E0
:20659000012908BF40F010009DF80410012908BF40F020009DF80510012908BF40F04000C5
:2065B0009DF80610012908BF40F08000A7F89A00707D87F89C00B07D87F89D00B28BA7F819
:2065D000A42022B1D7F8A000B1690AF075F9B07F87F8A600306AC7F8A800B7F8A400C0B10A
:2065F000D7F8A000A8B17868401E7860F82101707868401E78600470B7F8A410B7F8A46083
:206610007868401A786039897018801C38817868B8650848007839460DF05AFA2046BDE819
:20663000FE8FC0469E0D0020201500206C0F002078A40100B01600202DE9F047DFF80CA227
:206650000746AAF13500DFF8F8810068800880F0E78010F035FC814908310B6800261C17F6
:20667000641C990D0AD2C0F13E0110F10A0F4FEAE101D8BF08218C42B8BF0C1CDFF8C4C15A
:20669000990E0FD2590E0DD36246143A1168C1F304211629A8BF20391268C2F30462162AFF
:2066B0000EDB0CE0634AD2F87C11C1F304611629A8BF20391268C2F30442162A00DB203AEF
:2066D00061189146162905DA11F10A0FB8BF6FF0090100E01521584C584D01F01F0242F49A
:2066F000F85222802A6812F0030F18BF0126D20828BF46F002060FB146F00406424692F9E8
:206710000740041B052C04DA9479B44208BF918866D00F28A0F10F0827DB08EB0014A4F15E
:20673000F0084FEA282EBEF1070F88BF4FF0070E7546062D88BF06255CF82570042404EB02
:20675000850465462C59E41B04F0FF05F70824BFC4F307273D44B70824BFC4F307473D4409
:20677000770828BF05EB146501E00025AE465CF82EC0F7080CF0FF0424BFCCF307273C44B0
:20679000B70824BFCCF307473C44770828BF04EB1C64ADB2A9EB0101A8EB0E277D4300293F
:2067B00005F1800504EB1524D8BF012103F0FF0334254D43A9B259434FF6FF73B1FBF4F150
:2067D0008B4238BF191C802889B2918005DA10F1800FB8BF6FF07F0000E07F20D071967131
:2067F000194800681F2910604FF0000008D340F2FF128A4206D24908401C8A42FBD301E0DF
:206810001F219180124F0F39090940EAC10047EA0001CAF8FB1F0026CAF8FF6FBDE8F087F1
:206830000C490D4F424608200F60921D1070BDE8F087C0463C1100506E62084024220840E4
:20685000A82E00209C130050082009403500094000E7A48030100940FDFDA400AC3F0050D7
:206870002DE9F04F0128ADF1140D40F0EE80DFF814B2DBF8DC00012840F0E4800220CBF83F
:20689000DC0011F0AFFF029001200EF01DFD5FEA000806D00120CBF8DC00029811F09EFF73
:2068B000D5E011F097FF6C49039000200860012010F046F9012818BF002003D100200DF03B
:2068D00017F80120654900900020654F08603868112011F0ADFD00280CBF00240124102016
:2068F00011F0A6FD08B144F002040F2011F0A0FD08B144F004040B2011F09AFD28B15948F2
:206910000068594E016B308888470A2011F090FD002600B101264FF0805A0AF5DC75301CFA
:2069300004D02868514E016B308888475048012606602868816944F0200088474D48066094
:2069500011F070FD00F001010191400814D24A4811F013FD8146B9F1040FF8D0B9F1010F5E
:2069700005D1DAF8D80142684348032190474349086820F0030008600020FFF75DFE2B68DB
:206990003868986B8047019801280DD0B9F1010F05D1DAF8D80142683748314690473749AC
:2069B000086840F0030008602C48066028684169204688470B2011F03BFD20B128682A4B39
:2069D000C16A188888470A2011F032FD20B12868264BC16A188888472548032206602549E1
:2069F000CBF8DC2000230B602868416B204688470128F9D1386804200EF066FC044616480A
:206A10001F490660386808688009FCD30098012802D130460CF06CFF11F0F2FC08200EF0AA
:206A300053FC07460398CBF8DC6011F0CFFE0DF0ADF8029811F0D2FE57EA040018BF4FF0DA
:206A5000FF3804E06FF0040801E06FF00108404605B0BDE8F08FC0460C40094000022243F6
:206A70002C200940B80100102EA201002AA201002820086080010443004003402422084081
:206A900014100940B80F0020804A2DE9F04F13680546ADF13C0D0DF12A00036052684260DF
:206AB0007B4C94F8B30005F1280105F12807002800F0E8806878002840F0E48011F052F914
:206AD000DFF8D091DFF8D48100B3042046466A68A873301D12780068042A00F0958095F8F3
:206AF0003000022812D14846007801280ED06A4905F1280002220E46203110F01BFC28B9AA
:206B100006F1160105A811F095FD05AF686E002800F0B880012102AA0AF0CAFB002840F058
:206B3000B1809DF80800A873E86C40B139460DF11E0208ABFCF7EEFC002840F0A38008A8BF
:206B50000090686E39460DF11E0306F0BFFF002840F0988048460078012851D04FF400501A
:206B70000DF122010DF034FF0DF122000DF12A01082210F0DFFB38B10DF1220039460822B5
:206B900010F0D8FB00283BD194F85900002837D0A66CB4F8445042F2010004A90DF018FF82
:206BB000049A4FF000410020E2FB0610061C206D11F0E6FA86190498B04202D86D1C361A24
:206BD000ADB24746786880475FFA80F8206CB04204D1208FA84208BF002608D0266425875A
:206BF000002084F8350010F0A1FC0126E064B968404688470EB10BF0BDFC012084F85800CE
:206C1000002084F859003DE08B468047264C0D9095F8307022480A264FF00009804610F8CE
:206C300007A0207AB84206D152462046594610F00DFD012804D0761E04F10C04F1D100E053
:206C5000A1465FEA09070FD198F80601164F461C810088F8066101EBC001F0B27F180A2826
:206C700004BF002088F80601384659460A2211F009F90C48094900788968B8720D988847A1
:206C90000420A8730FB0BDE8F08FC046B0A40100A82A002021150020340F0020C0150020C7
:206CB000CC100020E01900205A1100202DE9F043002B08BF002A10D10029BCBF00204FF0DB
:206CD000004106DB50EA01071CBF6FF000006FF0004109F08AF8BDE8F0835FEA530898EAAD
:206CF000610803D50026404266EB01015FF0000913F0004E03D00026524266EB03031C4659
:206D10001546002C08BF8D429CBF2C1C0025070C47EA01470E0CB44208BFBD429EBF240497
:206D300044EA15442D04070A47EA01670E0AB44208BFBD429EBF240244EA15642D02470865
:206D500047EAC1774E08B44208BFBD4200F29280870847EA81778E08B44208BFBD427BD847
:206D7000C70847EA4177CE08B44208BFBD4265D8070947EA01770E09B44208BFBD424FD8C9
:206D9000470947EAC1674E09B44208BFBD4239D8870947EA81678E09B44208BFBD4223D81F
:206DB000C70947EA4167CE09B44208BFBD420DD8E60146EA5566EF01B14208BFB84201D358
:206DD000C01BB14159EB09094EEB0E0EA60146EA9566AF01B14208BFB84201D3C01BB14154
:206DF00059EB09094EEB0E0E660146EAD5666F01B14208BFB84201D3C01BB14159EB0909EB
:206E10004EEB0E0E260146EA15762F01B14208BFB84201D3C01BB14159EB09094EEB0E0EFB
:206E3000E60046EA5576EF00B14208BFB84201D3C01BB14159EB09094EEB0E0EA60046EA9C
:206E50009576AF00B14208BFB84201D3C01BB14159EB09094EEB0E0E660046EAD5766F0018
:206E7000B14208BFB84201D3C01BB14159EB09094EEB0E0EA14208BFA84201D3401BA1415D
:206E900059EB09094EEB0E0EA34208BFAA423EBF2D0A45EA0465240A8AD373464A465FEAB6
:206EB000080803D50026404266EB01015FEA480803D50026524266EB03031E4617460B464B
:206ED000024631463846BDE8F0832DE9F043044694F830900F46984615468B20ADF1340D56
:206EF0000DF10A0104F062F88A20694604F05EF894F8250000283ED1B9F1000F19D1BDF848
:206F10000A104FF6FE70884205DCBDF80A1088422FD1694615E0B4F844009DF80A608DF838
:206F30000C0000128DF80D00BDF80A008DF80E601BE0B9F1020F09D0B9F1030F19D104F1B5
:206F5000280103A811F076FB092612E0207CC00934BFB4F84200B4F844008DF80C000012E1
:206F70008DF80D00208D8DF80E00001205268DF80F00002013E002280CBF052609260128D3
:206F900018BF04F11C0104D1892006A904F00EF806A9324603A810F075FF94F8260006EBE8
:206FB0000D01C8723A4603A831460BF0A7FA002840F08E80B9F1000F19D1BDF80A104FF61E
:206FD000FE70884205DCBDF80A1088422FD1694615E0B4F844009DF80A608DF820000012A5
:206FF0008DF82100BDF80A008DF822601BE0B9F1020F09D0B9F1030F19D104F1280108A812
:2070100011F018FB082012E0207CC00934BFB4F84200B4F844008DF8200000128DF821009F
:20703000208D8DF8220000128DF8230004203E6881460BA9822003F0B9FF9DF82C10307B24
:207050008142D8BF9DF82C00002841D007460024722029460FF020FFB0689DF82C1020181B
:20707000C8F80000007881422EDD2B68C10001EB0011D8F80000C91829604278012A1FD09B
:20709000807828BBB9F1040F06D0091D08A810F05BFD012816D017E008884B888DF828002E
:2070B000042208A98DF82A3000128DF8290018128DF82B000AA810F0C9FA012802D003E01D
:2070D000807828B9002004E07F1E04F10304BFD1F3200DB0BDE8F0832DE9F04F7C4C074648
:2070F00060688946ADF11C0D8047A046714E724D6F4C8346012F68D010F094FE00285FD022
:207110006348007800285BD162480078002857D161480078002853D16048007800284FD1A1
:207130005F48007800284BD15E480078002847D15D480078002843D15C48007800283FD1D1
:2071500000200BF073FB00283AD127463878002836D1286A436CF068022104AA98479DF839
:20717000100068B32C46B9F1010FBA4635461ED0524F226AE86897F9001011F1020F05D03A
:20719000926B97F900109047E868226A4C4E96F9001011F1020F05D0926B96F900109047FB
:2071B000E868226A6FF001013170397001E0E868226A01218AF80010D169884700206070CE
:2071D000D8F80810584688475EE001200BF02EFBD8F80810584688473A4800780F2842D12E
:2071F0002078012842D1384F97F8C2000028FBD1286A436CF068022105AA98479DF81400EC
:2072100068B197F8C20050B9207801282ED10020B9F1010F207029D010F010FE26E0D8F8E4
:207230000400804702222270002302938DF80C20284F7B8181468DE80C00274BF068083790
:20725000394602AAFEF7B2FF002C01D511F000F8224991F90000401C0870D8F80810EF6052
:207270004846884702E0484607F0FEFA2078174D022803D1287808B110F0EAFF287801283D
:2072900002D020780228FCD007B0BDE8F08FC046C22E0020C42E0020C62E0020C32E002056
:2072B000C52E0020921B0020931B0020941B00209F1B0020E019002018170020901B002034
:2072D000911B0020410F0020182900209E1B0020C0150020D8120020894401009A1B002086
:2072F0002DE9FE437B4E80460F46B8F1450F06D13046342210F0C6FDC6F89C60E7E010F05F
:2073100052FA3B2808BFF42000F0E280724C04EB8004A07810B9E178002938D0E1788142C9
:2073300008BFFB2000F0D480B8F1580F25D0B8F1600F1BD0B8F1E00F0FD0B8F1E80F05D023
:207350003A78904220DC91421EDB20E006F1E7003978007881421AD1B9E097F900000CF0F7
:20737000F7FA4FF6FF7181420ED010E038880A280ADBB0F5804F07DA09E038888F2803DB5C
:2073900046F2B041814202DAE820BDE8FE83544D686880478146207862783946801994309A
:2073B00010F070FDA968484688474046503800F08C80801E73D0401E00F084808D387CD094
:2073D000401E63D0401E75D0801F1BD00D387ED10E2096F815718DF8000017B11B208DF8FC
:2073F000000096F9D6109DF90000884203D0E0206946FFF775FF10F029FB96F815010028CC
:2074100041D164E0032096F8E7108DF8010081294FF005008DF8020006DB842904DA8DF872
:20743000010008208DF802009DF8010096F8B910884204D04F200DF10101FFF751FF9DF8B7
:20745000020096F8C510884204D057200DF10201FFF746FF214C94F83800A0B110F082FC66
:2074700088B1E26E7AB1022000278DF803000DF103018DF8047042F21B009047E26E42F2D2
:207490001C0001A990470CF01BFD20E096F8D7000DF0DAF901281AD01A20BDE8FE8396F8F5
:2074B000BD0018B902200EF05DFB10E0022010F00FFF0CE010F086FC09E096F9D60010F0DA
:2074D000F1FD04E010F08AFC01E010F0E1FD0020BDE8FE83A00E0020889A010020150020F9
:2074F000C01500202DE9FF4707467878002840F0E78097F8961002291CBF0329E82097F831
:207510008B108029C8BFE82097F88C10092901DB0A2900DDE82097F88D1009B1042905DB44
:207530008029C0F2CC80862980F2C980002840F0C780684C04F1E7000078884204D007F1ED
:207550008D01E820FFF7CCFE07F18C01E720FFF7C7FE07F18B01E120FFF7C2FE07F19801B2
:207570005020FFF7BDFE97F8960002280CD04FF6FE70A4F8B40007F18E0104F1AA0011F085
:2075900059F807F18E0504E007F18E052888A4F8B400514807F180010B2210F073FC4FF0A3
:2075B00001080220A7F816802946387501A810F0D9FA97F89A60B7F89890786807F19A01F0
:2075D000002EA0F1010078600CBF002040464E780EB140F002008E780EB140F00400CE789C
:2075F0000EB140F008000E790EB140F040004E790EB140F0800079684A1E7A60374B08707B
:207610003E7D7968481C3862701E0026087038893E65801C38811878BE65002840D04FF0B1
:20763000040A87F86960F88A87F86BA0C00934BF94F8B90094F8E20087F86A00296807F1F7
:207650006C0001602B8903816C68446010F08AFB30BB07F16C0007F18E0110F0EBFF204CEC
:20767000206810F47F0F0CD087F82CA0206807F12C01424600F47F003863384602F05AFDAF
:20769000206810F0FF0F0BD02A2087F83C00206807F13C0100F0FF003864384607F04CFB60
:2076B00000963846832101AA4B46FCF76FFB061C02D1384607F06AFC301C01D106E0E8208D
:2076D00078701820387038460CF0AAFC0090BDE8FF87C046A00E0020A02C002058150020AA
:2076F00098A001002DE9F047064637680C465FEA0208ADF1180D14BF00214FF0FF3107F146
:207710004800814611F05EF8002808BF0B2000F0DF80002565707148FC60B8F1010F05704D
:2077300004D065700220FC600FF032F82078012840F29080801E012857D9801E01282CD923
:20775000801E012800F2B88011F05CF88246A078009021782846062908BF01200190012093
:207770000290A068228A6368E16807F04DF90746504611F043F8002F40F0A080B8F1000F0C
:2077900002D010F0E3FA02E030460FF0C3FC002800F0878010F062FF21E011F033F801273F
:2077B00082460097A168A278606824782B46042C08BF3B1C08F0BCFC0746504611F01EF86A
:2077D000002F7BD1B8F1000F02D010F0BFFA02E030460FF09FFC002863D00EF079FF3E4991
:2077F000C1F8B0510D60074668E011F00BF88246E08A0090E0680190208B0290A078039036
:20781000207D04900121059122782846022A08BF081CA368E178626802F0CEFE0746504681
:2078300010F0ECFF002F49D1B8F1000F02D010F08DFA02E030460FF06DFC002831D00EF00C
:2078500077FF071C3AD1E078A168E28A23690AF03DFBC8E710F0D6FF8246E08A0090E0685B
:207870000190208B0290A0780390207D049001200590277807B90546E1786268A368284652
:2078900003F014F80746504610F0B8FFB7B9B8F1000F02D010F05AFA02E030460FF03AFC64
:2078B00008B9142014E00EF02BFF071C06D1E07821690CF001FF96E74FF0FF37B8F1010F24
:2078D00002D002200EF008FD484610F093FF384606B0BDE8F087C04650450240C02E002046
:2078F0002DE9FE4F794C074694F83D00002800F0DA80DFF8DC81B7F84210B8F8BA0088425F
:2079100040F0D18007F128000FF07AFB002800F0CA80002598F8BD0084F83D5010B1022082
:207930000FF074FE6148007810B101200FF06EFE387C400905D310200FF068FE802010F04E
:20795000CFFC20200EF00EF9594E06F120000CF0A3FF7A6851781078334600EB0120C0F340
:207970000321C0F3003684F8391000F00F0184F83A60C0F3031684F83E1098F8E30088F886
:20799000C0600F2804D0884202DDD67806B9014688F8A11098F8A1A083F84050BAF10F0FD9
:2079B00009D194F83B0002287DD10EF017FD07F0E7FDBDE8FE8F3F480078012803D0012063
:2079D0002946FFF789FB43484068804700900FF08DFC3948DFF80091DFF8E0B0066898F84E
:2079F000A12099F80030D9F80400311A980091FBF0F05BF822100DF00DFFC9F804605BF8CB
:207A10002A0001912E4EB060F0600DF09FF8019831680EF017FD09F0BDFE2E490098896832
:207A3000884794F83B0002280DD127480CF034FF98F8A12034F812004FF470719140091A53
:207A500021480FF005FB98F8C030388929460CF0E9FC20630F2B14D098F8A11094F8390076
:207A7000994208D0401C6FF00F0598408101A1EB80016D1805E0401C98408501A5EB8005D4
:207A9000A03D6563022004F1200584F8380028460CF002FF0B48A062616B28460FF0D8FA76
:207AB000102010F01DFCBDE8FE8FC046AB2C0020A02D00209E1B002058170020D4A2010072
:207AD0007C1B0020D51B0100B02D002038190020A00E0020C0150020201B00202DE9FE4FFF
:207AF0000CAF89469A4604467D680292294604F05FF9061C00F0D9803888F082DFF8CC81CD
:207B1000347598F8380018B1012C04BF1520307506F1800029460B2210F0B4F9012C04D090
:207B30000D2C1CBF7068401C00D170683062002598F8380035650028B5654CD0052C18BFC5
:207B5000012C43D14FF0040B86F86BB0F08A86F86950C00932BF57485D48163000780299E5
:207B700086F86A000A6806F16C073A604B687B600889388110F0F6F840BB06F16C0010F073
:207B900059FD4D4F07EB8407386810F47F0F0CD086F82CB0386806F12C01012200F47F00A4
:207BB0003063304602F0C6FA386810F0FF0F4FF003090BD02A2086F83C00386806F13C014E
:207BD00000F0FF003064304607F0B6F898F8380008B10D2C13D00095029A5346304649468B
:207BF000FCF7D4F8071C61D1E41F012C03D8707E40F020007076304607F0C8F956E010F0CE
:207C1000B1F8294600B101212B48343009B94FF00309052186F86B10016811F0F70F12D014
:207C30002A2186F83C1098F80120006806F13C01012A00F0FF0030641CBF20F0080030649D
:207C5000304607F079F80095029A534630464946FCF79CF8071C29D1184806603489756863
:207C700001A964200DF076F8154E6D1E231DA01C99B2A6F87800C1F3022040F0080005F805
:207C900001090A1F297091B2AA1CC6F88450104609F014FF9DF8040000280CBF09480A48DC
:207CB000C6F8C000C6F8800000E01A27F8B2BDE8FE8FC046590F002090A00100141A0020EE
:207CD000D81200204E9055550E7A5555201500206C0F0020754A2DE9F84F074621F0004026
:207CF000884682420AD9724981422DD955A20CCA4146384601F01BF9BDE8F88F6D4A0FF2C0
:207D10004C1982420AD8C0F3130057EA000601D1080815D238460B460246EBE74DA20CCAC4
:207D3000384609F046FE98BF0FF2301905D94DA20CCA384609F0FAFD06D85F492220086096
:207D500099E80300BDE8F88F48A696E80C004146384601F0ECF805464FF4002202EB05323D
:207D7000120D140596E80C0001F0DCF80B4602464146384601F0D6F8504B803505F0FF05C6
:207D90006A0003EBC20595E88001561C03EBC6030CCB01F0C7F84A4D89468246A542CCBF66
:207DB000484E494E4B4652464146384605F0CEF930A200900CCA8B464946504605F0C6F9BA
:207DD0002EA20CCA01F0B3F84B46524605F0BEF92CA20CCA01F0ABF836194B46524605F0D7
:207DF000B5F92AA20CCA01F0A2F84B46524605F0ADF928A20CCA01F09AF8024600980B4680
:207E1000594605F0A3F90B4602464146384601F08EF8A5420BDCB4F1804F05D10B4602465C
:207E300001F085F81DA207E03346002205E03346002205F08BF91BA20CCA05F087F9BDE8DD
:207E5000F88FC046000000000000F03F000000000000000000000000000090400000000086
:207E70000000F07F0000000000CC90C0000000000000B842745C870380D8553F0004F788A4
:207E9000ABB2833FA6A004D7086BAC3F75C582FFBDBFCE3FEF39FAFE422EE63F000000003B
:207EB0000000E07F0000000000007001000090400000903C0000F07F301C002028880100BA
:207ED000000030C00000707E0000F03F2DE9F0411C4615468C4208BF854282BF002300229F
:207EF000E5E0002C08BF002D0AD100290EBF00286FF000006FF0000100F0E1F8BDE8F081F6
:207F10005FF000085FF0000E002C08BF8D429CBF2C1C0025070C47EA01470E0CB44208BFB0
:207F3000BD429EBF5FEA044444EA15445FEA0545070A47EA01670E0AB44208BFBD429EBF4F
:207F50005FEA042444EA15645FEA0525470847EAC1774E08B44208BFBD4200F29380870828
:207F700047EA81778E08B44208BFBD427CD8C70847EA4177CE08B44208BFBD4266D807098A
:207F900047EA01770E09B44208BFBD4250D8470947EAC1674E09B44208BFBD423AD88709CF
:207FB00047EA81678E09B44208BFBD4224D8C70947EA4167CE09B44208BFBD420DD8E60141
:207FD00046EA5566EF01B14208BFB84201D3C01BB14158EB08085EEB0E0EA60146EA9566D7
:207FF0004FEA8517B14208BFB84201D3C01BB14158EB08084EEB0E0E660146EAD5666F015D
:20801000B14208BFB84201D3C01BB14158EB08084EEB0E0E260146EA15762F01B14208BF87
:20803000B84201D3C01BB14158EB08085EEB0E0EE60046EA5576EF00B14208BFB84201D385
:20805000C01BB14158EB08084EEB0E0EA60046EA9576AF00B14208BFB84201D3C01BB141B6
:2080700058EB08084EEB0E0E660046EAD5766F00B14208BFB84201D3C01BB14158EB080850
:208090005EEB0E0EA14208BFA84201D3401BA14158EB08085EEB0E0EA34208BFAA423EBF79
:2080B0002D0A45EA0465240A89D3734642461E4617460B46024631463846BDE8F0817047FA
:2080D000F0B542F20400ADF11C0D0DF115010CF07FFC42F2050005A90CF07AFC664C6748A7
:2080F0009DF81510A0666420414321666449C4F884109DF814104843E0676248C4F8A00093
:208110006148007880B942F2020069460CF060FC68460FF07BF904F15C000CF087F804F1D6
:2081300034000CF0A1FA27E042F2030069460CF04FFC0EF0C9FF0546684629460BF068FEA1
:208150002D1A04F1780084F85B500CF06FF804F134000CF015F8012742F20200694684F816
:2081700054700CF035FC68460FF050F904F15C000CF05CF884F85870E8200DF116010CF00A
:20819000E9FD9DF81600032804BF012084F8B40094F8B80000286DD13C4D0021302205F163
:2081B0000C000AF009F82046002133220AF004F837482862374FAF6105F114000CF036F803
:2081D00042F21B000DF117010CF002FC9DF817000DF1170185F8300042F21C000CF0F8FB82
:2081F0009DF817109DF8170085F8311095F83010012641B148010EF03FFF686308B910F052
:2082100023FA95F8310040B100EB800080B20EF033FFA86308B910F017FA1F4905F13C003E
:208230000A270A684B6802607F1E436000F10800F7D1002195F8307085F88C1047B1686B43
:20825000FF220346C2777F1E997703F12000F8D195F8317047B1A86BFF22034602717F1E2E
:20827000D97003F10500F8D1281D062209F0A4FF84F8B86007B0F0BDA82A0020494901005D
:208290002D030100D985010021150020CC10002021C00000002A7515C0A401002DE9F041AB
:2082B000704B714ADFF8B8810C46D128014610DCD12878D0713800F0B080401E00F0A98029
:2082D000401E00F0A280113810D04C3800F0868007E0D23853D0401E40D0401E33D0401E3A
:2082F00028D008460FF070FF0B2802D1F420BDE8F0815A4D05EB8005A97809B9E87850B12A
:20831000E878884208BFFB2000F0A6802278914269DC904267DB554E7068804729786A78A0
:2083300007464046401821460FF0ACFDB1683846884790E02178022955DA1846641C042226
:2083500000EB810084E0207803284CDA1746C100241D182201EB0011781879E026783046C1
:20837000022840DA2C2505FB0680611C102239300FF088FD616905FB0680C1646BE02278DC
:208390006178022A2FDA02292DDA40462C2301EB42064F1C03FB0205022285F8387000EBE0
:2083B0004600A23018E022786178022A1BDA032919DA2C23404603FB020595F83030994248
:2083D000A4BF4B1C85F8303002EB4202891801EB4101032240189030A41C39E02078677859
:2083F000022800DA17B1E820BDE8F08141462C22C5197E1C02FB00136A0083F8286002EBCC
:20841000C50288180A227C30E6E724B3184608221EE004B3104648221AE0B4B9404600F18E
:208430007C04A0F1080200F1900300F1A201022042F82C4F9360401E116104F10A0403F168
:20845000090301F10401F3D105E040465822243021460FF017FD0020BDE8F081E49C0100DB
:208470003C27002030280020E8270020C01500202DE9F043071CADF1240D00F0D880F86BE7
:20849000002800F0D480B7F84020002A00F0CF80007817F130014FF0000603D097F8381048
:2084B000052902D0002E00F0C280DFF88C91401E2ED0801E18D0C01E40F0B980012A40F0D4
:2084D000B6805C4C0725E0788DF81C5000280CBF0121311C3046E1700AF046FCE078022258
:2084F0008DF81D0028460EE0012A40F0A080B9F86000401CA9F8600002200FF07FFB0420C6
:2085100001228DF81C00394607AB03F0A9FE8EE0684631460C2209F04FFEB7F840000B2893
:208530005ED1FC6B14F8010B89F82C0025786078A41C05EB002520460FF026FD0346201D78
:208550000FF022FD8046387A4C4689F82800022806D0396804F1200001607A68426001E0BE
:208570003888208405F00100A90828BF40F00200E90828BF40F00400A90928BF40F02000D2
:20859000290A28BF40F08000290928BF40F00800690928BF40F01000E085854218BF0226EC
:2085B000B3F57A7FADF8020007D32448984204D3236318460EF01CF900E00226206BB8F535
:2085D0007A7F019008D342F21070404504D3C4F834800FF0F9FC00E00226606B029001E06C
:2085F0004C46012602258DF8016068468DF800500CF08AF80DF10D009DF801108DF80C5012
:208610000FF028FFBDF802100FF024FF01990DF07AFB02990DF077FB39460D2203AB28465B
:2086300003F01EFEB4F86600401CA4F8660009B0BDE8F083D4110020B8130020407E050027
:208650002DE9F843644C0746207808B10FF000FEA0460120614988F800000978012902D0C0
:208670000021FEF739FD5F4D60495F485C4C012F2A68D1F800900078A77035D9BF1E52D043
:208690007F1E13D07F1E02D0781E47D043E092F86900607192F86A0020710020A07103F09E
:2086B000B7F92A68002A64D1BDE8F883002860D0564ED6F8981021B1032088472A6896F893
:2086D0003800002855D0776D002F52D0D06D20B102210023B8472A68776D106E002848D049
:2086F00008210023B84743E000206071D18A4048C90934BF90F8B91090F8E2102171A778E7
:2087100037B990F897701FB10229C4BF0220207103F07EF92CE00FF09BFD29E00020607192
:208730000FF0B6FF24E0334F38788600D9F83C00804779683C22401AB0FBF6F0B0FBF2F12D
:2087500051436278401A9101A1EB8201091AD9F83C003C318FB28047274906FB0700086714
:2087700091F8740000F0F00040F0020081F874002A682248007878B912B90FF069FD2A6886
:208790005168087800F02000E0708878E0710878800901D20FF07CFEA078042819D0184DF8
:2087B00068688047A17802290CD016490F7817B915490F7837B1022188F80010A9688847DC
:2087D000BDE8F883832188F80010A96888470EF09DFFBDE8F883C046C62E00209E1B0020A8
:2087F000401A0020700D00205815002038170020A00E0020201B0020D8120020BE2E002017
:20881000C0150020C22E0020C42E0020201500202DE9BC4305466D4800880021820804D2BE
:20883000B5F89A20D20828BFE82110F0600F04D1B5F89A00800828BFE8212889B0F5006F2F
:20885000A8BFE82195F8980030B995F89400002808BFF52100F0B580002940F0B280DFF8DD
:208870007091D5F8A800DFF8708199F8381010B9012903D02BE0002900F0A2800FF072FA5A
:2088900068B9D5F8A8104046BD3041F002010078C5F8A81018B141F00801C5F8A810D5F849
:2088B000A81011F0FF0F05D02A2085F83C0001F0FF072F6411F47F0F07D00420D5F8A8700C
:2088D00085F82C0007F47F00286399F83810002069B3404995F894700B6804226FB92523A2
:2088F0002B750968C98AC90934BF98F8B91098F8E21085F86A10891C08E015212975D98AA9
:20891000C90934BF98F8B91098F8E21085F86A1085F86B2005F18C0785F869003B6805F1A0
:208930006C010B607C684C603B890B8101E00121297595F89C70EF760446AC65B5F89A101E
:208950002C6595F89D30E9826A682B7795F82C702A620F2F09D00246B5F8A40005F12C01B5
:2089700000B90122284601F0E5FB28BB95F83C10FF2901D1AF6D27B105F13C01284606F08B
:20899000DBF9C8B9009495F89810B5F8963005F18C022846FBF7FAF9071C0CD12889B0F509
:2089B000006F03DA284606F0F1FA04E0E520687028460AF0DFFD3846011C02D1BDE8BC83B5
:2089D0001821284608F0C0FABDE8BC83BC16002020150020700D0020A00E00202DE9F0434F
:2089F000894614460546ADF12C0D69460DF0BCFB5FEA000800F0C480AD1C0226284602A92A
:208A10000BF0E1FD071C00F0BB809DF80900814509D0F6197D1908F10200B61CAD1CB6B23F
:208A3000B042EBDCACE0401E05F1020500F08B80401E52D0801E38D0401E2BD0401E24D0BA
:208A5000401E18BF622040F0AB80202F40F0988028686F6805F10801206004F108066760AD
:208A700001F108050A684B68326004F1100773602A6868683A6005F108067860306804F1EC
:208A90001801086073684B6089E0022F78D12888208084E0202F73DC20460021202209F0C8
:208AB0008BFB3A462046294677E0042F68D12888AD1C208015F8010BA070287800F0010035
:208AD000E0702878C0F3400020712878C0F38000607128784011A07161E00A2F50DD0DF1C7
:208AF00012000021162209F067FB28682D1D20602988271D42F20B00398004A90BF068FF4A
:208B1000BDF81000A18888423ADCA81C10F8011BA17110F8011BE17110F8011B217210F848
:208B3000011B0123C1F3C202A2720DF1120200F0D5FA28B39DF82700A0819DF81670E7814D
:208B500004F1100026E0042F1ADD0DF112000021162209F031FB15F8010B207015F8010B80
:208B7000607015F8010BA07015F8011B0DF112020023C1F3C2002071284600F0AFFA08B9BF
:208B900067200DE09DF82700E0809DF81670278104F10A000DF11601112207F08DFE002089
:208BB0000BB0BDE8F083FEE72DE9F04F684C2068ADF12C0D002840F0C78004F1240630682F
:208BD000002800F0C18063480078022800F0BC80624D281D006880470A90606AB0460746E9
:208BF00078B35D4E4FF0000A4FF01D093B7D0820711E11F8012F9A421ED0401EF9D14046C1
:208C1000394652460DF008F8787E30F07F0005D194F82F00401E84F82F0004E094F82E0063
:208C3000401E84F82E0087F8019057F80CBC38460AF0A0FC5F4602E0BA4657F80C7C002F54
:208C5000D4D1352007F020FF454EA968002849D1452007F019FFA96800283DD1D8F8000083
:208C700038B1017D252904D050F80C0C0028F8D110E078B196F8580050B3684601A907F0B9
:208C90009DFB384800990078001F884213D8012086F85500152007F0F7FEA96848B10A9806
:208CB000884720680DF106016C3000F0A3FC58B10FE00A9847E0252007F0E6FEA9680A9889
:208CD0008847002086F855000420FFF7B9FC3BE0192001F099F837E00A98884708200CF071
:208CF00015F831E00A98884796F8B400B8B10EF0EDFB317800290EBF0921491EC9B201EBAD
:208D100081017118D1F802100FF0A0FC42F21071814292BF00206431081AC0B200E00020B0
:208D30006968002808BF0620D9D0C6F8980088470446D6F8A010D6F8980006F1A8020DF0A3
:208D500063FAA968204688470BB0BDE8F08FC046700D0020CB170020D0A40100C015002072
:208D7000A82A0020932B00202DE9F843664C002605466676687D0628A4BFE8216176A97D47
:208D90000E2903DD03281CBFE8216176032805D15E48008840083CBFE820607695F82800C1
:208DB00008B1E8206076E87D092801DB0A2801DDE8206076287E08B1042805DB802801DBBD
:208DD000862801DBE820607604F11807294638460DF0ECFB291D112207F12C0007F06CFD39
:208DF00095F8280004F11809002804BF84F86060A87D04D095F8290084F86000688DA4F855
:208E10005600687E84F85800A87EDFF8048184F85900E87E822784F85A00287F98F8D76088
:208E300084F85B0098F8E63084F85C70394F84F85D6005F11D01E763042684F8406098F868
:208E5000E72084F85E3009F1490084F85F200B220FF018F8607E00284ED1687800284BD12E
:208E7000287EA77E8DF800000FB1EA20607605F11701E720FEF734FA94F8600028B1287E4F
:208E9000022808BF01208DF8000098F8E7009DF80010884203D0E8206946FEF721FAA77E86
:208EB0001E4C601C007808B10FF0D2F9B8F8BA0019490880C7B1032F12D0052F05D0012FA8
:208ED00003D0022F01D00FF0C3F9022060700CF0B7F94FF6FF70A8F8BA001149088005E07F
:208EF0000CF0AEF9032000E0012060702720287030460EF08BFB01E02A20287028460BF0C6
:208F10008FF8BDE8F883C046E42C0020BC160020A00E0020F1820100EA1900200C2E0020B3
:208F30006A1700202DE9FC4F83F0004301E02DE9FC4F1F03FF0847EAD2574FEA42284FEAC8
:208F500043095FEA595906D147EA080A1CBF00210020BDE8FC8F57F000575FF4E06E1EF106
:208F7000FF0EF14505D14FF00000190D0905BDE8FC8F002B05D55FF0000AD8F100086AEBA1
:208F900007070C03E40844EAD0544FEA40254FEA4106760D08D144EA050A19BF0021002096
:208FB000191C101CBDE8FC8F44F00054764504D10020090D0905BDE8FC8F002904D55FF033
:208FD000000A6D426AEB0404B6EB090E08D5A2463C465746AA464546D046CEF1000E4E46DD
:208FF000BEF1360F5CBF4FF0000B23E0BEF1000F04BF4FF0000B1AE0CEF1390ABAF120096A
:209010002EBF08FA09FB07FA0AFB4BEA080BDEF1200A07FA0AFA38BFBA4647FA0EF72DBFD8
:2090300028FA0EF8AEF1200E4AFA0EF8D04415EB08057C4154EA050A02BF00210020BDE80F
:20905000FC8F002C58BF4FF0000A06D55FF0010A5FF0000E6D426EEB0404A6F101066D003C
:209070006441FAD515F4806E11D005F480794BEA090B15F5806554F1000428BF761C0BD2CB
:2090900005F400795BEA090B08BF25F4006525F4E0656D0044EB0404B61CDEBF00210020FE
:2090B000BDE8FC8F5FF4E06E1EF1FF0E76450AD34FF0000013F00043FF21C900C91D0905B9
:2090D0001943BDE8FC8F270547EA1530210B41EA065141EACA71BDE8FC8F70472DE9F04F02
:2090F000154601F00708C1F3C2074FEAA119044683460C22ADF1240D0021684609F05CF869
:209110006248B8F1000F36D0B8F1010F7ED1228801A9A6780A80E41C8E7014F8011B01F0BC
:209130000F018DF8081022880DF10A031A80BDF80A30A41C4FF0000C6B75019ECDF818C00D
:209150004168B14207D1017A9DF80820914202D14189994208D006990C30491C062906912A
:20917000EED96046614601E0017840788DF800108DF8010022E014F8013B14F8016B8DF857
:20919000003000228DF801600C38079210F80C1F994202D14178B14207D00799491C062912
:2091B0000791F3D91046014603E04168027A4089687501918DF80820ADF80A0003A806F061
:2091D00065FF9DF800109DF80100B8F1000F11D0B8F1010F1AD1019904989DF808209DF81B
:2091F0001460484086EA02010918BDF80A20BDF8160004E09DF80C2051409DF80D2050409D
:20921000401803D1EF701FB1022F05D0002039E02188281DA41C0180B9F1010F27D0B9F11A
:20923000020F2CD1BDF80A10281DC91DCA10214607F042FBBDF80A00C11D04EBE104F0B18F
:20925000401E811000EB5171C910C9B26D182B798710012600EB577121F00701401AC0B28F
:20927000401C06FA00F0FF301840287107E0291D20460BF07FF9207804EB8004641CA4EB52
:209290000B04A0B209B0BDE8F08FC046701700202DE9F04FADF1840D209002F055FC0EF05E
:2092B000E7FA0026012804D10EF0E4FC022808BF01265B490868C0F38150012806D151F8C2
:2092D0000C0C0127010E07FA01F00643554800780DF07CFF544D2C46286038B1FF2204F1CD
:2092F000400107467F1E01F8012BFBD1209909684FF0000901F0FF02FE2A1DD0DDF880C0B4
:2093100001F0FF074A460123FF2F0ED0B84203D903FA07F73E4201D002207EE001F0FF01F3
:2093300047EA0909611881F840205CF8041F521C01F0FF07FE2FE7D1092006F0F3FA209803
:20935000002124220823606017A80FF037FA4FF0010804F1240017AA8DF8748041460FF09B
:2093700029FA236843B3002794354FF0040BBA4608FA07F0064219D119EA000F04BF07F004
:20939000FF0141F4C04105D0E019209B90F8401053F82110254804F05FFDF8B24FF0FF31D4
:2093B0000EF090FA2368C5F800A001E0C5F800B07F1C2D1D9F42DBD301A800213022082324
:2093D0000FF0F4F91A4E30780025102101AB0990184A009504F108000FF0E4F90DA8282217
:2093F000082329460FF0DAF90DAA7068124914952B46139004F160000FF0CCF90F4951F890
:209410000D0C474620F4F85040F4005041F80D0C0B4EC1F8FF7F2846376021B0BDE8F08FDA
:20943000B43F0050BF2E00202C260020007FC767E0A40100F1780100B95001000D3009402E
:20945000080009402DE9FE4F544E0746301D00688047534C00258346A01C05701FB10DF052
:2094700009FC0AF0D5FA94F83800B04610B1E06B00B180470AF046F9DFF8749109F11C00A5
:2094900090F900000EF00EFE0DF00AFC0EF000FE0EF0A4FC0EF096FCDFF808A107270AF153
:2094B000240656F8040B00B180477F1EF9D13E480560456005614FF470018160C1600AF18F
:2094D000040007680FB10CF065F938484E4600688AF80E50BA3EC0B112E048460CF09CFD15
:2094F000029002A80CF056F921E048460CF094FD019001A80CF04EF914E068460CF04AF95B
:2095100008F08CF900280090F7D129480078012803D028460146FDF7DFFD2648264F05707C
:2095300007F12409786A0028DFD109F10409B86A0028D2D17D62BD622048A06187F82E50E4
:209550001F4BE36187F82F501E4A22621E4961621E4B87F830501E4AA362204BE2621D494F
:2095700063601F4A21631C4FA260204B65701D4967631D4FE16058462761D8F808106361CF
:20959000884706F1BD015220FDF7AAFE96F8D7000BF05AF92846BDE8FE8FC046C0150020DB
:2095B00020150020B01600207C1B0020B42E00209E1B0020C12E0020700D002053D30000FC
:2095D00027860100257201002188000089E30000DD750100D1820100B9C4000053CE0000DB
:2095F00059B60000E14301004D0601004D3601005A0F00202DE9F04F0546824660480E4662
:209610000178ADF1140D0EF0ADFB5F4C00283FD0DFF8808108F104000068012914D0287A8D
:20963000022835D15749504602220F4620310DF081FE38B903208DF8080007F11601684610
:209650000EF0F8FFEA4623E095F8089014F809A080470A274FF0640B8E340390207A4845D6
:2096700006D15246204629460DF0F0FF012804D07F1E04F10C04F1D104E00027F772A07ABB
:20969000BB463073D8F80810039888475F4672E021464FF0000864278B468D6B91F8310011
:2096B00086F81E804446D9460AE099F800106D1C2034ADB234E099F83100641C6D1DA4B2D8
:2096D000A04217DDE8780028F5D028790BF0CAFC514608220DF02EFE0028ECD1E878B0779F
:2096F000288800047060287986F80B80F077A87847463073DBF83440002F08BFBB46C5D0A2
:2097100086F81E8042F219000DF10A010BF060F90DF0FCFE83461D480178642745468146F8
:20973000A94228DDA07F0028BFD0E07F0BF09AFC514608220DF0FEFD0028B6D1E07A022877
:2097500003D0E07A58B1612710E0616858460EF07DFFBDF80A200E495143814201D9474676
:2097700004E0A07F6C2740F00800A07730462146202207F0A1F8384605B0BDE8F08FC046E8
:2097900021150020340F0020CC100020FC100020808D5B00C01500202DE9F04F0746880F42
:2097B000ADF1140DC0F0BC8000200AF00DFC62485D4E4FF0000900F11408C8F800900120B0
:2097D00048F81C6C0DF0E2FE58480EF007FE584DBC68CB4640F60A0605F1140095F820104A
:2097F0002A7995F82130A5F816908246C5F818B001F0F0010680012A85F8201003F0F00025
:20981000A4F8029040F0010085F8210001D17B7CC3B1B8680088A6F10801814208D0B0F576
:20983000C15F05D0218B4FF60F400840208304E0218A4FF60F4008402082B86887F81190AB
:2098500004F02EFDB868694604F06CFE68460EF017FD3346D91F4A1C00E03446666836B106
:209870003088834203D0814218BF8242F5D1C4F804A0607B00F0F000607305F13C000EF046
:20989000EFFE8068008881421FD082421DD03E8D06B397F8340097F83560C7F82CB000F002
:2098B000F00087F8340006F0F00040F0010087F8350007F12803AB619AF80D00A7F82A9003
:2098D00000F0F0008AF80D0004E0DA4605F1580080E80006B9680A8A4FF6FF301040088246
:2098F000D8F800000028FBD0A87AC8F8009070B901200DF025F901280FD0607B00F0F000FB
:2099100040F0010060730B480EF068FD05E00CF0CFF80028FBD00CF0E9F8B86848F81C0C7D
:2099300005B0BDE8F08FC04601010E0469390000A00A002021310100081004402DE9F84FAC
:20995000884605460DF06AFF01464FF6FF70884210D042F21C0BAB4509D0ABF10100A84228
:2099700005D01A38A84202D0001DA84205D10EF0F9F910B16820BDE8F88F534C480000EBE0
:20999000C1002418D4F8027017B9D4F8066016B3D4F80610B94208BF692000F093806078A9
:2099B000401E12D0401E09D0801E14D1D8F80000874200F2818081427ED30CE0B8F8000061
:2099D000874279D8814277D305E098F80000874272D8814270D33D4F78688047ABF11A0ACF
:2099F0002B463B4E0090A3EB0A03012B25D90A3B012B14D9DB1F3DD12078627800213018C7
:209A100008F0DAFB637840460EF074FB834298BF181C02D940460EF06DFB02462BE00DF034
:209A300053FBBF68B8F80010884243DD207862784146301806F040FF23E00DF045FB81467A
:209A5000404649460AF0E4F9BF68A9EB00005FFA80F9B9F1000F2DD0207862784146301886
:209A700006F02AFF1B485146A94218BF401C80F8009006E0627820784146301806F01CFF5F
:209A9000BF680AF11900A84204BF002086F887005846A84213D196F8870096F886104218AA
:209AB000322A01DC08430AD1022086F88600302586F887500098B8476A20BDE8F88F009882
:209AD000B8470020BDE8F88FB0980100C0150020642B0020022B00202DE9F843634C5C4D48
:209AF0005C4EDFF87881604F94F8E4100846401E0B2864D8DFE800F07E2C43062343062359
:209B100043067967042907D001220A2945F8212C14BF0220032004E0202045F8210C012061
:209B3000024684F8E200002045F8390C0827C5F8FF7FC5F8F37F45F8392CBDE8F883052944
:209B500014BF09200620002784F8E400376078E094F8E170383D0120002FC5F81B0004BF20
:209B70000620002102D00021F160032084F8E400032045F8010C31603068800861D294F8EA
:209B9000E4103548012703290ED00068456800216022052300914046A84794F8E40006288E
:209BB00014BF0A200720CFE700684568002160220523022000904046A8470420C4E70EF0E7
:209BD000E5FDBDE8F8832648264F0026012506600E203D6005F018FC02200CF07DFB84F8F8
:209BF000E45084F8E360BDE8F883002038600C25786024E04FF08059D9F8A001016820204A
:209C100088472C3D0F2045F8010C41F61D56C5F80360D9F8A401466800214FF4C0720723D5
:209C3000022540460095B047D9F8A401C66800214FF4C07207234046B0470120386084F8C5
:209C5000E45004F178000EF0D1FDBDE8F883C04639400C4038600C40A401001000A00C4017
:209C70002C500C4004800C4034600C40B80F00202DE9F04304466668A7680D46ADF1340DD3
:209C90000EF0C0FD3178012903D10EF0B7FD0020A9E04FF0010886F800800EF0AFFD287867
:209CB00070706878B07068687060A868B060E868F06028693061287D3075687D7075A87DF9
:209CD000B075A869B061287F3077687F7077A87FB0774FF00009C6F82090C6F830904D46FC
:209CF00075627563B562B56386F82C50102386F83C3086F82D5086F83D50786805F012FE74
:209D1000204605F0DFFB204606F056FF70B937480068C16838688847786805F075FB0EF062
:209D300071FD35700EF06AFD2C465BE001A82946302208230EF03AFD0694387BCDF8009082
:209D50002B4A0990B96801AB06F180000EF02AFD01A82946282208230EF020FD05942549CD
:209D7000386901AA2B46079006F19C000EF012FD01A82946242208230EF020FD8DF81C801A
:209D9000B07838B906F1D000294601AA0EF012FD19483061707838B906F1EC00294601AAE4
:209DB0000EF008FD1548F06001A82946242208230EF0E8FC0695ADF814501149079406F5E4
:209DD00084700A2201AB0EF0D9FCB969FA6906F140000EF0F0F90B4A06F16C0004212346EB
:209DF0000DF096F820460DB0BDE8F083D001001049CD0000115F0100B7850100AF850100B3
:209E1000ED0F0100218301002DE9F8435E4D804695F83800002798B12A6F8AB1D5F8900068
:209E300070B142F21A0069469047D5F89000804730B19DF8000018B1B8F1E10F08BF012732
:209E5000524A02F1E70000780CF032FD407B02280CBF05260126514C2068002800F0928088
:209E7000B8F1000F914675D0B8F11B0F02D1017D05296FD1B8F1E90F2CD05FBBB8F1E10F1C
:209E900016D10EF0ABF890B12068C18AC9080FD299F8C810817699F8B6104A1C89F8B620F0
:209EB000406881703046FEF7CBFBBDE8F8832068B8F11C0F1DD1216A002950D0884734493E
:209ED00000200978206001295CD00146FDF704F9BDE8F883F1200DF052FE2768B87E50B977
:209EF0000EF07CF820B12068C18AC90801D2CFE7206847462FE07868398907F0DFFD786869
:209F10000088000905D395F8380010B10BF066FE2768F88AC00811D3387E00F07F00387653
:209F3000387D032803D1787E40F004007876F0200DF025FEE168206888470FE01549012601
:209F5000B87E0E70401EB876F0200DF018FE12480078A8E70027477009F00CFB2068C08A7D
:209F7000000A0AD395F8380018B999F8D7000AF06BFC99F9D6000EF095F8002020601020C8
:209F90000EF0AEF9BDE8F88320150020A00E00209E1B0020BE2E0020421A0020700D0020CB
:209FB0002DE9FE43604C614D0E46B00959D35D4800F1280980464DE00178D0290EDBD02999
:209FD00009D181783970C17879700179B97085687D60C168B9600EF000F947E004F1080504
:209FF00028600AF01DF828460BF0D4FB3EE0884798F83010491E88F83010A9688847009826
:20A0100001788DF80410A0604778CFB1DC2F0DD0DD2F0BD0E42F09D0F32F07D0DE2F05D049
:20A03000DF2F03D0E82F18BFDB2F0BD104F0A4F99DF80400162805D168460BF0ABFB01E0ED
:20A0500009F0EEFF9DF80400162803D004F108000BF0A0FB48460BF0DFFF002869680090DD
:20A07000C5D1F00BA846C00305D0314F07F0D6FB00280090A0D1700905D32E208DF8040020
:20A0900001A809F0CDFF700805D325208DF8040001A809F0C5FFB00805D326208DF804005F
:20A0B00001A809F0BDFFF00805D327208DF8040001A809F0B5FF300905D329208DF8040059
:20A0D00001A809F0ADFFF00908D300208DF805002D278DF8047001A809F0A2FF300A08D3FF
:20A0F00000208DF8050030278DF8047001A809F097FF6068D8F8041080B188476168002782
:20A110000091D8F8081067608847009804F10806306009F085FF30460BF03CFB0020BDE80B
:20A13000FE83C046700D0020B0160020C0150020A01B00202DE9FE4F07461046002F00916F
:20A150000CBF4FF0E80B4FF0000B002900F0AB80BBF1000F40F0A98060B17868401E786029
:20A17000F82101707868401E7860002606703889801C3881009C4FF000094FF0020ADFF877
:20A190003081CDF80490083C14F8080F00F00F010F2900F08580012820D004287AD1454DEF
:20A1B00095F83800002875D0296D60688847061C26D03889B7F84C103018801C81421FDBAB
:20A1D00078686D6D6168019B3A46801BA847B8B178683D89801B786076195AE00098019EC4
:20A1F000042309EB0001C91C11F8010FFF2841D021283DD13889B7F84C200B30824202DAEF
:20A210001A20BDE8FE8F7868B8F8D020401E7860121202707868401E786098F8D02002706E
:20A230007868401E7860019D057098F8D2007A68107098F8CE2078681201401E786042F048
:20A250000F02027098F8C0C098F8A1207868401E786042EA0C1202707868401E78602125DC
:20A2700005707868F61DB6B2401E7860052505705B1EB9D17868C6F30121401E786041F004
:20A29000880101707868401E7860067038893618B61C3E81BAF1010A09F108097FF474AF31
:20A2B0007868B86501E04FF0E80B5846BDE8FE8FA00E0020201500202DE9F04F5D4C054642
:20A2D00000208A46ADF12C0D80461746B4F952100A93DDF850B084F88901B4F950008BF87D
:20A2F0000080401A40F6F87101400829A8BF012080F29280B4F95000401CC0F30B030CF041
:20A3100077FF0646D4F87C01B384854207D194F88801410824BF00F0FE0084F888010A9876
:20A33000006800B940463062387B00F00F00022814BF4046B868BAF1000FF06175D00AF134
:20A350009C000EF0A3F9002865D128460BF084FD051C1AD1E36BC3B109F092FF236C0890F0
:20A370002BB1216CE26B304606F078F838B9236C5BB9E26B3046694606F070F828B10123DA
:20A3900084F88931E06B3060E66394F88991B9F1000F4AD10DB9E56B95B12A683046294606
:20A3B00006F05CF818B92D68002DF6D108E00223286884F889312246306092F889912E60EC
:20A3D000B9F1000F31D10A980179504604F082FB0146012926D094F88901002825D10129CA
:20A3F00023D0E16B09B10868D0B9387B00F00F02022A1AD1C01118D141B9206CA8B1216C6A
:20A410003046424606F02AF828B10EE03046424606F024F848B902208BF80000464604E029
:20A430000968E0E7042084F8890130460BB0BDE8F08FC046A00A00202DE9F04F504E7068BA
:20A45000ADF11C0D80474F4A934611784E4D04919BF80020B168012A0BD001248BF8004079
:20A4700088472878012805D020460021FCF734FE00E08847464C454FDFF81891E06807F11E
:20A49000B001814206D1494691F90000002818BF002761D170688047404B0590002003F11D
:20A4B0003801A7F8B2000F78002F07BF4FF48601021C39492022804639489A460378CDF873
:20A4D00008809B0904D20078000938BF012000D302208DF80C008DE8060036493148324B5B
:20A4F000006802AAFBF762FEB7680028A08030D4494691F900009AF801302C4A401C087055
:20A510002C49002B92F90000E16000F1010010700CBF40468020B4F84410254B4FF67F72B6
:20A530000A4010430143A4F84410B3F8BA00B3F8BE10A4F852000822A4F8501003F1D8017B
:20A5500004F1470318460DF09DFC0598B847012702E00598B847474670688047B16817B961
:20A57000049A8BF8002088472878012803D000200146FCF7B1FD384607B0BDE8F08FC046B8
:20A59000C0150020921B00209E1B0020D8120020181700209B1B002000004F8C20150020B1
:20A5B000C32E0020EC190020F11400009A1B0020A00E0020881300202DE9F04F8A4609AF15
:20A5D0004FF08051ADF11C0D90463D69059001F5D8700490D1F8B001D7F808B0416906936D
:20A5F00027208847524C4FF00309143CC4F884970126C4F87C67C4F880970220C4F8FC06AC
:20A61000F868C4F8080430460DF0F3FFD4F808040008F8D2D4F88C07800F28BFB14655D200
:20A63000681E41460C238DF800000DF1010011F8012B5B1E00F8012BF9D1022D19BF002087
:20A65000011C98F80C1000208DF80D108DF80E008DF80F000099C4F83C15019BC4F84035C5
:20A67000029AC4F84425039BC4F848353968BAF1020F4FEAC542A1EB0A08A2F5002106D366
:20A690004FEA4A52A2F580026FF315021143264A0A43C4F84C258246C4F85085BBF1000FF1
:20A6B000C4F854A5214DC4F858B511D02E6078682060C4F808B030460DF09BFFD4F88C07EF
:20A6D0008008F8D3D4F88C07000801D3CA4627E0C4F88497D4F88C0710F0030FFAD1D4F8E6
:20A6F000800720F00200C4F880073F7D47B1049F3868016A272088473868016927208847D6
:20A71000C4F87C670598C4F8806748B12E6006982060C4F80880C5F800642062C4F828805A
:20A73000504607B0BDE8F08FC801042000004842184002402DE9F04704466668A7680D46C0
:20A75000ADF1400D0EF05EF896F8DC10012903D10EF054F8002097E04FF0010A86F8DCA00D
:20A770000EF04CF82878307068687060287AF060786805F0D7F820460AF050F9E86865684B
:20A7900028B9A06890F8149090F8158003E090F8009090F80180B9F1FF0F15D0B8F1FF0F1F
:20A7B00012D03B4840EA09010D91FE230F9340EA08000DA90E9005F1980006F0B1F9C5F81E
:20A7D000A400D5F8A40070B9324800240460324D2C60786804F018FE0EF014F886F8DC4090
:20A7F0000EF00CF84FE049460D220CF0D5F9D5F8A40041460E220CF0CFF901A80021302288
:20A8100008230DF0D3FF0025387B069401AB234A0095B968099006F110000DF0C3FF01A8E5
:20A830002822082329460DF0B9FF38691C49059401AA2B46079006F12C000DF0ABFF01A8AA
:20A850002422082329460DF0B9FF8DF81CA006F16000514601AA0DF0ADFF307838B906F140
:20A870007C00294601AA0DF0A5FF0E4870603572C6F8BC500C4AC6F8C05006F1C8000421F2
:20A8900023460CF045FB204610B0BDE8F087C04600200084042800401004054205C8000083
:20A8B000793E010077850100B18201002DE9F04F894609AF4FF08051ADF1240D9246059077
:20A8D00038683D69079001F5D8700490D1F8B001D7F808B04169069327208847504C4FF084
:20A8F0000308143CC4F884870126C4F87C67C4F880870220C4F8FC06F868C4F8080430461F
:20A910000DF077FED4F808040008F8D2D4F88C07800F28BFB04653D2681E51460C238DF84A
:20A9300000000DF1010011F8012B5B1E00F8012BF9D1022D19BF0020011C9AF80C1000205A
:20A950008DF80D10019B8DF80E0000998DF80F00029AC4F83C15B9F1020FC4F84035039BB6
:20A97000C4F844254FEAC542C4F84835A2F5002106D34FEA4952A2F580026FF315021143DE
:20A99000254A079D0A43C4F84C258146C4F85055BBF1000FC4F85495204DC4F858B511D07B
:20A9B0002E6078682060C4F808B030460DF021FED4F88C078008F8D3D4F88C07000801D3A6
:20A9D000C14624E0C4F88487D4F88C0710F0030FFAD1D4F8800720F00200C4F880073F7DF5
:20A9F00047B1049F3868016A2720884738680169272088470598C4F8806740B12E6006980E
:20AA10002060C5F800642062079FA760A762484609B0BDE8F08FC046CC0104200000484261
:20AA3000184002402DE9FE4F524D286808B90DF00FFC554C04F13800DFF83C91DFF840A1E7
:20AA5000DFF8408107789FB94D46686880474B490F7847B95246A96817782FB983234246E4
:20AA7000137088476DE0A96802234246137075E0D4F8981009B104208847676D2A685FB1FA
:20AA9000D06D20B102210023B8472A68676D106E10B108210023B8473C4E306A3C4F016C47
:20AAB000F86888474D46834668688047029033480578002D48D150460078002844D1D4F87D
:20AAD000841000208847F42001A90AF043F99DF90400304D58451ADCAB79C3B9D9F80810BC
:20AAF00002988847A878042801D00DF0B1FB04214046AF790170D4F88410781CA87109B10C
:20AB1000032088470320688100F0FAFA27E083214046346A0170636CF8686A460021984724
:20AB3000B6F90600BDF90010884214BF002001200AF0E8F9D9F808100298884708352878A2
:20AB500038700CF0E3FD0AE0022140460170D9F8081002988847D4F88410042088470E4862
:20AB70000078012803D000200146FCF7B5FABDE8FE8FC046700D0020C0150020C22E00206E
:20AB9000C42E0020C62E00202015002018170020E0190020401A00209E1B00202DE9F8431E
:20ABB0004E4E84460120002430704D484F4D04704C48DFF83481047005F14E000088B1463E
:20ABD00014EA03074FF0020606EA020608BF002E13D120464FF0E04710401F4008BF0028DB
:20ABF00003D11D2006F05EFE54E0454695F90000401E28700DF02EF94CE0424692F900300C
:20AC10003C4E5B1E137043F20842824207D06F8E931C834203D0BA4218BFBB4217D1304612
:20AC300008300068826C60469047008843F6030181420BD0204601F0F9FF98F9000000288E
:20AC50003FD098F90000002838DD42E06F8EB5F86A1043F60400884205D0B84203D0B5F86B
:20AC70004E20904203D12248007803281AD1B1F5505F05D0080B0BD31D2006F013FE07E072
:20AC90001D480168304601F5C071016004F0A0FA0DF0BCF898F9000098B198F90000002806
:20ACB0000CDD16E0022811D0204601F0BFFF98F9000030B198F9000000280ADC0DF0C8FAB5
:20ACD00007E020460146FCF707FA02E0204606F0E9FD89F80040BDE8F883C0469E1B0020F8
:20ACF000941B0020931B00209A1B0020D8120020421A0020301700200C0100212DE9F84F5A
:20AD1000994692468B4606460DF07CFD4E4C0090B4F95210B4F950000AAF401A40F6F871F1
:20AD3000014008297CDAB4F95000401C6FF31F30A4F85000B4F950800CF05AFA054606F136
:20AD500078000CF0D3FCC5F808B085F826A0C5F80490A5F824803D48EE6097E80C002021B7
:20AD700000271940104005F1100383E8030004F13C0085F827700368002B43D129460BF023
:20AD9000C5FA002844D0A6F8C08095F8270040F0800085F8270086F8C270E07920B1207850
:20ADB00010B1E7710120207200980DF027FD206C002845D12078F0B96079012840D00DF0E4
:20ADD00021FD0646A07988B9A86808F03DFB40B930460DF013FD04F1EC0004210DF0A6F842
:20ADF0002EE004F1C8000DF001FD02E0184901200870304622E001200CF09CFD19200DF03D
:20AE10007FFA1DE004F13C0029460BF07FFA50B9B4F9500000F6FF706FF31F30A4F8500090
:20AE30006FF0010809E0A6F8C08095F8270040F0800085F8270086F8C27000980DF0DEFCAC
:20AE50004046BDE8F88FC046A00A0020FDEFFF9FBD2E00202DE9F0434D4CDFF8388194F8CD
:20AE70003F600027ADF1140D002E57D198F89660002E53D0C768007A454600F00701C0F331
:20AE9000021900E0BF1C0E46701EC1B24EB17A783878B5F8BE6000EB0220B042F2D1022720
:20AEB00010E005F19406443600E008374846411E5FFA81F9A0B3304639460CF045FE0028FA
:20AED000F3D0032794F83F0040F0040084F83F0002A80CF0A9F801200CF098FB04F134019A
:20AEF000872000F063F804F13C01852000F05EF804F13D01862000F059F804F13E0188203D
:20AF100000F054F80120009004F134060196B5F8BA30394602AA0520FCF7E0FD002F33D184
:20AF300098F8A1100F292FD0404690F8C0208A422AD090F8BD0038BB1748007820BB17488C
:20AF50000078012803D001200021FCF7C5F8144C606880472146134C94F83B20022A11D1D1
:20AF700094F83820FF2A0DD00F4A176857B9576A47B98968884704F1200009F08DFC06F0E1
:20AF900021FE01E08968884705B0BDE8F083C0466C2C0020A00E0020BE1600209E1B0020BB
:20AFB000C015002038190020700D00202DE9F0410C4601467138022840F29780133825D042
:20AFD0004D4F4C387BD0401E62D0401E4AD0401E38D04A4D401E2AD0401E1AD008460DF006
:20AFF000F3F806460B2E11D0414D6868804741498046B000425CBF1840184278394620465F
:20B010000CF040FFA968404688470DE0F420BDE8F0812278022A68DA2946601C483101EB10
:20B03000820104220CF02EFF0020BDE8F0812278032A5ADAD3002946201D03EB0213182241
:20B05000C918EFE72678022E4FDA2C25601C05FB0671102239310CF015FF05FB0670C06CA0
:20B070006061E1E7207802283FDA2C2101FB0070667890F83800B04237DD2378627839460B
:20B0900002EB430201EB42010222A231A01CC9E72078022829DA2C2101FB0070667890F8F8
:20B0B0003000B04221DD20786278394600EB4000121802EB4202891803229031E6E72078FD
:20B0D000022812DA2C2101FB0070667890F82800B0420ADD6278207839468018420002EB72
:20B0F000C00289180A227C31D0E7E820BDE8F081C0150020E49C01003C270020E827002007
:20B110002DE9FC414948484C494F4A490278A37865893878042B71D101F13C06337803F006
:20B13000F003337000268E630DB901256581884641490832554300FB05F291F838500092C1
:20B15000002D50D00D46AA6F002A4CD0EB6F002B49D004F108016846904784463B4B2179D5
:20B17000DFF8E0E060791A68BCF1650F31D0BCF1000F28D1107D052811D13048017871B93F
:20B19000186890F82C00042809D119686D6D906D096B3346A847002808BF1A2016D02C4DA9
:20B1B0006868804726490E68002E08BFA96807D0A96804F10C02964213D03668002EFAD1C0
:20B1D000884738780FE0704606706046FEF71CFE22E082F8690082F86A107046E96F0670B3
:20B1F0001C20884718E01849009E04F10C076161B6FBF0F138460CF061FC0DE091F83C3028
:20B21000083280005543884603F0F0036843886343F0030381F83C3098F8740000F0F00080
:20B2300088F87400BDE8FC81401A0020E1190020201B0020D8120020201500205D0F00200E
:20B250007C1B0020C62E002035AA0000700D0020C0150020F8B5071C00F0A180B86840F66B
:20B27000030120264A1C02E04068761EF6B260B15EB10388994218BF9A42F5D1F9681CC804
:20B2900028311CC149C881E849007868BA690026BE6168B3F96848680078022818BF42F086
:20B2B000020297F82700002300F00700401E09D0401E04D0801E08D14FF0805304E04FF095
:20B2D000804301E04FF00053324697F82700000908D397F8270010F0070F03D04FF0807048
:20B2F00032430343B7F92440084621467C68A0470DF088FA2A4C0546B4F95200401C6FF3F2
:20B310001F30A4F8520004F14C00016881F827600CF02FFE28460DF071FAB4F95000B4F98D
:20B33000521088423BD1F86890F8C20000280CBF0520072004F0AEFD04F5AA742568F86839
:20B35000854208BF656890F8C240002C0CBF0468341C80F8C2604DB195F8C23023B92868C2
:20B37000A04228BF041C01E085F8C260A4B10D480068B4F1FF3F12D0B4FBF0F101298CBF78
:20B39000B4FBF0F10121F86878300DF0F3F9F86878300DF02BFAF8BD012009F0A7FEF8BDA7
:20B3B000A00A002010A501002DE9FE4F514C814604F13C0A50460DF053F990468B46074628
:20B3D00008F0010000900DF01DFA0325BBF1FF3F019015D1266C2EB1206CC068814508BF85
:20B3F000206C0BD00DF00EFADAF8006074E0F168894570D10DF002FA301C71D0B0F924B0E0
:20B4100058460BF021FC00286AD0216C814248D0B84217D104F1C8000CF068F9E06B0068ED
:20B43000E06397F82700394640F0040087F827000AF110000AF06AFF5FEA980022D3E76B14
:20B4500001221BE017B9832D20D01CE03968884225D104F1C8000CF049F93968086838604D
:20B4700091F8270040F0040081F827000AF110000AF04CFF5FEA980004D300224846394601
:20B4900007F012FE832501980DF0B8F96079012829D004F1EC0002210CF048FD23E03F68BC
:20B4B000D0E7009F90F82720012505FA07F13E1C41EA020180F8271014BF0C480C480BF08D
:20B4D00013FD5FEA980004D3E16B48462A4607F0EBFD832504E03668002E88D10DF08EF936
:20B4F00001980DF08BF92846BDE8FE8F0100020401000104A00A00202DE9FF410646080BF6
:20B51000C0F092804A49C8680025012788460D70C3694F722BB1016AC90802D304212A468F
:20B530009847444908F170002A460DF086F842480CF054FFD8F80C004168414C886808B99F
:20B55000C86820B1A4F11C00C5613C490160384608F03AFD25603B4844F81C0CB1684D801E
:20B57000B068028840F60200904208D0B2F5C15F05D00B8B4FF60F421A400A8304E00B8A0F
:20B590004FF60F421A400A8200F1080C7774ACF10702531C00E039464F6837B13888844593
:20B5B00003D0824218BF8342F5D12F464F60487B00F0F00040F00100487308F13C000DF09D
:20B5D0004FF88068008882421BD0834219D0308DC8B196F83400758596F83530F76200F019
:20B5F000F00086F8340003F0F00040F0010086F8350006F128024A60487B00F0F0004873A9
:20B6100001E0C8F86050B068694602F08BFF68460CF036FEB06802F043FE20680028FCD0E1
:20B630002560B06844F81C0C0090BDE8FF81C046A00A0020097A01006939000051000706F0
:20B650001C10044001010E042DE9F04106467478ADF1180D002C40F089804948B6F89610CA
:20B670000088884218BFE82406F18C0101A80D460CF078FA01A80BF0C3FC424B40B996F820
:20B69000990040B1A3F13800007820B9E8246DE0002086F89900002C68D196F899000028AF
:20B6B0000CBF01200520042737752946F0820DF10E000CF057FA706896F89840401E7060EC
:20B6D000411E7160B6F896800470327D71680024481C3062501E0870308934651A78B4656D
:20B6F000801C3081A2B386F86B70296806F16C0001606B6843602A8902810CF033FB06F11D
:20B710006C0228BB06F18C0110460CF093FF1E4D286810F47F0F0CD086F82C70286806F156
:20B730002C01012200F47F0030633046FEF702FD286810F0FF0F0BD02A2086F83C0028682C
:20B7500006F13C0100F0FF003064304603F0F4FA0094304603210DF10E024346F8F716FB06
:20B77000041C02D1304603F011FC2CB174701A203070304608F054FC06B0BDE8F081C04625
:20B790005A0F002058150020A0A001002DE9F04706464FF00108ADF1600D0922B07D8DF879
:20B7B0004C8006F117018DF84D000DF14E000CF069FB464D68688047814616A98120FFF7D9
:20B7D000F5FB707D002854D09DF85800022817DA042000238DF80300347D8DF802809DF80C
:20B7F00058708DF8013069468DF80040781C8DF85800D220FCF752FD812016A9FCF74EFD04
:20B8100000274FF0FF0A3C46307D8DF8217008A980F001008DF82000D120FFF7C7FBC0B97B
:20B830009DF82200FF2814D08DF800006946D420FFF7BCFB20B1A96848468847192042E0C7
:20B85000307D69460DEB80000461D420FCF726FD01E08DF822A08DF82440307D8DF82340EF
:20B8700008A98DF82000D120FCF718FD7F1C032FCADB307D00279DF84D208DF840000DF15E
:20B890004E018DF841700DF142000CF0FBFA8DF84B80D02010A9FCF701FD071C0FD1307D48
:20B8B000314610228DF828000DF129000CF0EAFA30690AA90F90D320FCF7F0FC0746A96800
:20B8D00048468847F8B218B0BDE8F087C01500202DE9F04FFF25ADF1140D8DF800504FF626
:20B8F000FF79ADF80290ADF804900AF043FDDFF81CB104900BF1020000880027001F84B2DC
:20B91000082C64DB4E46B046C246201F02A9082280B20AF0ADFEBDF80800814508D1BDF816
:20B930000A10894506D1BDF80C20924502D107E0BDF80A1051EA000317D1BDF80C30A3B984
:20B95000BDF80E1008466FF30E0060B908460830844206DA0CF07CFC04980CF03FF800209E
:20B970004FE008462EE0241F2EE0C20BD30327D1BDF80C20854203D18E4208BF90451FD069
:20B99000C5B28DF800500E46ADF802609046ADF804809DE80600384607F088FD80B9BDF87E
:20B9B0000E20A01A07F18851001F083280B292B20AF05EFEBDF80E003F180837BFB201E0EE
:20B9D000BDF80E00241A083CA4B2082C9DDA09F081FE3FB10C484FF088513A460CF088FD3C
:20B9F0000CF0A6FB04980BF0F9FF5A46507800281CBF0020011C03D1C7F58054391DA0B257
:20BA1000518005B0BDE8F08F04E00100141700202DE9F8430020444C8DF800000CF095FD28
:20BA30002279484E424DDFF81091012191404FF6FF725218024096F83800628120B3326F4C
:20BA500012B342F21A0069469047384867790378A3B19FB99DF8003083B1D6F8940068B142
:20BA700080474946491C2A78097830B1678908314A43B0FBF2F0C019608167799DF8001075
:20BA9000608907FB01006081A078002847D1294F386AC06B80474E46804664892978707895
:20BAB0003B6A08304443D86B8F0080476968234D2A787578224E3C23401AB0FBF7F103FAF0
:20BAD00002F0B1FBF0F205F108034243891AB1FBF3F25A43891A05F10803691A641896F84E
:20BAF000581096F83C5098B2083401F0F00107FB048341F0020107FB0032736596F8744041
:20BB100086F8581005F0F000B26340F0020086F83C0004F0F00086F87400BDE8F883FFF75D
:20BB3000EFFABDE8F883C046401A0020BE2E0020201B002018170020E0190020600F00200E
:20BB5000D8120020201500202DE9F0434A4D95F8E700ADF12C0D00287AD13F4F387B012472
:20BB70000021242285F8E7407E6885F8E6000823C5F8106101A80CF005FE002605F10C0038
:20BB9000069601ABADF814603449079632460CF0F5FD334905F1300001AB32460CF0EEFD07
:20BBB000304905F1540001AB32460CF0E7FDB96820468847DFF8BC802B4808F104037A7BDD
:20BBD00000781868C0F3815922B1B9F1030F04D185F8E140B9F1030F1ED0B9F1020F1BD07E
:20BBF000B9F1010F2DD14FF08059D9F8A4011F4F456831464FF040521C230320009038461C
:20BC1000A847D9F8A40131464FF400720923456800943846A84714E002200AF0B9FDB9F139
:20BC3000030F0CBF4FF47A7142F21071104800685435B1FBF0F128460CF09CFD28460CF0F1
:20BC5000D5FD40460068C00802D230460AF0A0FD0BB00020BDE8F08358A40100EB90000000
:20BC7000DD1C010095160100BF2E002000A00C4010A50100B03F0050B80F00202DE9F84FDC
:20BC9000064630798028D4BF0020E82071790027092901DB0A2900DDE820B17909B10429F4
:20BCB00003DB802975DB862973DA002871D1DFF8F88098F8A1000F286BD0B8F8BA104FF686
:20BCD000FF70884265D0B8F8B410884261D0F079314C01280BD040B1FF285AD194F83B0083
:20BCF000002856D101252F4602E0012500E00225DFF8A8A00AF12000834608F0CDFD0AF17B
:20BD1000100008F0C9FD04F1200008F0C5FDDFF89C9009F1040000688047214B84F83B50D3
:20BD30000246FF21002060631D6884F83810002D0CBF0121011C012F84F83D10554684F818
:20BD50003C7008BF032085F840004846816810468847B11DE820FBF7C3FA711DE720FBF7D8
:20BD7000BFFA311DE120FBF7BBFA94F83D00012802D120200CF0ACFA0A4898F8A1104FF487
:20BD90007077A86207FA01F000F2636158460BF095FEBDE8F88FC04638190020A02D00203E
:20BDB000700D002059320100A00E0020C01500202DE9F84F05464448DFF8109183462E18CC
:20BDD000093699F8380034788846B0B1D9F8501099B10BEB8507786B00F0FF00884782460A
:20BDF000D9F85010786B00F47F008847504480B218B131784018001DC4B23548007801289C
:20BE10000CD198F808704FB1324898F80930C1190E79C05C0019401DC4B200E000260D2D41
:20BE300009D106EB0408B8F1F80FD8BF2A4F1CDD0CF00EFA05E030198046801C0BF068FA71
:20BE5000074697B902200BF063FA011C0AD00BEB050090F825001A270870204E4F7030788E
:20BE700007F036FE0020BDE8F88F08F10202384600210CF005FC07F10C00002174220CF0EB
:20BE9000FFFB07F13C00FF2110220CF0F9FB07F12C000F2110220CF0F3FBE0197860022DB2
:20BEB0003E810BDB0B2D09DA7868401E78606D1E05703889641EE4B2401C3881A7F84C4083
:20BED0003846BDE8F88FC0465CA00100201500206C0F002078A40100A40D0020B0160020E1
:20BEF00070B5ADF1380DFFF72FFE3E4908682822082340F00200086001A800210CF04EFCF1
:20BF1000394D3A4E3A49A878002301AA079006F1EC000CF03FFC00213022082301A80CF09E
:20BF300045FC287800241921ADF81C40314A099001AB009406F170000CF034FC2822082355
:20BF500001A821460CF02AFCE8782B4901AA2346079006F590700CF01DFC01A821463022AE
:20BF700008230CF023FC01206A78ADF81C001A2101AB099206F18C00204A00940CF012FC9A
:20BF90001F49224606F1C80013460CF0F7FB1D480CF024FA1C4A2346042106F128000AF02F
:20BFB000B7FF25464FF6FF70A6F8C400052386F8683006F1580181E830004FF4FA70C6F8A8
:20BFD0005C01C6F860012B4686F8C73033717371B371F37133727372B372F3720B4A1370F3
:20BFF0000EB070BD0020094004A50100A00A0020F57E0100610C010065090100394301009B
:20C010006168010049C10000794A0100BC2E00202DE9FE4F0BF07AFA434C04F10C02029078
:20C03000116820614FF40050491C1160694608F0CFFCDFF8FCA0DFF8FC9094F8330000285E
:20C050005FD0A66B94F8310000254FF0FF0BA0462F4654E0B07F800821D3F07F09F002F8C9
:20C070000146082268460BF065F9C0B1716802980CF0ECFA2D49814211D8F07FB7770AF0B9
:20C09000DFFA86F81FB0DAF80000804794F8323013B15B1E84F83230D9F80810884798F880
:20C0B00030006D1C2036ADB236E0F078800822D3307908F0D7FF0146082268460BF03AF943
:20C0D000C8B13088010402980CF0C0FA1749814211D83079F7700AF0B3FA86F804B0DAF803
:20C0F0000000804794F8333013B15B1E84F83330D9F80810884798F831006D1CADB2A84213
:20C11000D3DC94F8320048B1A046666B98F8300000254FF0FF0B2F46A8429BDC04F11400E5
:20C1300008F084F8BDE8FE8FCC10002000A493D6C4150020C0150020F8B5424C0D46A80814
:20C150005DD2E8087CD301260420E6720AF020FB0BF04EFF04F1580282E8030004F13C0074
:20C170000CF07EFA0746E06877B1FD6850B1854208D0EB6933B1286AC00803D3284604217E
:20C19000002298472846E06041682F4A09781160416812680978914207D087692FB16FF04F
:20C1B000FF0100224FF00073B84702200AF0F0FA112003F0B7FB6671E168087C10B12079C2
:20C1D000012803D00E2003F0ADFBE16849681F488F680FB9CF681FB10021C1611C4F07604E
:20C1F0001C4A40F2FF711160002787611A4941611A480CF0F3F819200CF0B8FAF8BD04F1C8
:20C210004C0630460CF02CFAFFF724F830460CF027FA25F0020504F13C0158B9E80803D25B
:20C2300008460CF01DFA58B104F1C8000BF05EFA042101E045F0020104F1EC000BF076FEE6
:20C25000F8BDC046A00A0020D02108400010044051000706000004600A000040A997000070
:20C270002DE9F04F0C4692468046994600213822ADF13C0D684605F09FFF20686D46286024
:20C290006068686020892881207A032804D0022003268DF80C0002E003268DF80C60374CB8
:20C2B000207818B104F138000BF0B2FF208FADF80A0060781F28B4BF411C00210027B8F1F6
:20C2D000050F617040F080000BD0B8F1040F05D0B8F1020F08BF40F0600004E040F0200008
:20C2F00001E040F040008DF80D00ADF828A04FF0010BCDF8249022498DF80EB00A680BA847
:20C310000260496841608DF8356005238DF83660B8F1050F8DF8343012D0B4F86200B8F1BD
:20C33000040F08D0B8F1020F0FD1B4F86800401CA4F8680009E0401C80B2A4F8620004E09B
:20C35000B4F85C00401CA4F85C000E4918206A4612F03EFFC0B258B1B8F1050F09D1206B56
:20C370000AF046FAB4F85C00401CA4F85C0000E05F4638460FB0BDE8F08FC046B813002040
:20C39000E19F0100096400002DE9F041414C0746206800287BD0DFF80081002F18BFE92F0D
:20C3B00017D10BF083F84546297801EB81016918C1F8020095F8B560287800EB800029184B
:20C3D0004E702878401C2870C0B20A28A4BF00202870324D68681C2F32D0314E4FB1F079B8
:20C3F000032806D1E12F04D0002088F8B200072000E0052008F08AFC2468F07903280ED04D
:20C410006CB1002084F86900E18A2648C90938BF2938007884F86A003846FDF7F5FC98F896
:20C430005700012833D168688047044606F0D0FCA96820468847002088F85700BDE8F08172
:20C4500080470646A96894F82F0002281ADA216804F124000BF00AF994F82F00A968401C07
:20C4700084F82F00304688472068007D252819BF012088F85600012088F855000020206005
:20C49000BDE8F08130468847F120FDF7BDFCBDE8F081C046700D0020A82A0020C0150020D3
:20C4B000C4170020820F00204549B0B5044601F13800007800287FD094F88B00002871D1E9
:20C4D0003520207504F18D01112204F16C000BF0D9FC04F13C00FF2110220CF0D1F804F13E
:20C4F0002C000F2110220CF0CBF894F88C0004F13C0500283ED0401E29D0401E14D0401E64
:20C5100058D12A20287002272764042305F8103C4FF410222263032184F86B10204607F06A
:20C5300055F9071C3BD137E02A200A272870042327644FF44C1205F8103C0221226320469A
:20C5500084F86B1007F042F9071C28D124E02A2002272870042327644FF4102205F8103C07
:20C5700001212263204684F86B1007F02FF9071C15D111E02A2002272870042327644FF48E
:20C59000502205F8103C00212263204684F86B1007F01CF9071C02D1204602F0F7FC381C2C
:20C5B0000BD1B0BD01280AD1886C8047002808BF002002D0192000E018200BF087FDB0BD45
:20C5D000201500202DE9FC410746BE6833687D68986B20F4FA609863AC6B44B13168886BAC
:20C5F00040F4FA6088634FF0FF30BDE8FC81AA6329630024EC776C630CE09DF80000296B1E
:20C6100008706B6B286BAA6B401C2863581C6863501EA863A86B90B93168886B40F4FA60FF
:20C6300088636A6B6878296B0128A1EB0201296303D1EB68384698476A6B144646E005F1A3
:20C650004000694609F006F90028D6D50CF0DAF8204F8046387820B902200AF099F80120B6
:20C67000387040460CF0CAF81B49086840F4007008603168886B40F4FA6088636878D8B968
:20C69000696805F1EC000CF09DF890B9AC630CF0B9F80646387818B1022009F01DFE3C709A
:20C6B00030460CF0ABF81027696B286BEF77401A2863686BBDE8FC8195F82D0030B1686B09
:20C6D00020B1AC6305F19C000CF04CF82046BDE8FC81C046BA2E0020301000402DE9F04F2D
:20C6F00009AF9A4616460D46ADF1440D3C89D7F80480109000203F888DF83C00BC4201DABB
:20C71000C24501D30BF0A4FD002E69D0364810F80690042EA4EB09044FF00000A4B2B8BF35
:20C7300001205FEA000B0EBF3F1BA04400242F49082307A8A7EB0907BFB211F801295B1E34
:20C7500000F8012BF9D1290E00F8011B2B0C00F8013B2A0A00F8012B9DF83C1000F8015B98
:20C77000234D06702868109A4369686898470646B6F1FF3F24D001208DF801009DF83C6031
:20C790008DF802600BAA04928DF800B08DF80390CDF80880CDF80CA002218DF81410ADF8DB
:20C7B000164007ABADF818702E686868326A01936946904706462868826968680FA99047F2
:20C7D000002E18BFE4200CD1B9F1000F08D0444448460BA911F8012B401E04F8012BF9D183
:20C7F000002011B0BDE8F08F7CA401007F0F0020A02E0020B0B53F494468096880684968C4
:20C81000006888473E4D012205F118031A6050B1217AFF2907D0FF214009217264D20420A7
:20C8300043F8180C45E0207A00285DD0324B3349401E1AD0401E02D0FD3855D051E01D68F4
:20C85000D4F8B4000570D4F8B870D4F8B400401CC4F8B400781EC4F8B800D4F8B87027B3BB
:20C87000012F3BD9092202201BE0D4F8B000401EC4F8B000D4F8B070EFB9D4F8B870A7B1F6
:20C890000220D4F8A8202072127C2D1F012F4FEA420242F001022A609CBF0321696001D9D8
:20C8B0000B220A600BF0A5FEB0BD0020207204220A600220F6E7D4F8AC0000781860D4F851
:20C8D000AC00022F00F10100C4F8AC00F0D2D4F8B870002FECD100202072052243F8042C2B
:20C8F000E7E7FF202072B0BD04F12C000BF03AFFB0BDC046AC0100100828004004280040DB
:20C910000428004070B5424C0646683C607800287DD0B4F95200B4F95010884213D030467C
:20C9300009F09AFA38B9216C21B1216CC9688E4208BF206C38B1B0F9241002224FF0E043DD
:20C95000304604F043FD0BF05DFFA178002943D0491EC9B20029A1703ED10BF04FFF0025D8
:20C9700065702078E66058B1012008F0BFFB022008F0BCFB06F140004FF0FF310BF022FF85
:20C9900006F140000BF0EAFE06F178000BF0E2FE06F19C000BF0DEFE04F1EC000BF0D6FE09
:20C9B00004F170000BF0CEFE04F590700BF0CEFE04F18C000BF0C6FE04F1C8000BF0CAFEBB
:20C9D000E56004F128000AF0F1FD307C012817D10E2002F019FD13E00BF010FFE0688642FD
:20C9F00004BF0020E06006F140000BF0B7FE06F178000BF0AFFE06F19C000BF0ABFE0025AA
:20CA100004F5AA742068B04214BF6560256070BD080B00202DE9F043404C054660781F469B
:20CA300090460E46ADF1440D012803D0FFF758FA01206070AEB13648337801684FF001095E
:20CA500009FA03F001420CD0B8F1000F6E6008D0C5F808800BF0D6FEA178022903DB0BF022
:20CA7000CDFE002051E004EB8102491CC2F85451C9B2A1700BF0C2FE4C461FB909A80BF0F7
:20CA9000CBFA09AF386828607868E860387C2874B86868617869E861B8696C742862788AC9
:20CAB0006882F86800B1A8610021A02205F1280005F082FB68460021242208230BF07EFE38
:20CAD0008DF8184005F1400000216A460BF072FE68460021242208230BF054FE0D49069579
:20CAF00005F1780000226B460BF048FE68460021242208230BF046FE0749069505F19C00A8
:20CB100000226B460BF03AFE284611B0BDE8F083D4210840D17901001B860100A00A0020C4
:20CB30002DE9F8430BF0BEF83E4E054615F00A0F4ED0376C002F4BD03869B9693A4A344622
:20CB50004FF0000840F00A0028400843B8613B69C4F84080A2F1100000F108021168994365
:20CB700007F11003116093E806000168121C91430160394604F14C00814609F0C7FB022177
:20CB900004F1EC000BF0D2F9A06C08B3F8684068007802281CD197F8270040080CD297F815
:20CBB000270080083CBFA06C20640FD3A06C2730017841F0020104E0A06C2730017841F048
:20CBD00001010170A16C484609F0A0FBC4F84880326C05F0020005F00807074316D102F162
:20CBF000100003C8002301EA03072840002F08BF00280BD010699769054072644FF4804139
:20CC100006F1EC003D4395610BF090F9306C30B906F13C000BF024FD08B103F0DBFABDE82D
:20CC3000F883C046A00A00201C1004402DE9F0473E4C8246A07830F0010708D0042806D070
:20CC5000032804D0052802D00BF002FBA078384E677904210528DFF8CC90DFF8CC80317007
:20CC700007F10101CDB265711DD1022D55DC48460768BAF1010F50D07868398904F01EFF7C
:20CC900078680088000905D34146087810B108F0A5FF657928460BF0FBFC8320307009F05D
:20CCB00097FEBDE8F087234FE73F97F8B810A94233DB032831D007F023FFA078042809D168
:20CCD0004146383991F8380020B1D1F8841009B102208847207997F8C510421C9142C4BF01
:20CCF000401CC1B22171484605686868298904F0E5FE68680088000904D34146087808B177
:20CD100008F06CFFFEF784FEA078042808D08320307008F01BF9BDE8F087E12004F0C2FDEE
:20CD3000BDE8F087700D002058150020401A0020C62E0020870F00202DE9F8438146D9F870
:20CD500008703868066CD9F8045046646A6CAB6CA86B16F4F06F0146A2EB03082AD1F0092E
:20CD700011D270095DD301B395F83C40641EA14298BF0C1C4846214609F06AF9A86B001BF7
:20CD9000A8630DD04DE081B1484609F061F995F82D10A86311B9002843D101E00020A86374
:20CDB00005F19C000BF0DEFC3BE04846414609F0AFFD36E0F20A19D24FF00008444602E077
:20CDD000A86B401EA86340B34846012109F040F93868446814F00F04C0F80480F0D0286B00
:20CDF000401E2863686B401E686316E0386844680022202904F00F044260CCBF20270F1CEB
:20CE10004846394609F024F9C7F12007B845C8BFB8464846414609F07BFDEC77484606F011
:20CE3000DBF8B0090BD3A96A49B10F46484609F07FF9A86218B94846391D07F055FDBDE86A
:20CE5000F88370472DE9F04105463E4804780F46002DADF1280D42D03B48466A002F3ED025
:20CE70008046D6B17069C0B10123ADF8223006208DF8200029460C2200236846ADF82430BE
:20CE900003F01AFD03A839460E2203F015FD766908A803C81A226B46B047787B012668B9A0
:20CEB000002C14BF0FA013A06988102207F00AFF397B13A00A2207F005FF08E0002C14BF69
:20CED00012A017A00BF052F919A00BF04FF988F802600020314605F047FF88F803600AB046
:20CEF000BDE8F0815265737461727465643A20307800C046537461727465643A203078007D
:20CF10004368616E6E656C3A2000C0464465766963652052657374617274656400C046C004
:20CF3000446576696365205374617274656400C04672657175656E637920486F7070696E9A
:20CF50006700C046B8130020D411002070B53F4C0646A07EADF1200DF0B994F85C00822844
:20CF70001AD0394B40F2016046F25C05ADF8080034491868ADF80A50426A086802A99047C0
:20CF9000812814BF6FF07F009DF90C000AF0D5F894F85C10226B505494F85C00822814BF30
:20CFB000401C002004F1180584F85C0094F85C0005EBE00292F82C00411082F82C1040083C
:20CFD00007D294F85C00401C84F85C00C0B28128ECDB94F85C0081282CDA05F14401E12097
:20CFF000FAF77EF902204FF6FF738DF81800A17EADF8103031F0020018D0012919BF07200B
:20D0100083210820802100224935009204AA0195FAF764FDDB2807D0E52805D0F32803D021
:20D03000DF2818BFE8280AD1607603E0304605F0B1F904E02A203070304606F0F1FF08B067
:20D0500070BDC046EC19002038170020E42C00202DE9F04707467D68D7F8089090460E46B9
:20D070000BF0D0FB8246A86A002864D105F584700AF03CFB0024EC772E6250466C620BF00E
:20D09000BDFB0BF0BFFB2F4E3378824623B9022009F07EFB0120307050460BF0AFFB2A4944
:20D0B000086840F4807008603846414609F040F8A862C0B93846414607F016FCA878D0B9F4
:20D0D000A96805F1D0000BF07DFBE8B9AC621020E8774946284605F0D5F90BF093FB8246A7
:20D0F000307840B323E0D9F80010886B40F020008863A87810B12046BDE8F087A96805F109
:20D11000D0000BF05FFB10B1686ABDE8F0873846414607F0E9FB1020AC624946E8772846B1
:20D1300005F0B0F90BF06EFB8246307818B1022009F0D2F8347050460BF060FB4FF0FF30C1
:20D15000BDE8F087BB2E0020301000402DE9FC4191EA03084CBF4FF000484FF000084FEA2F
:20D17000C32545EA52554FEAC2264FEA43077F0D11BF45F0004500210020BDE8FC815FF4B1
:20D19000E06E1EF1FF0E774555D04FEAC12343EA50534FEAC0224FEA4104640D11BF43F03A
:20D1B000004300210020BDE8FC81744543D0E419A3FB0501A3FB06E7A2FB06631EEB030EA1
:20D1D00057F1000751F10001A2FB05631EEB060E57F1000751F10001FF1851F10001C019C6
:20D1F00051F100014CBF4FF4806E4FF4007E10EB0E0051F1000148BF641C01D4400049416D
:20D210005FF44077FF37E41BDEBF00210020BDE8FC8117F58067BC420DD24FEAD02040EA9C
:20D2300041504FEA41014FEA113141EA045141EA0801BDE8FC810020FF21C900C91D090584
:20D2500051EA0801BDE8FC8181F000412DE9FC414FEA01244FEA41052D0E04D1002C18BF63
:20D270000020BDE8FC8144F00044FF2D5ED04FEA9404002948BF64424FEA00224FEA40030C
:20D290001B0E05D1002A14BF0020081CBDE8FC8142F00042FF2B4AD04FEA9202002848BF68
:20D2B00052425E1B41BF171C221C3C1C764248BF2B1C192E47BF44FA06F73A444FF0000835
:20D2D00003E0C6F11C0704FA07F8002A04BF0020BDE8FC8146BF524201270027A3F10103D5
:20D2F0005200FBD512F080040DD002F0200548EA0508803228BF5B1C02F0400458EA0408AF
:20D3100008BF22F480729B1CDCBF0020BDE8FC81FF2B0ED222F0FF024FEA42024FEA522055
:20D3300040EAC35040EAC770BDE8FC8108464FEAD0774FEAC777FF204FEAC0503843BDE850
:20D35000FC8170472DE9F043DFF8E0808946054617464FF0FF31ADF13C0D40460BF032FA8F
:20D37000334C04EBC504666825680BF04BFA2168096800290BD42968002905DCB9F1000F75
:20D3900009D04FF0FF3108E0B9F1000F03D00BF035FA002442E02968491C29600BF02EFAAF
:20D3B000286802283ADA1FB90DA80BF0D8F80DAF38686860B76800213022082301A80BF0B2
:20D3D000F5F94FF00009069401AB307B194A09903946CDF8009005F12C000BF0E3F901A8A4
:20D3F0002422082349460BF0E9F9012705F1640001AA8DF81C7049460BF0DCF905F1480065
:20D4100001AA39460BF0D6F9706802F08BFA0A4A05F118002346042109F07AFD40460BF0D8
:20D43000E9F920460FB0BDE8F083C046302E0020D8A4010071710100A78501002DE9F04165
:20D4500006AF3D793E68984604460B1CADF1180D074611D0012B15D130797379641C38709C
:20D47000B17904F8013B337A04F8011BB17A04F8013B7389181201E03178707804F8011B62
:20D4900004F8010B8AB9002D0CBF42F20C0042F20D00694607F09CFA9DF80000BDF8003002
:20D4B00004F8010B181204F8010BB8F1010F34D0B8F1020F39D1002D0CBF42F2020042F23F
:20D4D00003000DF1020107F083FA7589CDB1681E01468B100DF1020201EB5371C910CBB2D8
:20D4F000811000EB517121F00701401AC0B20121401C01FA00F0D15CFF3080F0FF0008437A
:20D51000D054E81D0DF10201C210204603F0D4F97089C01D04EBE00407E0002D14BF022126
:20D530000121204602F00CFC0419E41B06B0A0B2BDE8F0812DE9F04390460A68D8F800407E
:20D550001678814600271D463846ADF1140D531C242E0B6053D112F8016F5B1C4C2E0B6079
:20D570000ED1AA68E41C24F00304241D54F8040C494606F01FFC2968EF600127091A29609E
:20D59000462E1AD1E41C24F00304241D54F8040CE41C029024F00304241D54F8040C0027F3
:20D5B00049460390AA68ADF8047001A803F0E6F82968EF600127091A2960532E1FD1E41C6F
:20D5D00024F00304241D54F8040CE861C8F80040288B0090A968EA69D9F800004346F7F74B
:20D5F000A9FAD9F80040002714B10119C9F80010D8F800402968EF60091A01272960662E38
:20D610000AD12B8B23B9E41D24F00704083403E0E41C24F00304241D1FB9E9690E70012722
:20D63000EF60C8F8004005B0BDE8F0832C4870B50568B5F1FF3F08BF00250AF019F90128B3
:20D650004DD107F067FF142849DB26482649002601230660254A0B60254C136020680028E4
:20D67000FCD1264A131D2349186820F00300014321480068C0080CD2106810F0030F0AD00F
:20D6900041F003001860106800F003000328FAD101E041F001011A481960006820B11948E4
:20D6B00000682846F5F768FA174818490660184D0A686FF35B4245EA0200086015490868D3
:20D6D000C0F30130012806D10A681348104040F400320A60086020680028FCD170BDFEE772
:20D6F0001C130050840460425C600C40082204430C00684204000020B03F0050004003405C
:20D7100080012843000120438C210840482003400000390104000940FFFFFCFC2DE9F04F37
:20D7300009AF3C897D6816464FF0000A0246002EADF1440DA04610933C888DF83CA05CD093
:20D75000304810F80690042E03DAA8EB0900C8462D18F868A4EB080407AB0827A4B2C01D96
:20D7700010F801C97F1E03F801CBF9D1080E264F03F8010B080C03F8010B080A03F8010BD3
:20D79000386803F8011B9DF83C101E704369786898478346BBF1FF3F2AD0042E04DA032008
:20D7B0008DF80000022002E002208DF800008DF8140002959DF83C608DF8026001218DF83A
:20D7D000011038688DF8039007ABADF816800BADADF81840026A0193109E049569467868F8
:20D7F0000396904783463868826978680FA99047BBF1000F18BFE42000D1504611B0BDE883
:20D81000F08FC0467CA40100A02E0020394833492DE9F047012500240570DFF8C480DFF869
:20D83000C8900C702F4901F16A06378882460220104014EA030608BF00280FD120464FF0B6
:20D85000E04710401F4008BF002832D0424692F90000401E10700AF0FDFA2AE0424692F9F2
:20D870000000401E1070BFB94A8E43F2084320464646934204D191F84010090938BF281C28
:20D89000FFF7D4F94846047096F90000F0B196F90000002817DD1DE0B7F5505F07D114484C
:20D8B0001249006800F5C070086001F091FC0AF0ADFA48464246047092F9000030B192F968
:20D8D0000000002806DC0AF0C3FC03E020460146F9F702FC8AF80040BDE8F087941B00204A
:20D8F0009A1B0020D8120020931B0020301700200C0100219E1B00202DE9FE4F83460020B1
:20D91000304E00907068019180472F4C0290E06804216A4605F0F2F92C4DDFF8B4A0DFF833
:20D93000B490DFF8B8802C4E2BF0010725F00105BD4213D0504620F00100B8421CD14946CD
:20D9500091F9000010F1020F18D03068826B91F90010E068904781280ED10FE0414691F96D
:20D97000000010F1020F09D03068826B91F90010E0689047812801D00AF06AFC3068C66ACC
:20D990001749019AE0685B46B047061C01D50AF05FFCBD4207D0504620F00100B84204BF15
:20D9B00049460E7001E041460E7001200090E06804216A4605F0A2F9024902988968884761
:20D9D000BDE8FE8FC0150020E01900207DEC00002D080100911B002038170020901B002052
:20D9F000D81200202DE9F84F07463248DFF8C89000EB4706183699F83800348890468B4608
:20DA1000B8B1D9F85010A1B12C4D05EB8705686B00F0FF0088478246D9F85010686B00F4C4
:20DA30007F008847504480B218B131884018001D84B225481230007801280CD198F8086070
:20DA50004EB11F4898F8093081190D79C05C2418641DA4B200E00025281980B209F058FC73
:20DA70000646184890F80090D6B13046002122460AF006FE4FF00008A41937700D4986F8CF
:20DA9000018006F180007460CA5D358159460AF0F9F94846314606F01BF84046BDE8F88F82
:20DAB0008DF8007068461A2103F04EFA1A20BDE8F88FC046749B0100201500205CA001006F
:20DAD00078A40100B01600205A0F00202DE9F04F364E0025ADF1340D07464FF0010AA84648
:20DAF000A9460C93DDF858B00B914AE017F8020FAD1CADB2401E1BD0401E09D0401E04D0EB
:20DB1000401E36D1022C34D138E0032C31D135E0072C2ED1B9787878FB1C40EA0120A6F8AC
:20DB30004400186806F14802106086F859A025E0052C1ED1CDF80890B91C0A8802A80280D4
:20DB5000897881700B9803A9FBF754FD9DF82A00A0B1029B40F0020000F0F7008DF82A00BC
:20DB700006F1500203931068049003A805F008FC04E008EB0400801C1FFA80F8E719641981
:20DB9000A5B23846694608F0DFFC041CAED1022D03DC4D466720A84600E048460C990D80C9
:20DBB0000DB0ABF80080BDE8F08FC046A82A00202DE9F84F0D46064628684FEA900A324880
:20DBD000504502D3287A022802D00320BDE8F88F0AF018FEDFF8B4800090D8F8580108F50D
:20DBF000AA79B04214BF00240124A00080F0040059F8007006F19C0083460AF047FD68B954
:20DC100057B107F19C000AF041FD38B93846022100F060FF074602E0022700E000271C487C
:20DC300000686FB998F8880140F0020088F888010098C8F87C610AF0E1FD0020BDE8F88F97
:20DC50002A68A10001EBC40149440A612E7A0E76BAFBF0F1012998BF012158460AF08AFD54
:20DC700058460AF0C3FD00980AF0C8FD012F07D1D8F88001B8F9841198F886210AF07FFC9A
:20DC90008320BDE8F88FC04640420F00A00A002010A501007CB5354C054694F8A1000F282D
:20DCB0005ED03348697E0078890959D2297E002841F00201297639D069684A1C1078801095
:20DCD00010F0030F32D000F0030002280ED1B4F8B4304FF6FE70984208DD567911790020A9
:20DCF00001EB0621994208BF012004E004F1AA00491D09F029FFC8B9687E696840F00100CB
:20DD100068764A78C2F38102022A2DD1491D4A7809784FF6FF7601EB02218E4224D1297E13
:20DD300000F0EF0041F0200129761CE0687E114E40F0030068763078B0B994F8D7008DF8B8
:20DD50000000FF238DF8033094F8E6608DF8016094F8E7508DF8025068460AF00CFC7CBD9E
:20DD7000687E40F0010068767CBDC046A00E0020201500207319002070B50546344C287800
:20DD9000ADF1200D00284FD1208F04F148066B88ADF800003146ADF81030E2200AF030FA54
:20DDB0000DF1120031460AF0CBFB6988532009F00DFF208F04F13E063146ADF80E004A2027
:20DDD0000AF01EFA01A831460AF0BAFB00268DF80D60A08FADF8020094F83A308DF80C30AD
:20DDF000304608F01DFD5220314609F0E3FE94F850000F281CBF01206070E06828B102685E
:20DE10001AB10DF10E0069469047032008F082FB94F85200032818BF042813D104F1080010
:20DE3000102109F0BFFD0DE0002060700AF08AF941F2883008F0F4FC0649B1F85A00401C11
:20DE5000A1F85A00216E09B12846884708B070BD7C140020B81300202DE9F0470D460646CD
:20DE70005FFA85FA280824BF2E4845402E494FEA8A03C85885EA00023240C2F300672B4ADB
:20DE900006EA0504B043224006F4E0240243B4F5E02F01D1500E14D306F4E020074310D0EE
:20DEB00002F4E027B7F5A02707D0B7F5803704BF22F4003242F4A02203E022F4803242F4C4
:20DED000C022DFF86C80CA5008F1D00739680122002002FA0AF40C4218BF101C5FEA000922
:20DEF00006D1F00D04D34146C5F3805001F80A00300E0BD30AF086FC290E34BF0021211C35
:20DF10003A68A243114339600AF078FCB9F1000F06D0F00D04D34046C5F3805100F80A108B
:20DF3000BDE8F087006000A000100840007F077F002002402DE9F04117460D460AF062FCA7
:20DF5000324C8046207883266DB16D1E04D06D1E55D0681E11D00EE0B4F8C4004FF6FF7185
:20DF7000814202D005E0206C08B9802648E0206C808C388044E0032642E03868002150220A
:20DF9000054604F019F9022704F5AA7C04F5B272A5F110015CF8040B41F8100F137A0B734E
:20DFB0005068486052F80C3B7F1E18448860F1D1206C002808BF02200ED0206CC068276CFB
:20DFD000286297F82600236C85F82C00D869226C6862106AA8620320E76B8FB105280FDAD2
:20DFF000FA6801016A5097F826204C192273FA6962603A6AA2603F68401C40B2EDE73870E8
:20E0100040460AF0FBFB3046BDE8F081A00A00202DE9BE410546DFF8CC802978B8F86C00E4
:20E03000E1292FD0B8F86E00E92926D0B8F87000D9B92D4C2869676A02903FB37F692FB3C6
:20E05000A16A1931814221D806208DF800000422ADF802200023ADF804309DE8030002ABD6
:20E07000B84708B90298A06210E0401C80B2A8F8700019A00AF0C0FA08E0401C80B2A8F823
:20E090006E0003E0401C80B2A8F86C00687830F07F071ED000F06001402906D12F7827B9F9
:20E0B000B8F85E10491CA8F85E1000F06001202906D1287820B9B8F86400401CA8F8640061
:20E0D000602906D1287820B9B8F86A00401CA8F86A00BDE8BE81C04664617461436E663A02
:20E0F0002000C046B8130020D4110020F0B52A4A2A491778ADF1140D002F44D02C480778EA
:20E1100037F07F073FD1488C2A4F254D2A4B401C0024488407F16806012097F87410287080
:20E1300001F0F00187F8741019783C67012902D02146F8F7D1FF0AF077FA1C4D281D006813
:20E1500080470746029402201C4A164B8DF80C0021468DE803001068314602AAF8F726F804
:20E1700017490028A1F12001088008D40E49154C91F90000401C0870A4F114000660A968BA
:20E190003846884706E0888C401C88840020107009F06AFC05B0F0BDC42E0020401A0020D3
:20E1B000931B0020D51F01009A1B0020C0150020C62E0020D81200209E1B0020EC190020A6
:20E1D000301A0020381700202DE9FC47314CA11D0888401C088009F099F90026B04635462C
:20E1F00081462846694604F0FFF98246BAF1FF0F4CD09DF80030606B23B900EB4A10406849
:20E21000010402E000EB4A10416848460AF01EFA864203D29DF800700646D0466D1C0A2DB5
:20E23000DFDB1E4D281D0068804794F833106FB9A26B08EB88030026FF27491ED218D670D0
:20E2500013791771C9B284F833100CE0616B0022FF2701EB48118A77CB7FCF7794F83210BC
:20E27000491E84F832100C4A643BD9B2136804EBC1013C310B6052684A6094F88C10491EF2
:20E2900084F88C10A9688847BDE8FC870AF0DCF9BDE8FC87CC100020C0A40100C015002001
:20E2B000E0B501880025A1F6020159B143F20402891A04D0491E57D190F8246000E0022612
:20E2D000C76901E0C67B4769002F4DD03F1F052044F2380357F8041F0A04120C934203D0A6
:20E2F000401EF7D13F1D01E0C1F30345002D3BD01F4B3046401F18D01C4A401E10D0001F8D
:20E310000CD0801E0DD0C01E06D00F3819BF1A1C6032184A443204E0121D02E0121F00E01D
:20E33000083A1068C0F3834003E01A461068C0F303200F2806D0A84216D921F4702141EA55
:20E35000004110E0761F0AD0761F08D0761F06D00F3E1CBF21F4702141F4802103D121F4A8
:20E37000002141F4E0213960E0BDC0460011005020130050C4100050F0B5064600210B22B3
:20E39000ADF1240D0DF119000AF07AF92E4F2F4C3078C01E14D0801E04D0143810D0801F7B
:20E3B00001282DD801208DF8180006F18B0103A80AF040F9032538788DF8145068B112E034
:20E3D00000208DF8180006F18B0103A80AF032F9032538788DF8145028B9B4F8BE000225EA
:20E3F000ADF8020005E00DF1020004F1D8010AF021F98DF80A50B4F8BA00ADF8160017E0A8
:20E4100002208DF8180006F1320103A809F086FE0DF1020006F1280109F080FEBA342088AE
:20E4300006F11C01ADF816000DF119000AF0FFF80B208DF8000077788DF80170684600F0C2
:20E45000DBF809B0F0BDC04658150020A00E00202DE9F84F8A463149044601F1B400007803
:20E4700028B920465146F7F76FF9BDE8F88F0A25884642F2107B20465146F7F765F998F897
:20E49000B410002848D19AF80060D4F80090002937D023480168C88AC20832D280094FF02D
:20E4B000000702D3087D15282BD009F00FF898F800308446002B0EBF09235B1EDBB20A20D5
:20E4D00003EB830208EB0201491C0A78964207D0002B0EBF09235B1EDBB2401EF0D110E0F4
:20E4F000D1F8011060460AF0B1F8642101FB09018B4505D942F242706426401AB0FBF6F74E
:20E5100017B90020BDE8F88F20686D1E07442760B1D10AF099F86120BDE8F88FA82A00203E
:20E53000700D002080B50288A2F602073FB143F20502BF1A14BF002090F8240000E0C07B0F
:20E550002C4AD2F88832401F0B6048D0401E3CD0001F30D0801E24D0C01E18D00F380CD0CB
:20E57000D2F890024860D2F894028860D2F8BC0220F0784040F080503AE050694860D06A3A
:20E590008860506C20F0784040F0704030E010694860906A8860106C20F0784040F0F04068
:20E5B00026E0D0684860506A8860D06B20F0784040F0C0401CE090684860106A8860906B97
:20E5D00020F0784040F0A04012E050684860D0698860506B20F0784040F0405008E010683D
:20E5F000486090698860106B20F0784040F02050C86080BDC410005070B506463049307884
:20E610000D5C401F1CD0083851D0401F4FD0284608F07EFE041C0DD130780C2808D17068EA
:20E6300030B1301D07F0B6F8284608F071FE0446002C43D02A462046314609F023FC37E01D
:20E65000B07810BB327A307C51005410401901F00E01091804F0380040182430C0B208F0EE
:20E6700057FE041C2AD03146182209F00BFC04F1180060607168242209F004FC6068243069
:20E6900060617169327C0E46D6E7012816D12435E8B208F03DFE041C10D03146182209F030
:20E6B000F1FB04F11800606071682422EBE7344624B104480078214605F00AFA70BDC046FA
:20E6D00020A40100A01B0020F8B509F093FE04F01BFC09F0A7FE044604F00C000C284BD011
:20E6F000E0081ED208F034FB264E376805460120014609F049F831686943884211D2224CAB
:20E710008220B0FBF7F0291A20460AF033F820460AF06CF80120F8F7A3F8204608F0E6FF35
:20E730002CE0200928D2194809F027FE0428FAD0174A610905D220B11168104621F00101D0
:20E7500003E01046016841F001010160983210684FF0805540F003001060D5F8B80181690A
:20E77000202088470B4CD5F8B8712068B86B804701202060206801E009F062FF09F040FE20
:20E79000F8BDC04610A50100C40F0020004003408C2108402C200940F8B5324D6868804735
:20E7B00006462E4CA9682068002853D160698047676A40F01000002F4BD00022797E014059
:20E7D000884205D03A4657F80C7C002FF6D140E004F12400394607F01FFA002F39D02760B6
:20E7F000787E30F07F0005D194F82F00401E84F82F0004E094F82E00401E84F82E00A96823
:20E810003046884723681889D98A05F00BFEA0851348007808F04CF80546D88A000A08D350
:20E83000D87E06F011F8206890F91C0009F03AFC2368687B012803D002280DD1052005E09B
:20E85000187E401080F0010000F00100F9F7F8FEF8BDA96830468847F8BDC046700D002017
:20E87000870F0020C01500202DE9F047294E04463078ADF1280D012849D1DFF8B09009F100
:20E8900020000068244F436CF868022108AA98479DF82000002831D1DFF8948008F10400E3
:20E8B000006880470024022582461C48059404A90490F8688DF81850FFF77AF935700294D7
:20E8D00017498DF80C50174B4C8126468DE86000F86802AA0831F7F769FC002801D509F0E8
:20E8F000B7FC114991F90000124E45464F46401C0870A968FE605046884708E03078012890
:20E9100005D10020012C307001D009F097FA0AB0BDE8F0879F1B0020E019002000093D00BA
:20E93000D8120020894401009A1B002018170020C0150020E01200202DE9FF412E482D4F7C
:20E9500000683E78C06B80477968401AB100B0FBF1F4B868FF680025A8464146BC4271EBA0
:20E97000080101DAB84206D82946424684428A413CDA074600E0294638463246F317001B76
:20E99000A94109F0A3FA272704464FF47A7200230D46ADF802700820ADF800002046F8F771
:20E9B00085F901901548016868468847029843464FF0000100F6FC02A41A9D416042A94176
:20E9D00011DA0F48026829462046F8F76FF90D4604464FF000016042A94104DA204606F0AC
:20E9F00079FD002000E00120064908700090BDE8FF81C046201B002038170020E41500200B
:20EA1000CC190020C52E00202DE9F84F2E4C012683461D4690468946C4F87C670320C4F881
:20EA300080670AAFC4F88407D4F88C0710F0030FFAD1387A58B14FF0805ADAF8B001016AE1
:20EA500027208847DAF8B0010169272088470220C4F8FC063868C4F80804304609F0C9FD10
:20EA7000D4F808040008F8D2D4F88C07800F28BF301C26D22868C4F83C056868C4F8400565
:20EA9000A868C4F84405E8681049C4F848053879002814BF081D081CC4F84C05C4F850850C
:20EAB0000020C4F85405C4F8580509490E60C4F800B0C4F80880C1F80064C4F82090C4F843
:20EAD0002880BDE8F88FC046044002402800002000004842314A2DE9F0410446106C002349
:20EAF00001261F4687420CD0106CC068844208D1106C90F8260009F055FB3E46031C18BFA5
:20EB1000176CD56BDDB1D56B17E0C868844205D191F8270040F0080081F82700096826E092
:20EB3000E868844208D195F8260009F03BFB002608B10BB92F4603462D68002DF0D1002EE2
:20EB500018BF022027D1002B14BF002F002022D0106CC0683946844209D1106C884206D195
:20EB7000106C2730017841F008010170D16B0029CBD1C2F87C4192F8880140F0010082F858
:20EB90008801BE8CC2F8804103F00103A2F88461012082F88631BDE8F081C046A00A002069
:20EBB000F0B506460F4600251446ADF1240D8B200DF10E010095FCF7F9F98A2001A9FCF738
:20EBD000F5F9707A00282ED1387AA0B9BDF80E104FF6FE70884205DCBDF80E10884220D15C
:20EBF00001A90DE020489DF80E700488BDF80E008DF812700CE0022807D0032811D1394624
:20EC100004A809F017FD09240BE038888DF812008DF81040211200128DF8111005248DF84E
:20EC30001300284611E002280CBF05240924012818BF311C04D1892007A9FCF7B7F907A939
:20EC5000224604A809F01EF9B07A04EB0D01C8736A4604A8214603F051FC002814BF281CDC
:20EC7000009809B0F0BDC0465A0F00202DE9F041294D012001462870F8F72EFA27496FF054
:20EC9000010008702B480068C06B8047244C074621786068A2688B003E1AB6FBF3F05843E4
:20ECB000361A88001F4902FB03F8B1FBF0F0904201D209F0CDFAB91B1B4861604144FEF7A9
:20ECD0001BFE1A4CA06867682168404207F0BAFB002F08BFA16808D0A16878688142DCBFF9
:20ECF000401A78603F68002FF7D1E068884202D0A06005F02BFF02F04DFD0D4C606880470D
:20ED10000646FFF719FEA1683046884708F0C8FE00202870BDE8F0819E1B0020901B00200C
:20ED3000201B0020FFF6C2FF7DEC00007C1B0020C0150020381700202DE9F84F07460E1C5A
:20ED500014BF4FF000094FF0E809002F4FD0B9F1000F4ED17868401E78603F210170BD6D21
:20ED7000002D0CBF802000207968DFF890A00224083E491E7960DFF880B008703889A7F858
:20ED90005440801C388116F8080FFF282CD02A2828D1706830B35546296D88478046786886
:20EDB0009BF80020A0EB08007860716829B96D6D3A460023A84748B10BE06D6D7868716887
:20EDD0008DF800206B463A46A84710B9EB20BDE8F88F3889B7F854504044388108EB050015
:20EDF000A7F85400641ECED17868386501E04FF0E8094846BDE8F88F0C2E002020150020F8
:20EE1000F0B52F4C0546A07EADF13C0D022806D0012804D005281CBFE820607649D194F8E9
:20EE3000600000284AD1002109A81822617609F027FCCDF828D009A8294600F017FD94F8B3
:20EE50002E0094F85810814220DD266B70B10746BDF80A007189884204D13046694607F04D
:20EE700061FF98B97F1E06F12406F1D194F82E00276B8100242201EB40117818694609F0C9
:20EE900001F894F82E00401C84F82E000D48007828B19DF8340010B994F8580028B909A8FB
:20EEB000FFF7AAFB94F8580040B194F82E10884204D12A202870284605F0B2F80FB0F0BD0E
:20EED000E42C0020360F00202DE9B841804608F0FBF8C01DC51098F82300002849D198F896
:20EEF0007E4008F0F1F8A04243DD264A1368E010191891F86C1004F007042141CFB207E087
:20EF1000401CC0B21918C40091F86C7088F87E4047B9691E8142F3DC1068002188F87E10BB
:20EF3000417029E098F97E10C0000830884226DD401A79080BD298F87E10401E4FEA670748
:20EF500001F1010188F87E10F3D1BDE8B88198F87E000D49087098F87E0088F8810098F882
:20EF70007E00401C88F87E000320F9F769FBBDE8B881002088F87E00072005F0C7FEBDE8B0
:20EF9000B881C046700D0020E01900202DE9F041054609F069F8287E000904D2287D01282D
:20EFB00008BF022700D00527DFF89C80464670688047264C04F124010B68002B08BF0D60D9
:20EFD0000CD07F1E0026FFB202E07F1E1346FFB253F80C2C22B92FB143F80C5C012601E05F
:20EFF000002FF2D1D8F8081088471EB3216928468847E88AA168C00818D2D8F804008047F8
:20F0100094F82F10491C84F82F10D8F8081088470C4991F8380028B10846C06C10B180474D
:20F03000BDE8F081FFF7B8FBBDE8F08128468847BDE8F081F1206870284604F09BFABDE813
:20F05000F081C04620150020C0150020700D00202DE9F8430D46064668687468B7684FF048
:20F07000000810B9E86800284FD02078012814D109F0C8FBD4F8BC1049B1D4F8C0108D619A
:20F09000C4F8C05009F0BAFB0120BDE8F883C4F8BC50C4F8C05009F0B1FB022007F078FBE0
:20F0B00004F160004FF0FF31814609F08BFBB86809F044FB3046294602F042F90546B86861
:20F0D00009F054FB207888B9B5F1FF3F08D004F17C004FF0FF3109F075FB207A48B111E076
:20F0F00003202072022007F0F7F80BE0B5F1FF3F02D04FF0010805E00320207204F12C009F
:20F1100009F030FB484609F075FB4046BDE8F8831A481B4901641B4941641B4981641B493D
:20F13000C1641B490165022280F8202019494165194981651949C16519490166194941664A
:20F15000194981661949C16619490167194941671949016019494160194981601949C1606D
:20F1700019490161002180F83C1080F83F101749C161C162012180F8301070476C2C002021
:20F19000F57400008D430100CD4E01006947010021350100815F0100497201000D52010004
:20F1B0008940010065570100BD7D0100511B010095520100957A0100C1820100FD75010061
:20F1D000910D0100E935010085860100F1820100F8B5264C236813B909F03AF82368244849
:20F1F0000068044608F04AFFD860204608F020FC264C18826068804706461E48A16802788A
:20F21000832A30D11C4DEF782FB386210170082008F0FCF9E88C1B4F1949401CE8841748EA
:20F230003A7881621849812A09DB0978842A07DA40F6485292FBF1F101F6B83106E00978A3
:20F2500040F6485292FBF1F101F2A321203008F035FCA16807E085220270304688470020C1
:20F2700002F020FBF8BD30468847F8BD700D002030170020C62E0020401A0020101A0020E6
:20F29000A94B0100870F0020201B0020C015002070B5214E002086F85400802186F8550069
:20F2B000E82008F09FFC5220012108F083FC1B4D482205F17C0406F15C00214601F0FCFAAF
:20F2D0001748C5F88000343CF4601648C5F888001548C5F8AC001548C5F8A0001448C5F882
:20F2F00084001448164CC5F88C0013481549C5F89400124847F23052C5F89C0004F198006E
:20F3100005F094FD4EF660220F49A06104F1BC0005F08CFDE06170BD7C140020B813002000
:20F3300089DD0000495F0100052A01004DF600009168010031120100E11D0100512001008C
:20F35000D4110020057B01009D76010003B42DE9F0472C4C4FF0000908AF84F801903968DA
:20F37000ADF1100D02A80160B988818002A803C89A46164602F0CAF9A046051C14D04C4692
:20F3900086B128466946012207F072F91AF804009DF80010884205D1641C6D1CE4B2ADB22B
:20F3B000A642EEDCA64227D0B8F80200F61C4FF6FC7440F6F87134402018814203DA08F050
:20F3D00097FFFCF785FA396802A8BE88016002AD868095E803002246534601F07FF998F8F4
:20F3F0000100B8F80210002818BF814604D10919083188B2A8F80200484604B0BDE8F0474A
:20F4100002B07047141700202DE9B043044609F0F9F981462748021992F8EE10491ECFB229
:20F43000002F82F8EE703FD1254901EB84014A880C78904634F07F0718D1E1090FD24FF0FD
:20F45000805000F5DC75D0F8B8018169104688472868416B404688470228F9D11EE000EB88
:20F470008800D0F804110020884717E04FF08055D5F8B801016A10468847D5F8B801816A96
:20F4900040468847D5F8B801016B404688470A4901200860094908688008FCD304F03F0098
:20F4B0003F2801D0FFF7B0FF484609F0A7F90020BDE8B083B80F0020282008602820084019
:20F4D00000A20100F0B52B4D05F12C0158C9ADF11C0D02AA58C20AC94FF0805682E80A002F
:20F4F00047688468D6F8D001C16820688847216821488A6B10408863206840F2F27141645E
:20F5100097F83C0097F83D10C0100DEB80008068084321684863684609F00CF9D6F8D0013A
:20F53000397F466805EB8101BA698B68797F206855F821101943BB7F05EB8305AB690B435F
:20F550000199B0470D490A1F106840F010001060086840F001000860A07D0027FF2802D01D
:20F57000E07DFF2800D11FB1086840F44040086007B0F0BD94A201000DF8FFFF30100040AC
:20F5900029482DE9B0410025DFF8A080294C0570ADF1140D88F83B50012088F83800201DFD
:20F5B000006888F83D508047234924310F686FB1797E8A0806D341F001017976397E01F07B
:20F5D000FD01397657F80C7C002FF1D1A1688847102008F085FE082008F082FE98F83C00B7
:20F5F000E0B90920124C8DF80000B4F8BA108DF80F50E027ADF8021094F8D7308DF80170B5
:20F6100094F8E6208DF8043094F8E7108DF8052068468DF80610FEF7EFFF01E088F83C5049
:20F6300005B0BDE8B081C0462015002038190020A00E0020C0150020700D002070B5054693
:20F650002B4C2878ADF1200DEB2829D040B3E92806D0E12843D14FF4FA7007F0B1F83EE04A
:20F6700004F156010878401C087094F85200032818BF042803D14FF4FA7007F0A1F894F831
:20F690005600032809D094F85200022827D104F10800102108F086F921E007F089FC1EE0E0
:20F6B00094F85200022817D104AE6946304606F091F85220002108F07DFAE06820B102686F
:20F6D00012B1304669469047042006F023FF04F10800102108F066F9002084F8560005485B
:20F6F0002A30016809B12846884708B070BDC0467C140020D214002030B50446ADF12C0D99
:20F7100008F0DAFC002818BFFC2050D168462146112201F0D1F8A57C617D8DF81250607C0B
:20F730008DF81510E37C8DF81100227D8DF81330A57D8DF81420002105B10121257E8DF8B7
:20F75000161094F825208DF81850E07D8DF8252094F824308DF81700E58C8DF8243004F1D3
:20F7700019010B220DF11900ADF8265008F08AFB607C1A2550B9812007F07EFC04460A9465
:20F79000A4B1FF21812208F07BFF09E09DF81510880000EB411080B207F06EFC04460A94ED
:20F7B00024B10720694603F01BFD002528460BB030BD10B5401EADF1380D28D0401E09D013
:20F7D000801E4FD0401E43D0401E3FD0401E3BD0002048E001A800F059FC04460CA942F2AC
:20F7F000090005F0F5F89DF83000002808BF002203D0022007F078F9024601209DF830109D
:20F81000009001AB204605F0E8FB0A3028E001A800F03CFC04460CA942F2080005F0D8F84B
:20F830009DF83000002808BF002203D0012007F05BF9024600209DF83010009001AB2046C4
:20F8500005F0CBFB001D0BE020200CE002200AE042F2130004A905F0BBF804A808F04AFC17
:20F8700080B200E004200EB010BD7047F8B505460E460520287096F849006968E870F06B9C
:20F890004861686806F1280108F048FCB6F842006968488196F846006968487468680024A4
:20F8B00004761F4869680078C873686806F11C01193008F0BCFE307C69688873706810F89C
:20F8D000011B6A68918110F8013B6A68918941EA0321918107786A68F91117F00707117492
:20F8F000214607EB470218BF012189184018401C10F8011B297201F00702E860491001F0BD
:20F91000380101EB420140187268318968618B18834239BF2C72211C801A091A2974F8BD70
:20F93000860F0020F8B5064608F06CFF264D0746A91991F8EE00421C002881F8EE203ED191
:20F95000224C04EB8604267806F03F003F2801D0FFF7E8FF648836F07F0018D1F0090FD274
:20F970004FF0805000F5DC75D0F8B8014169204688472868416B204688470128F9D11EE060
:20F9900005EB8405D5F804110120884717E04FF08055D5F8B801C16920468847D5F8B80196
:20F9B000416A20468847D5F8B801C16A20468847074901200860074908688008FCD3384603
:20F9D00008F01CFF0020F8BDB80F002000A2010028200860282008402DE9F84F294C8A46C3
:20F9F0008346211D08880A254FF0FF09002604F13C084746401C088038465946082207F0DC
:20FA100099FC30B16D1E07F1080706F10106F3D100E0B146B9F1FF0F05D1207A401C20721F
:20FA3000FF20BDE8F88F4846694602F0DDFD0546FF2DF5D09DF80000012806D0A06B05EB97
:20FA50008501401880F804A004E0606B00EB451080F81FA009490A6808EBC90002604968E3
:20FA70004160074E7068804794F88C10491E84F88C10B16888472846BDE8F88FC0A4010053
:20FA9000C0150020CC1000202DE9FF47DFF8888001270446214E88F800703078012803D0B5
:20FAB00038460021F7F718FB204606F079F8214D68688047002482468DF80C7018490294E0
:20FAD00018484C8302238DE81800174B006802AA18318946F6F76AFB1449AA680028C88076
:20FAF0000AD4134B93F90000C1F80C90401C1870504690473C460AE04046047050469047B5
:20FB10003078012803D020460146F7F7E5FA20460090BDE8FF87C046941B00209E1B0020E8
:20FB3000D8120020EC19002009480100181700209A1B0020C015002010F47C1F70B51CD16A
:20FB500010F00F0F1CD001460024012202EA010091435200401E0BD0401E07D0801E03D00B
:20FB7000001F07D1093404E0241D02E0E41D00E0641DA4B20029E9D133E010F00F0F01D09D
:20FB9000002070BD064602244FF4803505EA0600AE436D00B0F5803018D0B0F5803013D0D6
:20FBB000B0F500300ED0B0F5802009D0B0F5002004D0B0F580100FD1072008E0062006E09B
:20FBD000052004E0042002E0022000E00120FFF7F0FD2418A41CA4B2002ED7D1022CD8BF13
:20FBF0000024204670BD70472DE9F0470020DFF89080224E234D88F83D0096F8A19095F84A
:20FC10004000401CC0B2042885F8400030D0202005F0A8FF96F8E3100F2917D098F83E7023
:20FC300096F8A100B84211DD194C8946606886F8A170804782461448144950F82700886073
:20FC5000C86004F083FFA1685046884795F8401096F8A13038F819404FF4707205F1100098
:20FC7000491C9A4001FB142107F0F2F9BDE8F08706F0B4FBFFF784FCBDE8F087A00E002001
:20FC900038190020A02D0020D4A201007C1B0020C015002090B5044600214022ADF1440DD2
:20FCB000684602F089FAA0788DF80000E0788DF801009DF8000000BB616811B101A805F01D
:20FCD00047FB217A01F007028DF82820E0689DF82870C1F302118DF8301027B19DF82810CA
:20FCF0000B9000EB41009DF8307007B10D90207C8DF8380067690F9719E0616811B101A8A7
:20FD100005F026FB677A8DF82970A37A8DF82A30207A8DF82800E27A8DF82B20217B8DF82E
:20FD30002C10677B8DF82D70E389ADF82E300348006801696846884711B090BD701B0020B1
:20FD5000F0B5012904460546ADF1140D04D0022941D142F2030001E042F20200694604F06E
:20FD700037FE04B16D1C07F0AFF9C01DC010C0B2002830D000230646ADF1010C1F4618463D
:20FD90001CF801EF00224EFA02F101F00101884211D028B97F1CBFB25CB102EBC30103E0C6
:20FDB0003CB102EBC301491E05F8011B091205F8011B80F00100521C082AE4DB761E03F189
:20FDD0000103DDD130B12CB1D800401E05F8010B001228700FB9002005E004B12770012080
:20FDF00000EB870080B205B0F0BD70472DE9F843254C80466068804781466946722007F020
:20FE10004BF83225FF27002600994046091D07F09BFE012808D000986D1E06F1010600F104
:20FE300018000090F0D100E03746A16848468847FF2F18BF381C22D1144DD4F804900A2748
:20FE500000263C3512492846082207F073FA30B17F1E05F1080506F10106F3D10DE04046EE
:20FE70000168296040686860C847064A92F88C10491C82F88C10A16888476436F0B2BDE857
:20FE9000F883C046CC100020C0150020CC100020C0A401002DE9B841044608F0B3FCDFF8A8
:20FEB0009880054608F5C4710878A04308F5AA7408702068002808BF002706D020689C30DF
:20FED00008F0E4FB002700B10127606838B19C3008F0DCFB0024384318BF0124274698F857
:20FEF000880120BB012F22D0D8F87C0110B3C76917B1016A890811D24069D8B10746284698
:20FF100008F07CFCD8F87C0100214FF400030A46B8470020C8F87C01BDE8B881284608F0BD
:20FF30006DFCD8F87C0102210022B847F1E7284608F064FCBDE8B881A00A002070B52348E1
:20FF5000214D4FF080562865D6F8D801204C036801210A46ADF1400D20469847D6F8D801BA
:20FF700042680121204690471A48012606601A48F9F78EF903F066FE05F06CFB284607F088
:20FF9000B5FE05F118044FF4E13029462060002005F080FB11493C2208230860002168469F
:20FFB00008F0C4FBF0344FF46170002307940C4908906A46069605F1580008F0B3FB08F05F
:20FFD000ADFB10B070BDC04608020020338601000040034004011CE29CA101009806002010
:10FFF0008930000038B504F08BFD03F0C5F8204DC2
:020000040001F9
:2000000005F13800007820B11F4808380168012088471E48007810B91D48007808B108F034
:200020001FF91C4C606880471B4AA1681378022B1CD1144CA31C1B78042B1CBF83231370B9
:200040008847A17831F0010008D0042906D0052907D10020607108F023FB01E0FBF7E0FCFF
:20006000A178042903D007F059FB00E0884795F8380020B1E86C10B1102008F039F938BD73
:2000800020150020401A002030170020C22E0020C42E0020C0150020C62E002070B5044690
:2000A000E820ADF1280D09A904F05CFE9DF82400694607F053FB00280CBF00981E480DF1C9
:2000C00025016060E82004F04DFE9DF8250004A907F044FB58B90599C8200322B1FBF0F00E
:2000E000401EB0FBF2F15143401AC0B200E00020207206F0F1FF00216081656821700F4B82
:2001000061700A4608925968A9420CD1197A267AB14208D15989814205D1187820705E782B
:200120006670104606E008990C33491C06290891E9D901200AB070BD38C40D007017002026
:200140002DE9F047254C01258246984691460E46C4F87C570320C4F8805708AFC4F88407A7
:20016000D4F88C0710F0030FFAD1387858B14FF08057D7F8B001016A27208847D7F8B001F3
:200180000169272088470220C4F8FC06C4F80894284608F036FAD4F808040008F8D2D4F89B
:2001A0008C07800F28BF281C15D2B8F1010F14BF08200C20C4F84C051021C4F850150020AC
:2001C000C4F85405064A1560C4F800A0A160C2F800542662A162BDE8F087C04604400240A7
:2001E00000004842B0B50546264CE968E06888423FD1A86803F030F9A0B1E9684968A06C55
:200200000978022900D168B9012004F077FF832835D1E068783007F071FA04F1C80008F0FD
:20022000EDFAB0BD16492869A1F10802136805F110071843106097E80C0051F8102C181C47
:20024000104341F8100C00270F60A86841F81C0C0F68002FFCD004F13C0007F092FE25643C
:20026000206CC06840680078022808D14FF4004101E04FF4806104F1EC0007F05FFEB0BD7C
:200280001C100440A00A00202DE9F041DFF8948006460C4636F07F0015D1002E3ED1224D1D
:2002A000243D686880471E49096831F81620144321F81640A968884741461431086807F036
:2002C0004DF9BDE8F081042007F02AF8071C25D04FF6FF7038807C8008F0EEF841468C789C
:2002E000A7F10C05FF2802D0C96A40184478FF2C06D1384607F079FF07F0A6FABDE8F08179
:20030000304607F0F1FB01463A46FF20A872204605F068FF10B1384607F067FFBDE8F08110
:20032000B42E0020B0190020E415002025483EB50078002843D042F20100694604F050FB83
:2003400042F2050002A904F04BFB1D4D95F8540010B39DF8080000249DF80810009B2864DC
:20036000642285F85440581A02FB00F1E96705F1780003F063FF01A805F0B2FA1248019935
:200380002E300078B1FBF0F2451E4243891A01918D4214D9204610E09DF80810642048430E
:2003A000E86705F1780003F049FF288F401C288700242C64012085F8540004F0AFFC3EBD43
:2003C000A82A00205D0F0020642B00202DE9F041224C064604F1580005780F46002D04BFE0
:2003E0000020011C1CD0204D1D49281D0B780068D3B91C480568E06C07F0CAFE228FB0FB0D
:20040000F5F1B0FBF5F3891889B203FB05F2236C3980801AC018306085421CD8401B491CCD
:2004200030603980BDE8F08180475FFA80F804F1780007F095FF226C4FF47A73410001EBE2
:20044000C001B1FBF3F0238F3060A9683B808018306040468847BDE8F081C046A82A0020B3
:200460005D0F00206C2B0020C0150020F8B50F46002302B90123DFF890C00021EFB13D6AB1
:20048000DDB1C669CEB1FC68C768A74207D0DCF854110CF5AA77A14214BFF968B968B4087E
:2004A0006FF05047A4EB9504641AA74225DDB4F1704F01DB002C20DD01210AB3D769FFB17D
:2004C000066AEEB1D268C068824208D0DCF854310CF5AA70934214BFC068806800E00020E3
:2004E000C0EB97006FF05042A0EB9600824204DDB0F1704F03DB002801DC0020F8BD0123C7
:2005000001EA0300F8BDC046A00A00202DE9F043254C0746243C606AADF1240D00283ED032
:20052000002F3CD0387A002839D004F04DFE5FEA000834D0062000250323A1468DF8080024
:200540002E46ADF80A30B5F5FA7F28DAD9F82400ADF80C5004AB02AA0469009392E8030055
:200560000A230022A047B0B9387A9DF81810814210D1022804D1BDF810103A88914207D089
:20058000032807D104A93846082206F0DBFE08B9284606E0761CB04505F10105D3DC4FF0AE
:2005A000FF3009B0BDE8F083F8110020F0B520480127F84201D004F01DFB204D204F214E7B
:2005C000BD4206D203CD0478A4003459401CA047F6E71D48002800D08047164D164FBD42BC
:2005E00002D210CDA047FAE7F0BD03251BE0416808300A1C2A400BD11A1C2A40AB4305D002
:20060000046804300C600431043BF9D1131C05D0047801300C700131013BF9D1021C2A40A3
:2006200001D0A84304300368002BE0D17047C046FFFFFFFF0000000000000000700E00004C
:20064000D00E00002C0E000055C5011070B504466068254E4078ADF1480DC00921D3B4F899
:2006600042003546E63DB5F8BA10884219D11D480078A0B995F8C40098B104F1280006F08C
:20068000C7FC70B9012000901C340194B5F8BA3005F1AA0203210620F7F728FA1FE007F04F
:2006A000C1F90BA80021182201F08EFD02A821460C900BA8FFF7E2F82C208DF82C000BA816
:2006C00003F0B6FC3546503D287810B19DF83C0028B105208DF82C000BA8FDF795FF12B08F
:2006E00070BDC04621150020860F002003B426482DE9F041058806AF1446ADF1080D984623
:200700004FF6FF70ADF800000222ADF802006946ADF8040044F40040ADF80600601986B289
:20072000304602F0DFF9BDF80600022269466FF3DF30ADF80600304602F0D4F9A11028467B
:20074000CAB2414602F0CEF9387840F40040ADF800007888ADF80200B88802226946ADF8B5
:200760000400304602F0BEF9BDF80000022269466FF3DF30ADF80000304602F0B3F902B0F2
:20078000BDE8F04102B07047161700202DE9F843002A894607464CBF47F6FF75151C002F1A
:2007A00008BF002033D03888002808BF002403D02A4600F085FB0446281B002826DD388851
:2007C00028B1291B484613A204F0A8FD0419B868E0B1D7F804802E1BB8F1000F0DD040469B
:2007E00007F090FC401DB04207DC291B48460AA2434604F093FD04192E1B122E06DBBB680F
:20080000291B484606A204F089FD04192046BDE8F883C0463A2000C0222573222C2000C039
:200820006C696E652025643A2000FEE7F8B5234D012001462870F6F757FC6FF00100204CFF
:200840001D4927690870381C28D0A1684268914203DA07F005FD27693846C8B105F0C8FB43
:200860007968884224BF2769381C11D200F09AFF14E026697068002802D507F0F1FC2669CD
:20088000304604F011F8B168307B88472769384620B105F0ADFB79688842EAD2094C606852
:2008A00080470646FEF750F8A1683046884707F0FFF800202870F8BD911B00209E1B00209A
:2008C0007C1B0020C0150020002A4AD05FEA000C8B071CD1830722D1102A08D370B4103A54
:2008E00078C978C0103AFBD270BC103238D0042A2CD3082A05D30C2A24BF08C908C008C938
:2009000008C008C908C092072AD0920F22E00B780370491C401C521E22D08B07F7D1C30703
:2009200014D18307D8D0121F12D308C903801B0C4380001D121FF8D20AE008C903701B0AE1
:2009400043701B0A83701B0AC370001D121FF4D2121D05D00B780370491C401C521EF9D16B
:2009600060467047F8B507F055FF234C0746D4F8C00010F4602F33D0D4F8C000400CC6B2F4
:20098000700807D2B00803D2F00828BF022602E0012600E00026751D002168B203F0B6F9F4
:2009A000D4F8C03006F111010120884023EA00013846C4F8C01007F029FFB00004F1A80104
:2009C0000A18D7682FB1085800224FF000632946B8470A48006830B9022004F08FFB02E01F
:2009E000384607F013FFD4F8C00020B104F59070002107F0A3FAF8BDA00A00200C10044086
:200A00001CB51F4C04F1780006F012FA04F15C0006F00EFA04F1940006F00AFA002188228E
:200A200004F1340007F034FE07F0CCFA06F054FB84F85A00134984F85B0013480860012075
:200A40000DF1010184F8B30042F2040003F0C8FF42F20500694603F0C3FF0C489DF80110DE
:200A6000A0666420414321660949C4F884109DF800104843E0670748C4F8A0001CBDC0463E
:200A8000A82A00202817002021660100494901002D030100D9850100D0B5244C04F124014B
:200AA0000F68002F3FD0002215280AD13B7D0126022B08D0032B06D0052B04D0042B02D05A
:200AC00000E03B7D0026984200D016B17B7E5B0905D23A4657F80C7C002FE5D123E0084626
:200AE000394605F0A1F8F88A2760000A03D397F91C0007F0DFFA387D022818BF052802D1CE
:200B0000012006F08BFD2068407E30F07F0005D194F82F00401E84F82F0004E094F82E0019
:200B2000401E84F82E003846D0BDC046700D00202DE9F843234D884606464FF0FF3105F1BF
:200B40002400814607F046FE00200CE0FF2909D02A688A4204D905EB8101D1F894700FB128
:200B6000002627E0401CB8F1000F03D018F82010FE29EBD10024346074600127B46011E085
:200B8000FF280ED005EB80000B787268C0F8946007FA03F0104370600A680949304605F091
:200BA00089FB641CB8F1000F04D008EB84010878FE28E5D1484607F025FE3046BDE8F88393
:200BC000007FC7672C260020B0B5456884682349607DA27DADF1180D40F000400090207D30
:200BE0000027FF2A41EA000001904FF0020002D0E27DFF2A00D13FB1E37DA07D1943039120
:200C000040F0004002900420FE214DF8201005F158006946FFF78CFF6866002808BF381C8B
:200C20001AD0617D0F2205F0BFFF686E217D102205F0BAFFA17D3846FF2902D0E27DFF2A96
:200C400000D140B1686E112205F0AEFF686EE17D122205F0A9FF012006B0B0BD0000C0A07E
:200C60003EB507F027F80446204D2149286981422FD1204905F17000002207F0E6FC01200B
:200C8000287006F05FFE00204FF6FF71B5F8C4306871994209D10220ADF80000684606F0FA
:200CA0002BF9BDF80800A5F8C400286C60B905F13C0007F0DDFC031C06D004F09BF840B9CE
:200CC0001846FFF78FFA04E005F1EC00022107F035F904F0804104F00200084305D005F168
:200CE000EC004FF0005107F029F93EBDA00A00206939000031CB000098B5244C0746A8B199
:200D0000401E0BD0401E2CD1204690F8402042F0080202F0EF0280F8402022E094F840200C
:200D2000204602F0E70242F01002F4E7214601F17402107891F83C3000F0F000107003F0B4
:200D4000F000002281F83C0091F840308A6343F0080000F0EF0081F84000F420413104F099
:200D600001F8002F08BF44F620600CD007F0FAFB4FF4FA670A2244F6206390FBF2F1514373
:200D8000401A07FB0030A06498BDC046D812002038B5054695F83000032839D195F83A006D
:200DA000032835D105F128044A202146F6F7A0FA8A202146F7F77AFA6C686178207800EBE5
:200DC0000120ADF8000069465020F6F791FAA41C6178207800EB0120ADF8000069464B20BA
:200DE000F6F786FA8B206946F7F760FAA41CE1202146F6F77DFA641C6178207800EB01205B
:200E0000ADF8000069465320F6F772FA002000E0E82004492A24087028462C7003F008F999
:200E200038BDC046FD2C00202DE9F8432020EFF3118780F31188214CA068012107F072FC5B
:200E40004FF001094FF0000865692168A4F81C906A1A2168A4F81E80461B401A904227D395
:200E600087F3118840464519361A4846294607F055FCB042F7D92021EFF3118781F311885C
:200E8000E18B012903D14046294607F047FCB0F1FF3F06D0A169801B814238BF081C411927
:200EA00001E0A069291807F035FCA4F820902560A4F81C8087F31188BDE8F883780100200A
:200EC0007FB503461F480D4601881F480088144614A6984205DB32462146284604F01EFA3C
:200EE0001DE0994206DB184606F028FC0028F2D04268F1E715480088002808BF0CA2EBD018
:200F00000095002C48BF47F6FF74114E0020114901946A46346802901846A047029800909E
:200F20007FBDC0467B6D6F64756C652325647D007B6D6F64756C652D726F70653A25787D0D
:200F400000C046C028A501002AA501008E14000024A50100116A010090B50C46214A0178CA
:200F6000575CADF11C0D0B2F8DF8007035D0002F36D00C2F04D0112F29D107F036F926E019
:200F80001A2C22D090F899100190C7688DF80210038A0297C28AADF80C30510905D21249B2
:200FA000827EC8310978891A00E000218DF80E10877F8DF8107090F91F308DF81130826ADB
:200FC0000592417F8DF80F1001E0002001908DF801406846FDF718FB02E04470FDF7D4F9B2
:200FE00007B090BD809B0100A00E00202DE9F04107467868BE68044600F5847006F07EFBC7
:2010000030681C4980690968C0F3C00008BB07F001FC194D8046287820B1022005F064F93E
:2010200000202870404607F0F1FB3168134D886B20F020008863286820F480702860606AA2
:20104000216A091A21622369626A38469847BDE8F0814FF4FA70B0FBF1F1012998BF0121B7
:2010600004F58474204607F08DFB204607F0C6FBBDE8F08110A50100BB2E00203010004027
:201080002DE9F04107467E68D6F8BC00C8B307F0C1FB1D4D00248046042305F10C0004603D
:2010A00002202B6007F0ADFA7368D6F8A810384622469847022005F017F90BE08069C6F806
:2010C000BC007368D6F8BC10224638469847022005F00AF9D6F8BC00D6F8C0108142EDD157
:2010E00034722046C6F8A800C6F8BC00C6F8C000064B2C6038461C6003F098FC404607F0AB
:2011000085FBBDE8F081C04604280040100405422DE9F04180461E4800680D46416927204D
:201120008847012404FA05F61A4DC5F80064C5F87C470327C5F8807717480460C5F8847761
:20114000D5F80404012818BFC5F80444C5F8FC6312480460C5F800801023AB60204607F003
:2011600050FAD5F88C074008F8D3D5F88C17204611F0404F09D1C5F884770021C5F8FC16CA
:20118000D5F80024164218BF081CBDE8F081C046B00100100440024000E0484200004842B4
:2011A0002248F8B50C460178012904D0417A012918BF012034D190F8C710CA080AD390F8D7
:2011C000C620A24206D101F0FB0180F8C710002780F8C67007F01EFB074607F003FB0646BF
:2011E0000121204602F092FD0E48210201F47F41084305F081FE0C4A1168054604F10C03DB
:201200000120984081433046116007F0E7FA384607F0FCFA05F0FF05012D0CBF8120022032
:20122000F8BDC0460100080408100440A00A002070B50546204C2878002836D16078012814
:2012400033D0281DFFF762F9B0F1FF3F2DD1298AC8132AD001F00F010F2926D12046018F6A
:201260004FF6FF728A4204BFE9890187A97C80F83A10AE888687298A01F00F020F2A05D042
:2012800080F85020C1F3031180F8511090F850100F290AD1012141700848064607F000F86C
:2012A000012802D1304607F0E7F96C34216809B12846884770BDC0467C1400209012002020
:2012C0007CB515460E46044600E004192046694605F042F900282ED014F8021F8E42F4D1BA
:2012E000491E04F1010420D0491E12D0491E08D0491E18BF622029D102281CD12078287014
:2013000023E0032817D114F8010B2870207868701BE007280FD161782078A41C40EA012011
:20132000288020682E1D30600FE0052803D120780628287001DD67207CBD2D1D0020641CCC
:201340002860A678AE702088288000207CBD704798B54368C3F8A8100868C3F8AC00486877
:20136000C3F8B0008868D3F8B070C3F8B400C8681949C3F8B80017488FB9D3F8A820127CEB
:20138000520042F001020260022018720A68D20916D2D3F8B820022A16D30B2215E0D3F8DE
:2013A000A820127C012752000260D3F8AC201F72541CC3F8AC40127882600868C00902D342
:2013C0004FF0FF3098BD022003220A6007F019F9002098BD00280040042800402DE9F04100
:2013E0001E4615460F46044607F0FCF98046384605F032FC071C04D097F8270030F07F00F0
:2014000003D1404607F0EAF928E097F8270010F00F0F1BD113487968884202D07968A16610
:20142000786004F1600080E86000404607F0D6F904F140004FF0FF3107F0CCF904F170079F
:201440000020A06697E80300BDE8F081404607F0C5F997F8270010F00F0FFAD102200021B1
:20146000BDE8F0812933010070B506467468B568606E06F082F929681C488A6B104088632B
:20148000304600F037F8304601F0AEFD2968C86A20F01000C862296815480A6B104008637A
:2014A0006868FDF7B9FF04F1800007F053F904F19C0007F053F9A07818B904F1D00007F07F
:2014C00055F9607818B904F1EC0007F04FF904F5847007F047F907F09DF90021217007F09B
:2014E00095F904F16C0006F069F870BD0DF8FFFFFEFCFFFF2DE9F04106467568B46807F0FB
:2015000089F9A96A39B921688969090903D207F07DF9BDE8F0810027AF6207F077F9A17DA2
:201520003846FF2902D0E17DFF2900D118B12846214600F0AFFF2168886B20F02000886309
:201540000D49086820F48070086007F063F90B4C8046207818B1022004F0C6FE2770404691
:2015600007F054F9686A296A091A29622B696A6A30469847BDE8F08130100040BB2E0020B8
:2015800038B50C4644220546002100F01DFE04F12801284606F0D6FB04F1320105F10A00B4
:2015A00006F0D0FBE06B6861B4F840002883B4F842006883B4F84400A88394F84600A877DA
:2015C00094F84700E87794F9480085F8200094F8490085F82100B4F850006884E06C6862F6
:2015E000A07B85F8280094F8520085F82900606D0B2204F11C01E86205F13000FFF764F9D8
:201600002089A5F840006068E86338BD70B51E4DAC68064606F02AFB4FF47A71001B48435D
:20162000030C05F055FC2969401A48BF404240F6B8319B19994210D306280EDAE9688C421A
:201640000BD8286848B1114A091B51438A0C02EB1141884288BF011C08E00D4948684008D2
:201660000ED208687D2100F0FF004143C82905D3B1F57A6F88BF4FF47A6103E0C82101E09F
:201680004FF4FA61084670BD642E002040420F00AC3F00507CB5042005F05AFA022818D003
:2016A000032816D019480068C0F38150032814BF41F288324FF47A721649174C09684C34FF
:2016C0002046B2FBF1F107F05DF8204607F096F87CBD4FF08056D6F8A4010D4D44680021F6
:2016E0004FF040521C23032000902846A047D6F8A40100214FF400720923012644680096F4
:201700002846A047022004F0EFFD7CBDB43F005000A00C4010A50100C00F002003B4204846
:20172000F0B505AF3E787D880088BF88ADF10C0D001F84B2082C2CDB201F6946082280B235
:2017400004F09EFFBDF8000086420FD1BDF8020085420BD1BDF80400874207D1BDF806002C
:201760006FF3DF30241A241FA0B213E0BDF80600C10BCB0309D100F108018C4202DA06F069
:201780006FFD06E0241A083C00E0241FA4B2082CD2DA002003B0BDE8F04002B07047C04605
:2017A00016170020F8B51E4C002528462268A168256190420CD05268914209DD04F018FCF0
:2017C0000146206842689142C8BF41602061A168676837B118B142687B689A4201DD3846C6
:2017E0002061C8B14068814216DD0F4D044605F108000068A04201D806F032FD094E706876
:2018000080470746EC60204600F0A4FFFDF79CF8B16838468847F8BD05F070FD2561F8BD2F
:201820007C1B0020C0150020201B00202DE9F8431C481F4D07786868804781461A48836856
:201840000026344680469C4212D013F8020C874208D134B163B138464FF40041FEF714FDA6
:2018600013E01C4604B91E4653F80C3C002BECD15FB9686880470D49096831F817206FF33F
:20188000DF3221F81720A96888472CB108F108002146324604F0C8F9A968484688472046C1
:2018A000BDE8F883B0160020B0190020B42E0020C01500202DE9F041804600271A481D4D42
:2018C00007701A481A4E077096F83800D8B1F36F2C68C3B1207D352809D16068218900F061
:2018E000F5F860680088000901D304F07FF9F16F404688471048007801280BD03846014614
:20190000F5F7F2FB06E003F003F901F03DFC4046F8F782FA286810B1007D352801D006F00C
:201920007DFABDE8F081C046BE2E0020C62E002020150020700D00209E1B002010B5994289
:2019400001D1904233D050EA020404D141EA03046400002C2BD050EA410401D19C4226E0D9
:201960004C006415641C07D15C006415641C03D1DC0FB4EBD1741AE0002B0CD4002916D43A
:20198000994214D190EA020401D490420FE0002A0DD101240BE0002909DC8B4207D190EA2C
:2019A000020401D4824202E0002800D10124EFF3008454BF44F0005424F0005484F3008820
:2019C00010BD10B58B4201D1824233D052EA000404D143EA01046400002C2BD052EA4304BA
:2019E00001D18C4226E05C006415641C07D14C006415641C03D1CC0FB4EBD3741AE0002917
:201A00000CD4002B16D48B4214D192EA000401D482420FE000280DD101240BE0002B09DCF1
:201A2000994207D192EA000401D4904202E0002A00D10124EFF3008454BF44F0005424F0B5
:201A4000005484F3008810BD2DE9F8431E4C00264FF001084FF002093746A41EA51C15F8E6
:201A6000020F03280ED0022822D16878236802281ED006F003FE0146384606F0F9FC85F888
:201A8000019010E006F0FAFD014623686878012805D0384606F0ECFC85F8018003E0404665
:201AA00006F0E6FC6F700246C9B2184604F0C0F9761C042ED3DB05F06FFA18B104F12400EF
:201AC00006F0D8FDBDE8F883AA1800200829C8B50BDA00293BD00278491E92FAA2F24FEA38
:201AE000226200F8012BF6D1C8BD464206F00306891B37188AB2361802F00301864209D94E
:201B0000361A0378761E93FAA3F34FEA236300F8013BF6D122F00302D71987420AD93A1A82
:201B2000D21C96100268761E92FAA2F212BA40F8042BF7D1CF19874209D93F1A01787F1EF6
:201B400091FAA1F14FEA216100F8011BF6D1C8BDF8B50546012004F00DF81D4C04F11400C9
:201B600002F0A2FE04F1240002F09EFE69684A78087800EB0220ADF800008F7804F1140651
:201B80006FB953206946F5F7B3FB05F128014A20F5F7AEFB05F128018A20F6F787FB06F114
:201BA000200005F11C010B2206F074F9BDF80010384604F001FC94F83F00800803D3687825
:201BC000002106F0EFF8002084F83F00F8BDC0466C2C00201C491B4898B5FF220F7890F874
:201BE0003B301A4980F83820012B15D091F8A10091F8C010884224D015480024047006F00A
:201C00001BFD01F055FD13480078012819D020460146F5F769FA98BD002380F83B3087B1F5
:201C20008DF8032091F8D7008DF8000091F8E6708DF8017091F8E7408DF80240684606F027
:201C4000A2FC98BD381900209F0D0020A00E0020C32E00209E1B002070B50025ADF1200D87
:201C600007A8ADF81C5006F0DBFA1B4CBDF81C10208F884227D194F85300032811D0042809
:201C80000DD0022810D104AE6946304603F0AAFDE06820B1026812B1304669469047042085
:201CA00000E0032004F03EFCA06D04F091FD5220294605F087FF4FF47A7004F0A1FD2846DB
:201CC00004F0B6FD05E0032006F044FA052004F029FC08B070BDC0467C1400202DE9B84139
:201CE00006F098FD1C4C1B4D804604F1E000007848B92C46A168022088470746102003F099
:201D0000EBFA0FB31DE001F075FB70B9134800683221B1FBF0F101B901213034204606F056
:201D200031FD204606F06AFD0EE0002084F8E0002C46A168022088470746102003F0CCFAA6
:201D400017B1A16803208847404606F05FFDBDE8B881C04658A40100B80F002010A501006A
:201D60001D491E482DE9F041352751F8048B51F804EB51F804CB51F8046B51F8045B40F834
:201D8000048B51F8044B40F804EB51F8043B40F804CB51F8042B40F8046B40F8045B40F878
:201DA000044B40F8043B7F1E40F8042BDDD151F8045B51F8044B40F8045B51F8043B40F814
:201DC000044B51F8042B40F8043B40F8042B09680160BDE8F081C046EC02000000C00021A1
:201DE00038B505461B491D4C2878E0B96878012815D0022809D0032826D108460021817032
:201E00004021083005F0D6FD1EE004F13A000078FF280CBF0120022006F09CF914E004F113
:201E200008002021EEE76A78032A08BFEA2804D0012A09D141F2883000E0074891F85420AC
:201E400081F8552004F0F4FC7434216809B12846884738BD7C140020E09304007C140020BC
:201E600070B51B4C05461022ADF1200D04F171016846FEF729FD0026049509208DF814607D
:201E800004F10D018DF8160001258DF815500A680DF1170002604A684260097A01720D490B
:201EA0006A4618200DF09CF90B4918208922631D0DF096F97120314606F0CAF9D520214648
:201EC00006F0C6F95D20294605F07CFE08B070BDD49F01009DB70000AD8200002DE9F043CD
:201EE0001C4E044600271D468846A2EB0409ADF1140DC6F8B071012006F083FB3068C00FA2
:201F0000F9D3306A0090706A0190B06A0290F06A039044B128462346694611F8012B5B1E9E
:201F200000F8012BF9D10320C6F838026CB108EB09016D1E491E11F8010F15F8012F904264
:201F400018BF042002D1641EF5D1384605B0BDE8F083C046504502401849B0B50546164CD0
:201F60000F7820781FBB164A8100B2FBF1F1A94202D206F075F920786168154F800005FB90
:201F80000014A7F10C000068C06B8047211AA1F54871090806D30B4A011B891A090828BFAF
:201FA00000F5487408482146FBF7AEFCB0BD074901200870B0BDC046201B00209F1B00201F
:201FC000FFF6C2FF00093D007DEC0000C52E002044170020F8B51A4E1A4D0120002414EA4F
:201FE000030730704FF0020000EA020008BF00280CD14FF0E04004EA0201184008BF0029A6
:2020000004D11249888D401C888503E095F90000401E287005F030FD05F000FF0A480470CF
:2020200095F9000030B195F90000002806DC06F017F903E020460146F5F756F83470F8BD70
:202040009E1B00209A1B0020931B0020401A00202DE918410446DFF870802078E02828D171
:20206000404642788178012A0AD049B990F85220012A05D190F8540001281AD001200CE029
:20208000104BB3F87220521CA3F8722041B9491CC9B2817000234370022006F05BF808E019
:2020A000002004F095FB032006F054F8052004F039FA40467C30016809B120468847BDE89C
:2020C0001881C046B81300207C140020F8B500680E4617464FF0FF310446483006F07AFB64
:2020E0004FF0FF35092E08D0217A0120B040084211D108433546207210E0227A0721012356
:2021000003FA01F0104202D0491EF9D503E0227A0D4610432072B5F1FF3F0ED06FB1294670
:202120003846FEF7F5FF40B1217A0120A8404FF0FF3580F0FF000840207204F1480006F0B4
:2021400061FB2846F8BDFCB590EA01064CBF4FF0004600264FEA00224FEA40031B0E12BF47
:2021600042F000420020FCBDFF2B24D04FEA01244FEA41052D0E12BF44F000440020FCBDBA
:20218000FF2D18D05B19A2FB0454002C5CBF64005B1E803424BF5B1C64087E3BDCBF0020B0
:2021A000FCBDFF2B07D24FEA142030F4000040EAC3503043FCBDFF27FF0546EA0700FCBD4F
:2021C000002213460A46194671B510F0030F0BD0002A82BF00F8011BB2F1010210F0030F8B
:2021E000F6D1002A08BF71BD11F0FF0141EA0121042A18D341EA0141082A0FD30E46102A83
:2022000008D30C460D46B2F10F0312F00F0272C0103BFCD812F0080F18BF42C012F0040F1E
:2022200018BF40F8041B12F0020F18BF20F8021B12F0010F18BF017071BD7047F8B505461A
:2022400006F0E8FA1A4C0126074605F19C00E67005F054FA2078012811D094F8880170B1C9
:20226000B4F95000B4F95210884208D1384606F0CDFA0720FDF716FE06F0CCFA0746B4F98F
:202280005200B4F95010884218BF85F8C2600AD105F1780005F032FA304602F02FFFE17945
:2022A00020780843E071384606F0B0FAF8BDC046A00A002070B51C4C06460E220D4604F1F6
:2022C0003800FEF701FB687B28B9022084F828006B88238409E003202B1D84F828001A6837
:2022E00004F120010A6058684860206B04F088FA30462946FAF7AEFD207801280BD0687BF5
:2023000048B9288869882A1D01F01AFC011C02D001A006F079F970BD4175746820457272CD
:202320006F723A20307800C0B813002038B51B4D95F8A1000F2824D0194C3B3C94F83810B1
:20234000FF291ED094F83A0068B102290BD103F04FFE216B0F4C95F89820401A21780831E9
:2023600001FB12010BE003F043FE616B0A4B95F8C020081A1988401A34F81210411A0029B2
:2023800001D5002038BD4FF6FF708842C8BF88B238BDC046E11900209C0D0020A00E002067
:2023A000731900201C4938B591F85C3001EBE304657F012203F0070302FA03F383F0FF03CC
:2023C0002B4063778B7E01F11800032B18D091F86030012B10D0022B08D0B1F856108A408C
:2023E0009102A1EB821101F570710EE0B1F856209101A1EB820108E0B1F856108A4001E004
:2024000004490A789102A1EB82111C3005F05EFB38BDC046690F0020E42C002000B5002108
:202420002022ADF1240D6846FFF7CEFE1848018FADF8181090F83A108DF80B10808FADF838
:202440000E0002218DF816100A208DF80C0001218DF81F1080208DF80D0000208DF8080030
:202460008DF81B006A468DF81A0007498DF81D0018200CF0B5FE0549B1F85800401CA1F850
:20248000580009B000BDC04633850100B81300207C14002038B50C4621680546886B20F0FE
:2024A00020008863686E217D012202F07FFC686E217D012203F0BCFC686E217D002204F041
:2024C00073FB686EA17D002204F06EFBA878012806D005F1D0004FF0FF3106F07BF903E07A
:2024E000216888690009FCD2686E217D102204F05BFBA17D0020FF2902D0E27DFF2A00D10A
:2025000018B1686E112204F04FFB38BD2DE9F84F8346894617467120114604F0C5FC812026
:202520006946F8F74BFD4FF0F308002507E0B8F1000F23D038686D1CEDB22C3038609DF873
:202540000000A8421ADD3868066890F804A0002402E0641C0A36E4B2A245E8DD737A002B40
:202560000CBF052009208145F3D14A463046594605F074F80128ECD14FF000084046BDE85A
:20258000F88FFEE71A487CB5007880B342F2050001A902F025FA42F20100694602F020FAAD
:2025A000144C9DF80400216C88420BD80098884203D806F051F801250DE00022012584F895
:2025C000542004E001259DF8040084F85450401A64214143E16704F1340606F1440004F0BB
:2025E00027FC06F1440001F029FE84F858507CBD5D0F0020A82A0020F8B50B461A4991F8A0
:2026000031708D6B4C7A6430C2B25FB100206D1F6D1DEE7816B12E79B24207D07F1E00F1E0
:202620000100F5D1641CE0B2487204E0FF281CBF0021197016D10120187091F830704C6B07
:202640004B7A5FB10020203C2034A67F16B1E57FAA4207D07F1E00F10100F5D15B1CD8B26C
:202660004872FF20F8BDC046CC10002038B5054601201A4C68712879B0B90DF086F9217813
:20268000002904BF6FF00704051C15D0491EC9B2217039B90DF0A3F9606804F0D1F900203A
:2026A000687118E0054613E00DF06FF905462078FF2805D16FF0060428460DF090F90BE07E
:2026C000401CC0B20128207002D1606804F0CFF928460DF084F90024204638BDB41B0020C6
:2026E00070B50D461A49154C154A0968064604F11400B2FBF1F106F06DF8002808BF002080
:202700001BD010480570104D20682978B14210D02E7005F0FFFE201D064605F0A9FD287854
:20272000012804BF094820613146002002F09AFE2060002100B10121084670BD502D00202E
:2027400020A10700B92E0020B82E002046A4010010A50100154998B50F7817BB144A117818
:20276000144F52688B00890000FB0324B7FBF1F1814201D205F074FD11480068C06B8047C3
:20278000211AA1F54871090806D30B4A011B891A090828BF00F548740A482146FBF7B4F8B1
:2027A00098BD06490120087098BDC0469F1B0020201B0020FFF6C2FF00093D00C52E00203D
:2027C000381700202D08010038B517481749007818B90846007828B906E00846007830F0EC
:2027E0007F0001D005F03CFD114D68688047114C0C3C2178A278914207D10F4AA96812786F
:20280000D20803D28847012038BDA968884705F013FFA078FDF740F9012804BFA078207064
:2028200005F0FCFA38BDC04658150020C62E0020C0150020EC190020C32E00202DE9F84395
:2028400080461848077817B9174D287810B90120BDE8F883154E7068804781466888012417
:20286000B8F1000F0ED1214603464FF6FF72B9404A40104068807BB170B9002004F000FB3C
:20288000044609E018B9204604F0FAFA68882146B940084380B26880B16848468847204655
:2028A000BDE8F883B01600209C0A0020C01500202DE9F8438146EFF31188202080F3118878
:2028C000174D154C134F012605F11C000660A4F114000660F86A016A14208847D9F8100072
:2028E000810C14BF000C04202060386802682321002090470948066054F8180C20F4C02068
:2029000040F4803044F8180C2E6088F31188BDE8F883C046840100101820094080022443AC
:202920000000244330B504460D4642F20900ADF12C0D09A902F054F89DF8240008B342F202
:202940000B000DF10E0102F04BF800230094BDF80E00029300040190684602F023FD04467C
:2029600004A942F2030002F03BF804F0B5FB024604A9B4FBF5F06843241AE0B202F060F95B
:2029800006E042F20D0003A902F02AF89DF80C000BB030BD2DE9F843194D064628780C4612
:2029A0009846012805D0687A012818BF6FF0010024D162600A20208001F0BEFB071C1CD4BB
:2029C000A77005F027FF8146204604F095FA0446484605F01BFF04F0FF04012C06D03846B6
:2029E000012101F093F96FF0010706E005EB8705A83545F8088C45F8146C3846BDE8F88366
:202A0000A00A0020F0B50546194C2878ADF11C0DE9281CD028BB002694F8520084F856601A
:202A200002281ED104AF6946384602F0DBFE5220314605F0C7F82046C06820B1026812B1A9
:202A4000384669469047042003F06CFD09E094F85600401C84F85600C0B2032801D104F096
:202A6000AFFA8C34216809B12846884707B0F0BD7C1400202DE9F04107461748174CC01F24
:202A800006786068804780461549A268087886281CD1104D05F12A021088401C1080872036
:202AA000087005F0FDFCA16840468847082004F013FCE879B04207D127B90020FEF7FAFE0F
:202AC000BDE8F0811B20F9E7E920F7E740469047BDE8F081401A0020182E0020C015002096
:202AE000C62E00202DE9FC4716460C46054604F0A5FC164F814678688047804603F042FC11
:202B00008246B2002146484605F0FAFC504604F06DFF02E02D1D241DADB23046411ECEB244
:202B200078B128466946042203F0AAFD68462146042204F007FC0028ECD005490120487052
:202B40000870B96840468847BDE8FC87C0150020141700200CB44FF07F4343F460034FEA8B
:202B60004102D21A1BD24FEA105040EA013010F5807024BF400801F580114FEA50200029CC
:202B800048BF40F000404FEA4101490DB1F560710CD4FF290DD240EAC1500CBC7047DB43B7
:202BA0001A40024305D0D8430CBC704700200CBC704701F00041FF204FEAC05008430CBCBB
:202BC0007047FEE72DE9F8430024002B16460F468046254606D5002FC3F1000302D57F427E
:202BE000761E2D2599463846494602F01BFE0CA0405CB7FBF9F7002F04F1010408F8010DD7
:202C0000F1D1A64205DD3021301B401E08F8011DFBD10DB108F8015D4046BDE8F883C0467C
:202C2000303132333435363738396162636465660000704730B5401E4FF00004ADF12C0D1E
:202C40000AD0401E04D0401E20D1F6F74DFF1DE000F026F8044619E001A821462422082311
:202C600005F098FD06940D4DADF8144009490794012201AB05F1780005F088FD064A234680
:202C80002C2105F19C00009305F094FD20460BB030BDC046F93B01008D510000B80F00202E
:202CA00098B5164C94F8E100002710B91448007860B105F0AFFD94F8E310002906BF0121F3
:202CC00084F8E310012705F0A1FD0FB1002098BD022003F065FD0E20FCF72CFE094A106808
:202CE00048B909494020C86008600127D761002084F8E20098BD012098BDC046B80F0020FB
:202D000066A4010004800C402C500C40F8B516460C46054605F07EFD07461CB3641E1AD072
:202D2000641E15D0641E0FD0601E0BD1306828B1012807D1802002F0E1F915E0802004F00A
:202D400001FE11E0032410E030780A4908700BE03088688208E00120EE68687406F16000DA
:202D6000E86001E0306828608324384605F04EFD2046F8BD080B002038B5042905462CDAEC
:202D800005F07CFC0346084605F072FB134C0246022904EB450000F10400017012BF032964
:202DA000002141702068D9B203F042F804F0F4F850B904F12400044605F072FA01280CD14E
:202DC000204605F059FC38BD04F12400044605F067FA10B9204605F04DFC38BDA818002053
:202DE0002DE9F843174C04F1240108688846074628B300261D25387D35281BD14046394634
:202E0000324602F011FF787E30F07F0005D194F82F00401E84F82F0004E094F82E00401E0D
:202E200084F82E007D7057F80C9C384600F0AAFB4F4602E03E4657F80C7C002FDBD1BDE89F
:202E4000F883C046700D002038B5164D95F8B41001290FD003280BD013480078812804DB49
:202E60008428B8BF49F6404419DB4FF4FA5416E0002414E0032844F6206410D00B48006855
:202E800090F8690058B105F06DFB0A224FF4FA6390FBF2F15143401A58432418A4B2A5F8E9
:202EA000B64038BDA82A0020870F0020700D002070B544688668D4F8A40004F05EFC154808
:202EC00000250C30056040F80C5C114805607068FCF7A2FA04F1100005F03CFC04F12C0014
:202EE00005F03CFC04F1600005F040FC207818B904F17C0005F03AFC04F1C80004F05EFB10
:202F000005F088FC84F8DC5005F080FC70BDC0461004054204280040164880B507683FB331
:202F200015498B6803EA5300C00E21D2134A106880081DD2486880081AD21068096810F0E6
:202F4000050F4FEA114101F0F00101F5E0710AD1B9420DD2190F38BF40F00100D90E38BFC6
:202F600040F0040003E0B94202D920F00500106080BDC04628500940AC3F00500000094057
:202F80002DE9F04180461748243007680E46ADF1300DBFB13869A8B1B8F1000F12D08EB190
:202FA00006208DF828000125ADF82A500022ADF82C2002AC00943C690AAB93E803001A238F
:202FC000A04708B100200AE002A940460C22FDF77BFC05A930460E22FDF776FC28460CB099
:202FE000BDE8F081D4110020F8B50646B06801687568886B20F4FA6088631349086820F433
:203000000070086005F006FC104C0746207820B1022003F069F900202070384605F0F6FB44
:2030200005F0F8FBA96B11B905F0F0FBF8BD0021A96305F0EBFB686B296BEB68091A2963C4
:203040006A6B30469847F8BD30100040BA2E0020F8B5844640F6FF741CF8013B002210E087
:20306000481B401E10F8015B7F1E01F8015BF9D103E01CF8010B01F8010B521C5B08082A64
:20308000EADA5808F5D21CF8010B1CF8015B05F00F07FF1CC5F30315122F45EA001508D161
:2030A0001CF8016B300A24BF1CF8010B60F3DF16F719AC42D4D1F8BDB0B5184C05460F464A
:2030C000101C28D00DE03868E06397F82700394640F0040087F8270004F14C0003F01EF9A2
:2030E000E76BD7B1F8688542EDD014E0386888B13868C06885420DD139680868386091F8A6
:20310000270040F0040081F8270004F14C0003F005F900E03F68002FE8D1B0BDA00A0020DC
:20312000084610B500F0005100F00400084321D0012003F00DFD114C012813D00E480168C5
:203140003220B0FBF1F2012A8CBFB0FBF1F101212046A0F12404204605F014FB204605F086
:203160004DFB10BD064805F041F906492046D8380839086010BDC04610A501008C0B00200F
:2031800069390000081004409EB5144C606880472146134C2289E38893421CD0114B1F785F
:2031A000CFB9114B89681F7837F07F0714D1E28088471027E088ADF8007001A9ADF80400D9
:2031C00009880DF10203198008480068426AE068694690479EBD896888479EBDC015002025
:2031E000E0190020C42E0020C62E0020381700202DE9F843DFF85880044608EB440000F1AF
:203200001805008B894604F08BF8074611480678AFB12A883846002105F03AFA00253C70F1
:2032200041467D700A5D381D494604F033FE3046394600F055FC40B92846BDE8F8838DF868
:20324000004068461A21FDF787FE1A20BDE8F883749B0100B016002010B5164A144C92F86D
:203260003D0094F8401048B91348006860B9012082F83D00202005F033F805E0481CC0B265
:20328000042884F840000DD00C49A1310A784FF4707304F1200003FA02F101F2636104F0EA
:2032A00015FC10BD202002F065FCFCF771F910BDA02D002038190020700D0020A00E0020AA
:2032C00010B5044600212822ADF1280D6846FEF77BFF134911226846FDF7F6FA05208DF8B9
:2032E00012008DF8114000218DF8151001208DF816100B228DF81700FF208DF818000A20A0
:203300008DF8130080208DF814000DF11900FEF75BFF044918206A460BF062FF0AB010BD5E
:20332000EB9F010009F700002DE998430446A76E9946904607B1B8470020022100EA090709
:2033400001EA0801002F08BF002917D104F1600106C909EA020708EA0101002F08BF00293E
:203360000CD161680978022910D100EA09000821002801EA080108BF002907D004F17000B6
:2033800080E8000304F1400005F03CFABDE89883C8B50146164AC87AB8B992F83170906BA5
:2033A0002FB3401F401DC6781EB1CA7F03799A4202D07F1EF6D1C8BD8A7FC270CA880280F7
:2033C000CA7F0271097B8170C8BD92F83070506B6FB120382030867F3EB1CA7FC37F9A422F
:2033E00003D12022FDF770FAC8BD7F1EF2D1C8BDCC10002038B5012003F0AAFB012820D034
:20340000114DD5F82401C4681048342101220023A047002808BF002014D0286803F094FD4F
:2034200004F024FC0B4A0A4D93681168D060C01AA1EB910105FB00F3180C884228BF011C4B
:203440001160012038BDC0468000001000A00C4040420F00642E002098B50446207B00F0FE
:203460000F00022824D100F013FFA168081A8108114800F10C021768002F14BFFB6840F6F6
:20348000C41303F57A728A4212D20A4A12686FF050448C420CD3C91AB1FBF2F3012B8CBF68
:2034A000B1FBF2F10121C83005F06CF9012098BD002098BD10A50100A00A0020001F06B4C5
:2034C00080B290B5082803AFADF10C0D22DB3A78B0F5805F1EDA00F18851091F0C686B469A
:2034E0001C6049685960BDF800108A420BD17988BDF80230994206D1B988BDF804309942DA
:2035000008BF012007D0BDF80610401A083880B20828DDDA002003B0BDE8904002B07047BD
:2035200010B50446012002F025FB208900280CBFEB2000201249607091F83F00C20824BFE2
:2035400020F0040081F83F00820809D2400813D32B202070EB236370204600F069FD0BE0A9
:2035600091F83F0000F0FD0081F83F00217C6078C1F3001104F016FC204604F0A9FE10BDD0
:203580006C2C002080B501460A7D012A05D0152A03D0252A18BF352A02D1087E000919D38B
:2035A000087EC3091BD2012A18BF152A01D1000909D24F781B2F04D0094807B10E30805CCD
:2035C00002E0232000E0312008700648007800F087FA80BD4A7808461146FDF7BDFC80BD58
:2035E00073A00100B016002030B5174C054605F12801ADF1140D04F1AA0003F09BFB08B37D
:20360000EF2309208DF801306B688DF800005A781978181D01EB0221ADF802102A890178D7
:20362000082A8DF8041014BF94F8E600C07805F11C018DF805000DF1070005F000F8684605
:20364000FAF7E2FF05B030BDA00E002010B504460320ADF1180D04F128018DF8020000206E
:203660008DF8030001A804F0EDFF6068007804F11C018DF80C000DF10D0004F0E0FF04F183
:20368000280003F0C5FC58B14FF6FF7453206946ADF80040F3F72CFE044920460A310880FC
:2036A0000DF10200FAF7B0FF06B010BD4A0F002070B5164D286808B104F0E6FE144C60689D
:2036C00080470C3DE9690A68002616710968E961A16888470A4A0B49107810B90846007817
:2036E00060B1167008460670FCF784FC06480078012803D030460146F3F7F6FC70BDC0466E
:20370000C22E0020C42E00209E1B0020182E0020C0150020F8B50025114C1348A5604FF481
:20372000700665600068E660C06B80470D49C0F1FF3008600D48C76865700FB90C49C16079
:203740000C480570012001F0CDFE08B104F088FD304601F003FAE068FEF7FCFFF8BDC0463A
:20376000201B00200830044038170020B0190020B13C0100C52E002070B5164604460D1C25
:2037800008BF052426D034F07F0001D004F05CF8002C18BF032407D155F80C0C18B915F842
:2037A000020CFF2804D00524284604F01EFD11E0012E094805F8024C03D0294602F064FE08
:2037C00002E0294603F05AFF20464FF40041FCF75BFD0024204670BDB819002030B5044640
:2037E000606800252062ADF1140DA5657820A4F84C0094F82C0025650F2807D004F12C019F
:2038000020460122F6F79EFC08B116E0284694F83C10FF2901D1A16D21B104F13C01204631
:20382000FBF792FA48B92B4601208DF80C30032101AA00902046F0F7B1FA05B030BD0000BD
:203840002DE9FC41144C154F06468846700809D320684568002101220B461FFA88F00090F8
:203860003846A847B00809D3206845680021022201231FFA88F000903846A847F00809D347
:2038800020681FFA88F600210C220223446800963846A047BDE8FC81A401001000A00C402B
:2038A0000246F8B5084611464C68203821D0401E1CD0401E18BF6FF001001ED18D6804F0BA
:2038C000A9FF0E4E07463068016928688847B0F1FF3FF8D10025A564606C401EE064256568
:2038E0003846A56304F092FF2846F8BD0021084601E00121002084F82D10F8BDD0010010B9
:20390000012898B523D1012003F022F901281ED004F0C4F9114C012104F1D800017004F095
:2039200089FD800915D20C4800683222B2FBF0F707B90F46083C3034204603F0DFFE204694
:20394000394604F01FFF204604F058FF01E002F097FC002098BDC04610A50100C00F00209F
:20396000F8B51549154A134D36395B320B681778E91C0978002F0CBF1C695C6901EB810147
:2039800064182679002101E0491CC9B28E42D8BF4FF6FF700DDD23680A4602EB42029B1866
:2039A00093F900209042EFD1B3F801002881B3F80100F8BDE01900206A1700205A0F0020D0
:2039C00038B5154C04F1180005461C3000F06CFF03F05EFC042003F07FFCA07E032801D1A0
:2039E000607EA0B105F14501E120F3F781FC05F14601E720F3F77CFC084894F85F1000788B
:203A0000884204D005F14701E820F3F771FC2846FAF7FAFD38BDC046E42C0020870F002034
:203A20002DE9B841DFF85080144CFC224146AC3CAC392046FCF748FF002102220B46181997
:203A400003278D3000F8031F41707F1E8170F9D1521E03F10903F2D104F1AC0503272846EB
:203A60004146182204F016FA18357F1EF7D10220A070BDE8B881C046BC9D0100E827002030
:203A800038B50120124C114D94F8A11085F83D000F2917D00F490870202004F021FC94F899
:203AA000A1200E490C4835F81220886201F1200091F84010491C5143490001F2A32103F07A
:203AC000CFFA38BD02F092FC38BDC04638190020A00E002020150020F9FB0000A02D002038
:203AE00070B502460D4632F07F0004D110460022FFF742FE70BD04F0DFFC104908398C7848
:203B0000A5F10C06FF2802D0C96A40184478FF2C02D103F099FE0DE0104603F0E5FF0146D4
:203B20002A46FF20B072204602F05CFB20B1284604F05BFB012070BD002070BDB819002010
:203B400000B5ADF1240DADF80000ADF80210116801A8016051684160002002460D49069054
:203B6000887D8DF80C200D318DF80D000B680DF10E0003604B684360097A017218208DF8D4
:203B80001C2005498DF81D206A460BF029FBC0B209B000BDD49F0100B55C000098B5154BF0
:203BA0001B1D18680004070C21D003F091F9104991F90720824205DD10F1800FB8BF6FF0B2
:203BC0007F00C8718C88BC4210D80A68D3F8D40F801A801C1F2888BF1F203F1B4008C74067
:203BE0004FF6FF70E719B84238BF071C8F8098BDA82E00203010094008B51348134A144948
:203C00000078801E0A2807D8DFE800F01814100614100614100609C004F0C0FD11E010684D
:203C20008008FCD250688008FCD20AE008688008FCD306E008688008FCD202E010688008E1
:203C4000FCD3F5F751FF08BD9C10002034600C4038600C4070B5002124220823ADF1280D7A
:203C6000684604F0B3FD0F4C012529466A468DF8185004F1140004F0A5FD01F0D3FB261DC4
:203C8000304604F0F5FA00203146257301F0EAFB05492060FF2008700449002008700AB0C2
:203CA00070BDC046502D0020B92E0020B82E002070B5134C60688047124900250646487888
:203CC0004D70A168820808D2C00816D33046884728460146F3F708FA70BD304688470A485F
:203CE0000078012803D001202946F3F7FDF9606880470646FAF728FEA1683046884770BD73
:203D0000C0150020201B00209E1B0020B0B50F46044604F07FFD05461148EC3890F8C710DF
:203D2000C90803D390F8C610A14215D0B0F8C430012101FA04F21A430A4BA0F8C420181DA4
:203D4000026804F10C0399408A430260006818B917B1022001F0D2F9284604F057FDB0BDEB
:203D60008C0B0020081004401549096821280ADC212819D00C380FD00D380FD0001F0FD0BB
:203D8000C01E0FD01AE0253810D0001F10D0401E10D0401E10D011E0086870474868704735
:203DA00088687047C8687047086970474869704788697047C8697047086A70470020704755
:203DC000F0010020F8B50646B08815460F46FDF777F80446002D02D4281B0A2806DB336850
:203DE000291B38460BA201F099FA0419B08978B1002D06D4B06804F085F9291B401D884255
:203E000006DCB368291B384603A201F087FA04192046F8BD257000C0282725732729000008
:203E2000F8B50746C81D01F00705C610002F4FF0010000FA05F0A0F1010C14BF00290020B8
:203E400019D00020BEB17F1E33460246941B17F8011FB4F1FF3F08D10DB10CEA010104E058
:203E600001F1FF04401C2140C0B20029F8D15B1E02F10102EAD1F8BD38B505466C68D4F875
:203E8000A810237A002203B9012263689847D4F8BC00D4F8C010814211D08069C4F8BC00F9
:203EA000D4F8BC102846FDF753FAB0F1FF3F0ED10320207204F12C0004F05CFC38BD0020C6
:203EC000C4F8A800C4F8BC00022002F00DFA38BD70B5F0F78BFC124D68688047064603F02E
:203EE00091FF104C94F9D60004F0E4F802F0E0FE04F0D6F803F07AFF03F06CFFA9683046C0
:203F0000884794F8D70000F0A7FC04F1BD015220F3F7EEF904F0BEFA08B9FFF7FBFB70BD60
:203F2000C0150020A00E002038B50C4620B141680122A240114201D1022038BD914341604F
:203F40000E480025231800EB8401C1F8945003F140010978FF291ABF406850F8211044F092
:203F600020410548F9F780FF20464FF0FF3103F0B1FC284638BDC046007FC7672C26002027
:203F80001248134908B54FF42C72FCF79DFC4FF00451002081F89003012081F87903022049
:203FA00081F87503032081F87703042081F8AE03052081F8AB03062081F88103072081F89D
:203FC0004D030448C1F8C00308BDC0461C0400213C000000CD05002198B5124CE2685168E0
:203FE000496839B110B102F0C9FDE268506840688047E2685268906808B9D7688FB10A49AD
:204000001C310F68002FFCD000230B6010B18047E0684268D06800B180470448503802F063
:204020006BFF98BDA00A00200010044051000706144BB0B5997B03EB81010A69017801F020
:204040007F014D000170AC185219527803EB82052F6907B19A732278141103EB84031F6C98
:204060002FB90C290CDA1821FCF776FFB0BD02F00F0257F8221011B904F0F2F8B0BD8847C7
:20408000B0BDC046B016002038B50546012001F071FD124C2046143000F006FC288900283C
:2040A0000CBFEB200020687094F83F00C10824BF00F0FB0084F83F0080080BD394F83F00E4
:2040C00000F0FD0084F83F00297C6878C1F3001103F068FE284604F0FBF838BD6C2C002093
:2040E0002DE9F041054612480E46002100782960012802D00120F2F7F7FF0E4C606880477A
:204100003768804630463FB16A687968914203DC38463F68002FF8D1056030682F608542FF
:2041200001D1FDF73FFBA16840468847BDE8F0819E1B0020C0150020134A38B5B2F8C45035
:204140004FF6FF71A9421BD00024012000FA04F32B4212D05940B2F8C4300C4D1940A2F8CC
:20416000C410291D0A6804F10C03984010430860022003F0E7FB204638BD641C0F2CE5DB4F
:204180006FF0010038BDC046A00A00200810044038B5044642F209000DF1020100F020FC1D
:2041A0009DF8020050B19DF8020002281AD1A08894F82710FEF7B6FB054606E042F20D00B8
:2041C000694600F00DFC9DF80050284600F044FB0020A4F87C5094F82130607013B110208C
:2041E00004F086F838BD38B5046845682068002808BF4FF0FF301FD004F00CFB21680029D1
:2042000054BF491E0021216004F000FB206890B904F12C0004F09EFA04F1480004F0A6FA44
:2042200004F1640004F0A2FA6868FBF7F5F804F1180003F0C3F9002038BD00002DE9B84106
:20424000124C0546201D00688047804603F056F96F7E002F08BF6B6807D069682A69AF6839
:20426000091A5218B9180B466960E968286105F11402184601F0D0FF012768686F76A168DC
:20428000A86040468847BDE8B881C046C015002010B504F0BFFA104C217829B10F490C68DB
:2042A00004F0B4FA204610BD04F0B0FA03F0A8FE0B4A002303F012FE626A002314001B1841
:2042C0004FF07A024FF0905044EB0104C11842EB04021046001C10BDA00A00200430044043
:2042E00000093D00B0B5134C6068628800B325880021AA42C8BF01210B46AA42C6BFA91A67
:2043000001F58061A91A8FB28FB1012B03D0A1183A46083109E0A118C2F58062083104F0A9
:2043200012F9606804F108012A4604F00CF96580B0BDC0469406002038B51248104C016825
:20434000114D0C40E1430160A10907D34068800904D328464FF4005103F0F0FD14F4602F29
:204360000DD02846EC3800F1C0010A6804F4602400F5907014430C60002103F0DFFD38BD91
:2043800020000E00081004408C0B0020134910B5044691F83F00ADF1180D40F0020081F83B
:2043A0003F00012003F03AF9607890B9211D02A803F0E0FB03F0EAFC01460120009004F1DA
:2043C00010030193E38902AA0520F3F78FFB607010B1002103F0E6FC06B010BD6C2C0020C3
:2043E0001FB5014604208DF8000048788DF80100B1F896000DF10203ADF80C008C311846A5
:2044000003F0B8FB02F004FE60B14FF6FF7453200DF10E01ADF80E40F2F76AFF04492046C1
:204420000A3108806846FAF7EFF800901FBDC0464A0F0020134A3D321278812A01DB842ABD
:204440000FDB00F11002490892B224BF00F129018AB21228CCBF05200220801880B2C0000A
:204460000DE04201490802F5C67292B224BF02F21E218AB21228CCBF28200C20801880B2F3
:204480007047C0464A0F00202DE9F0410120104E104D307028781F469046022801D003F05A
:2044A000DFFE0024022114EA070001EA080108BF002902D103F0D4FE07E0074991F9000096
:2044C000401E08702C7003F0C1FC3470BDE8F0819E1B00209F1B00209A1B0020C8B5071CD8
:2044E00001D103F0BDFE79684878C6111FD03B89F96400204A78C2F3C3020F2A09D00A78C4
:204500001018801C80B25218834202F10201F1DC01E0801C80B2834206DB79683E8941185D
:204520007960311A398100E00020A7F85000C8BD10B5044600211C22ADF1200D6846FDF74E
:2045400043FE60788DF80000A0788DF80100E0788DF8020020791122611D8DF8030001A8C5
:20456000FCF7B2F9A07D8DF8150008B1A06906900348006881696846884708B010BDC046E9
:20458000701B0020F8B504460D46084611220021FDF71AFE94F800C0BCF1000F1AD0641C06
:2045A00000214FF0010EE078A37843EA0023207809E0C610AF5D00F00702401C0EFA02F215
:2045C000C0B23A43AA558342F3DA491C241DC9B28C45E8DCF8BD80B502465378107840EAF6
:2045E0000320C7130F7007BFC0F3062300F0FF00C0F3C323C0F30A004B70802848800DDA46
:2046000002280BDB012B0CD0022B0AD0042B08D0052B06D0062B04D0072B02D000221046ED
:2046200000E0921C4A6080BD70B5114C2068E8B1104D686880470646216894F82F000228B4
:2046400006DBA96830468847F120F5F7E5FB70BD04F1240003F012F8002394F82F00A96814
:204660002360401C84F82F003046884770BDC046700D0020C015002038B5044642F2080033
:204680000DF1020100F0ACF99DF8020040B19DF80200022817D1204601F020FB054606E0B0
:2046A00042F20C00694600F09BF99DF8005094F8200030B9284600F0CFF8A4F87C50002060
:2046C00000E00120207038BDF0B5124D00260C460746ADF1140DC5F8B061012003F091FF5A
:2046E0002868C00FF9D3286A0090686A0190A86A0290E86A03903FB13846694611F8012B2F
:20470000401E04F8012BF9D1032005B0C5F838023046F0BD504502401249D0B524310F68D4
:20472000ADF1180DCFB17E69BEB1B0B106218DF810100226ADF812600024ADF8144043888C
:20474000ADF8003042680192816802917C6904AE96E803000C226B46A047032003F056FA87
:2047600006B0D0BDD411002010B50446012001F001FA2078212804BFEB2060700D4991F877
:204780003F00C20824BF20F0040081F83F00800805D22B2020702046FFF74AFC10BD91F82F
:2047A0003F0000F0FD0081F83F006078002103F0F9FA10BD6C2C002070B5114D95F8A10000
:2047C000B5F8C6400F2810D00E483430066801F00FFC2018864208D895F8A1104FF47070AA
:2047E00088402418A41B04F57074044D284600F05BF82146284603F069F970BD802C0020F4
:20480000A00E002038190020114898B501210170022111400F4A4FF0E0471F4008BF00299E
:2048200003D092F90010491E1170044692F9000030B192F90000002806DC03F011FD03E0F3
